:020000040800F2
:1000000000060020E1010008E3010008E301000808
:10001000E3010008E3010008E3010008E301000830
:10002000E3010008E3010008E3010008752F000860
:10003000E3010008E3010008E3010008E301000810
:10004000E3010008E3010008E3010008E301000800
:10005000E3010008E30100081D32000845320008F2
:100060006D32000895320008BD320008E301000837
:10007000E3010008E3010008E3010008E3010008D0
:10008000E3010008E3010008E3010008E3010008C0
:10009000E3010008E3010008E3010008E53200087D
:1000A000E3010008E3010008E3010008E3010008A0
:1000B000B9330008E3010008E3010008E301000888
:1000C000E3010008E3010008E3010008E301000880
:1000D000E3010008E3010008E3010008E301000870
:1000E00049330008E3010008E3010008E3010008C8
:1000F000E3010008E3010008E3010008E301000850
:10010000E3010008E3010008E3010008E30100083F
:10011000E3010008E3010008E3010008E30100082F
:10012000E3010008E3010008E3010008E30100081F
:10013000E3010008E3010008E3010008E30100080F
:10014000E3010008E3010008E30100082927000893
:10015000E3010008E3010008E3010008E3010008EF
:10016000E3010008E3010008E3010008E3010008DF
:10017000E3010008E3010008E3010008E3010008CF
:10018000E3010008E3010008E3010008E3010008BF
:10019000E3010008E3010008E3010008E3010008AF
:1001A000E3010008E3010008E3010008E30100089F
:1001B000E3010008E3010008E3010008E30100088F
:1001C000E3010008E3010008E3010008E30100087F
:1001D000E3010008E3010008E3010008E30100086F
:1001E00002E000F000F8FEE772B6374880F30888B6
:1001F000364880F3098836483649086040F20000E6
:10020000CCF200004EF63471CEF200010860BFF36C
:100210004F8FBFF36F8F40F20000C0F2F0004EF638
:100220008851CEF200010860BFF34F8FBFF36F8F8C
:100230004FF00000E1EE100A4EF63C71CEF20001E4
:100240000860062080F31488BFF36F8F01F034FF3D
:1002500002F02EFE4FF055301F491B4A91423CBF21
:1002600041F8040BFAE71D49184A91423CBF41F896
:10027000040BFAE71A491B4A1B4B9A423EBF51F83E
:10028000040B42F8040BF8E700201849184A914281
:100290003CBF41F8040BFAE701F012FF02F05CFEEC
:1002A000144C154DAC4203DA54F8041B8847F9E7A7
:1002B00000F042F8114C124DAC4203DA54F8041B22
:1002C0008847F9E701F0FABE00060020002200206E
:1002D0000000000808ED00E00000002000060020FB
:1002E0008037000800220020402200204022002009
:1002F000602E0020E0010008E0010008E001000895
:10030000E00100082DE9F04F2DED108AC1F80CD066
:10031000C3689D46BDEC108ABDE8F08F002383F3CF
:1003200011882846A047002001F076FAFEE701F088
:1003300005FA00DFFEE7000038B500F069FB01F0C8
:100340008BFE054601F0AEFE0446D8B90F4B9D4228
:100350001AD001339D4218BF044641F2883504BFCC
:1003600001240025002001F081FE0CB100F076F898
:1003700000F004FD00F0B2FB284600F0BFF800F0EA
:100380006DF8F9E70025EDE70546EBE7010007B05A
:1003900008B500F075FBA0F120035842584108BD94
:1003A00007B541F21203022101A8ADF8043000F0B4
:1003B00085FB03B05DF804FB38B5302383F3118867
:1003C000174803680BB101F0F3FA164A14480023EA
:1003D0004FF47A7101F0E2FA002383F31188124C92
:1003E000236813B12368013B2360636813B163681A
:1003F000013B63600D4D2B7833B963687BB90220F4
:1004000000F036FC322363602B78032B07D163683E
:100410002BB9022000F02CFC4FF47A73636038BDD6
:1004200040220020B9030008602300205822002049
:10043000084B187003280CD8DFE800F00805020804
:10044000022000F00BBC022000F0FEBB024B002299
:100450005A6070475822002060230020234B244A12
:1004600010B51C46196801313FD004339342F9D1CD
:100470006268A24239D31F4B9B6803F1006303F506
:1004800040439A4231D2002000F042FB0220FFF7A5
:10049000CFFF194B1A6C00221A64196E1A66196E76
:1004A000596C5A64596E5A665A6E5A6942F0800203
:1004B0005A615A6922F080025A615A691A6942F0F7
:1004C00000521A611A6922F000521A611B6972B651
:1004D0004FF0E0233021C3F8084DD4E9003281F316
:1004E00011889D4683F30888104710BD00C000089E
:1004F00020C0000800220020003802402DE9F04F03
:1005000093B0AA4B00902022FF210AA89D6800F01A
:10051000DFFBA74A1378A3B9A64801210360117035
:10052000302383F3118803680BB101F041FAA24A2A
:10053000A04800234FF47A7101F030FA002383F3CE
:100540001188009B13B19D4B009A1A609C4A009C35
:100550001378032B1EBF00231370984A4FF0000A34
:1005600018BF5360D3465646D146012000F076FBB3
:1005700024B1924B1B68002B00F01182002000F088
:100580007FFA0390039B002BF2DB012000F05CFB61
:10059000039B213B162BE8D801A252F823F000BFA1
:1005A000FD05000825060008B90600086B050008CF
:1005B0006B0500086B0500084307000813090008D5
:1005C0002D0800088F080008B7080008DD0800089B
:1005D0006B050008EF0800086B05000861090008BA
:1005E0009D0600086B050008A5090008090600081B
:1005F0009D0600086B0500088F0800080220FFF721
:10060000C7FE002840F0F581009B0221BAF1000FDF
:1006100008BF1C4605A841F21233ADF8143000F0B3
:100620004DFAA2E74FF47A7000F02AFA071EEBDBCE
:100630000220FFF7ADFE0028E6D0013F052F00F2B3
:10064000DA81DFE807F0030A0D101336052305935E
:10065000042105A800F032FA17E054480421F9E714
:1006600058480421F6E758480421F3E74FF01C08E6
:10067000404600F04FFA08F104080590042105A84F
:1006800000F01CFAB8F12C0FF2D1012000FA07F7A4
:1006900047EA0B0B5FFA8BFB4FF0000900F064FB9D
:1006A00026B10BF00B030B2B08BF0024FFF778FEDD
:1006B0005BE746480421CDE7002EA5D00BF00B03E5
:1006C0000B2BA1D10220FFF763FE074600289BD029
:1006D000012000F01DFA0220FFF7AAFE00261FFAF3
:1006E00086F8404600F024FA044690B100214046C6
:1006F00000F02EFA01360028F1D1BA46044641F244
:100700001213022105A8ADF814303E4600F0D6F9C8
:100710002BE70120FFF78CFE2546244B9B68AB425C
:1007200007D9284600F0F6F9013040F0678104351A
:10073000F3E7234B00251D70204BBA465D603E4613
:10074000ACE7002E3FF460AF0BF00B030B2B7FF4F4
:100750005BAF0220FFF76CFE322000F091F9B0F1A0
:100760000008FFF651AF18F003077FF44DAF0F4AB2
:10077000926808EB050393423FF646AFB8F5807FD9
:100780003FF742AF124B0193B84523DD4FF47A7027
:1007900000F076F90390039A002AFFF635AF019B2B
:1007A000039A03F8012B0137EDE700BF0022002078
:1007B0005C23002040220020B903000860230020B1
:1007C0005822002004220020082200200C220020B1
:1007D0005C220020C820FFF7DBFD074600283FF41D
:1007E00013AF1F2D11D8C5F1200242450AAB25F0E9
:1007F000030028BF424683490192184400F042FAA0
:10080000019A8048FF2100F063FA4FEAA8037D496E
:100810000193C8F38702284600F062FA06460028D2
:100820003FF46DAF019B05EB830537E70220FFF72F
:10083000AFFD00283FF4E8AE00F0B6F900283FF421
:10084000E3AE0027B846704B9B68BB4218D91F2FF8
:1008500011D80A9B01330ED027F0030312AA1344C8
:1008600053F8203C05934046042205A900F0B0FA55
:1008700004378046E7E7384600F04CF90590F2E788
:10088000CDF81480042105A800F018F906E700232C
:10089000642104A8049300F007F900287FF4B4AEA3
:1008A0000220FFF775FD00283FF4AEAE049800F07B
:1008B00063F90590E6E70023642104A8049300F09F
:1008C000F3F800287FF4A0AE0220FFF761FD0028B6
:1008D0003FF49AAE049800F05FF9EAE70220FFF7D0
:1008E00057FD00283FF490AE00F06EF9E1E70220DA
:1008F000FFF74EFD00283FF487AE05A9142000F055
:1009000069F904210746049004A800F0D7F8394695
:10091000B9E7322000F0B4F8071EFFF675AEBB074A
:100920007FF472AE384A926807EB090393423FF6B0
:100930006BAE0220FFF72CFD00283FF465AE27F0D8
:1009400003074F44B9453FF4A9AE484600F0E2F82A
:100950000421059005A800F0B1F809F10409F1E7B8
:100960004FF47A70FFF714FD00283FF44DAE00F00D
:100970001BF9002844D00A9B01330BD008220AA996
:10098000002000F0ADF900283AD02022FF210AA86B
:1009900000F09EF9FFF704FD1C4800F043FF13B080
:1009A000BDE8F08F002E3FF42FAE0BF00B030B2BA6
:1009B0007FF42AAE0023642105A8059300F074F8A3
:1009C000074600287FF420AE0220FFF7E1FC8046B6
:1009D00000283FF419AEFFF7E3FC41F2883000F045
:1009E00021FF059800F0F2F9464600F0BDF93C46BB
:1009F000BBE5064652E64FF0000905E6BA467EE63C
:100A000037467CE65C22002000220020A086010000
:100A10007047000070B50F4B1B780133DBB2012B20
:100A20000C4611D80C4D29684FF47A730E6AA2FB5C
:100A30000332014622462846B047844204D1074B80
:100A400000221A70012070BD4FF4FA7000F0EAFE27
:100A50000020F8E710220020082600209423002020
:100A600070B504464FF47A76412C254628BF4125BF
:100A700006FB05F000F0D6FE641BF5D170BD00004A
:100A800007B50023024601210DF107008DF807305C
:100A9000FFF7C0FF20B19DF8070003B05DF804FB2D
:100AA0004FF0FF30F9E700000A4608B50421FFF7D0
:100AB000B1FF80F00100C0B2404208BD30B4054C27
:100AC0002368DD69044B0A46AC460146204630BC2B
:100AD000604700BF08260020A086010070B501F025
:100AE000C1F9094E094D30800024286833888342BB
:100AF00008D901F0B1F92B6804440133B4F5404F33
:100B00002B60F2D370BD00BF962300206823002025
:100B100001F056BA00F1006000F5404000687047EF
:100B200000F10060920000F5404001F0E1B90000E2
:100B3000054B1A68054B1B889B1A834202D9104447
:100B400001F08AB900207047682300209623002016
:100B500038B5084D044629B128682044BDE838401E
:100B600001F09AB92868204401F07EF90028F3D0FA
:100B700038BD00BF6823002010F003030AD1B0F590
:100B8000047F05D200F10050A0F51040D0F80038E5
:100B9000184670470023FBE700F10050A0F5104015
:100BA000D0F8100A70470000064991F8243033B19C
:100BB0000023086A81F824300822FFF7B1BF012022
:100BC000704700BF6C230020014B1868704700BFBE
:100BD000002004E070B5194B1D68194B0138C5F3AE
:100BE0000B0408442D0C04221E88A6420BD15C681D
:100BF0000A46013C824213460FD214F9016F4EB1EE
:100C000002F8016BF6E7013A03F10803ECD18142E7
:100C10000B4602D22C2203F8012B0A4A052416881F
:100C2000AE4204D1984284BF967803F8016B013C30
:100C300002F10402F3D1581A70BD00BF002004E095
:100C40009C34000888340008022802BF024B4FF091
:100C500080729A61704700BF00000240022802BF04
:100C6000024B4FF480729A61704700BF000002404F
:100C7000022801BF024A536983F4807353617047AD
:100C80000000024010B50023934203D0CC5CC45452
:100C90000133F9E710BD000010B5013810F9013F2C
:100CA0003BB191F900409C4203D11AB10131013AA4
:100CB000F4E71AB191F90020981A10BD1046FCE72C
:100CC00003460246D01A12F9011B0029FAD17047D7
:100CD00002440346934202D003F8011BFAE770472F
:100CE0002DE9F8431F4D144695F824200746884601
:100CF00052BBDFF870909CB395F824302BB92022BA
:100D0000FF2148462F62FFF7E3FF95F82400C0F16A
:100D10000802A24228BF2246D6B24146920005EB05
:100D20008000FFF7AFFF95F82430A41B1E44F6B2F5
:100D3000082E17449044E4B285F82460DBD1FFF715
:100D400033FF0028D7D108E02B6A03EB82038342EC
:100D5000CFD0FFF729FF0028CBD10020BDE8F883D2
:100D60000120FBE76C230020024B1A78024B1A701B
:100D7000704700BF942300201022002010B5104CB3
:100D8000104800F0B5F821460E4800F0DDF8246860
:100D9000626DD2F8043843F00203C2F804384FF40D
:100DA0007A70FFF75DFE0849204600F0D3F9626DC6
:100DB000D2F8043823F00203C2F8043810BD00BF93
:100DC00068350008082600207035000870470000CC
:100DD00030B5094D0A4491420DD011F8013B5840FD
:100DE000082340F30004013B2C4013F0FF0384EA86
:100DF0005000F6D1EFE730BD2083B8ED02684368BC
:100E00001143016003B118477047000013B5446BEC
:100E1000D4F894341A681178042915D1217C022958
:100E200012D11979128901238B4013420CD101A9E7
:100E300004F14C0001F0F8FED4F89444019B2179B0
:100E40000246206800F0D0F902B010BD143001F065
:100E50007BBE00004FF0FF33143001F075BE000080
:100E60004C3001F04DBF00004FF0FF334C3001F02B
:100E700047BF0000143001F049BE00004FF0FF31C1
:100E8000143001F043BE00004C3001F019BF0000E7
:100E90004FF0FF324C3001F013BF000000207047CC
:100EA00010B5D0F894341A6811780429044617D183
:100EB000017C022914D15979528901238B401342B4
:100EC0000ED1143001F0DCFD024648B1D4F8944450
:100ED0004FF4807361792068BDE8104000F072B96A
:100EE00010BD0000406BFFF7DBBF00007047000043
:100EF0007FB5124B036000234360C0E90233012534
:100F000002260F4B057404460290019300F18402FF
:100F1000294600964FF48073143001F08DFD094B83
:100F20000294CDE9006304F523724FF480732946DF
:100F300004F14C0001F054FE04B070BDBC34000854
:100F4000E50E00080D0E00080B68302282F31188B0
:100F50000A7903EB820290614A79093243F8220050
:100F60008A7912B103EB820398610223C0F89414CA
:100F70000374002080F311887047000038B5037FA8
:100F8000044613B190F85430ABB9201D012502215D
:100F9000FFF734FF04F1140025776FF0010100F032
:100FA00069FC84F8545004F14C006FF00101BDE875
:100FB000384000F05FBC38BD10B501210446043054
:100FC000FFF71CFF0023237784F8543010BD000086
:100FD00038B504460025143001F046FD04F14C00FC
:100FE000257701F015FE201D84F854500121FFF7EC
:100FF00005FF2046BDE83840FFF752BF90F8443067
:1010000003F06003202B07D190F84520212A4FF0F0
:10101000000303D81F2A06D800207047222AFBD1DC
:10102000C0E90E3303E0034A82630722C26303640C
:10103000012070471122002037B5D0F894341A6887
:101040001178042904461AD1017C022917D1197993
:10105000128901238B40134211D100F14C0528461F
:1010600001F096FE58B101A9284601F0DDFDD4F843
:101070009444019B21790246206800F0B5F803B042
:1010800030BD0000F0B500EB810385B09E690446D9
:101090000D46FEB1302383F3118804EB8507301D24
:1010A0000821FFF7ABFEFB685B691B6806F14C008B
:1010B0001BB1019001F0C6FD019803A901F0B4FD38
:1010C000024648B1039B2946204600F08DF80023D4
:1010D00083F3118805B0F0BDFB685A691268002AD5
:1010E000F5D01B8A013B1340F1D104F14402EAE739
:1010F000093138B550F82140DCB1302383F3118831
:10110000D4F894241368527903EB8203DB689B695B
:101110005D6845B104216018FFF770FE294604F1AF
:10112000140001F0B7FC2046FFF7BAFE002383F35A
:10113000118838BD7047000001F016B80123037014
:101140000023C0E90133C36183620362C362436267
:101150000363704738B50446302383F311880025B4
:10116000C0E90355C0E90555416001F00DF80223BF
:10117000237085F31188284638BD000070B500EB58
:10118000810305465069DA600E46144618B11022F4
:101190000021FFF79DFDA06918B110220021FFF783
:1011A00097FD31462846BDE8704001F0B7B8000011
:1011B000826802F0011282600022C0E9042282618A
:1011C00001F038B9F0B400EB81044789E4680125E7
:1011D000A4698D403D43458123600023A260636084
:1011E000F0BC01F053B90000F0B400EB81040789B2
:1011F000E468012564698D403D4305812360002337
:10120000A2606360F0BC01F0CDB9000070B50223AC
:10121000002504460370C0E90255C0E90455C564C1
:10122000856180F8345001F015F863681B6823B1BC
:1012300029462046BDE87040184770BD0378052B4D
:1012400010B504460AD080F8503005230370436877
:101250001B680BB1042198470023A36010BD000058
:101260000178052906D190F85020436802701B6868
:1012700003B118477047000070B590F83430044649
:1012800013B1002380F8343004F14402204601F009
:10129000F3F863689B68B3B994F8443013F06005C1
:1012A00035D00021204601F093FB0021204601F0BB
:1012B00085FB63681B6813B1062120469847062307
:1012C00084F8343070BD204698470028E4D0B4F844
:1012D0004A30E26B9A4288BFE36394F94430E56B8D
:1012E000002B4FF0300380F20381002D00F0F280DC
:1012F000092284F8342083F311880021D4E90E23D5
:101300002046FFF771FF002383F31188DAE794F892
:10131000452003F07F0343EA022340F20232934266
:1013200000F0C58021D8B3F5807F48D00DD8012BBF
:101330003FD0022B00F09380002BB2D104F14C027D
:10134000A2630222E2632364C1E7B3F5817F00F068
:101350009B80B3F5407FA4D194F84630012BA0D1F7
:10136000B4F84C3043F0020332E0B3F5006F4DD0D7
:1013700017D8B3F5A06F31D0A3F5C063012B90D877
:10138000636894F846205E6894F84710B4F84830D3
:101390002046B047002884D04368A3630368E36312
:1013A0001AE0B3F5106F36D040F6024293427FF454
:1013B00078AF5C4BA3630223E3630023C3E794F895
:1013C0004630012B7FF46DAFB4F84C3023F00203AC
:1013D000C4E90E55A4F84C30256478E7B4F84430DD
:1013E000B3F5A06F0ED194F8463084F84E30204605
:1013F00000F088FF63681B6813B1012120469847FD
:10140000032323700023C4E90E339CE704F14F0348
:10141000A3630123C3E72378042B10D1302383F384
:1014200011882046FFF7C4FE85F311880321636805
:1014300084F84F5021701B680BB12046984794F8F0
:101440004630002BDED084F84F30042323706368CD
:101450001B68002BD6D0022120469847D2E794F88B
:1014600048301D0603F00F0120460AD500F0F6FFB4
:10147000012804D002287FF414AF2B4B9AE72B4BA2
:1014800098E700F0DDFFF3E794F84630002B7FF497
:1014900008AF94F8483013F00F01B3D01A06204675
:1014A00002D501F0A9FAADE701F09CFAAAE794F899
:1014B0004630002B7FF4F5AE94F8483013F00F015E
:1014C000A0D01B06204602D501F082FA9AE701F06F
:1014D00075FA97E7142284F8342083F311882B4699
:1014E0002A4629462046FFF76DFE85F31188E9E676
:1014F0005DB1152284F8342083F311880021D4E9EA
:101500000E232046FFF75EFEFDE60B2284F8342012
:1015100083F311882B462A4629462046FFF764FEAE
:10152000E3E700BFEC340008E4340008E8340008C6
:1015300038B590F834300446002B3ED0063BDAB282
:101540000F2A34D80F2B32D8DFE803F037313108B7
:10155000223231313131313131313737C56BB0F869
:101560004A309D4214D2C3681B8AB5FBF3F203FBD9
:1015700012556DB9302383F311882B462A4629462C
:10158000FFF732FE85F311880A2384F834300EE029
:10159000142384F83430302383F3118800231A464F
:1015A00019462046FFF70EFE002383F3118838BD4D
:1015B000036C03B198470023E7E70021204601F0C0
:1015C00007FA0021204601F0F9F963681B6813B19E
:1015D0000621204698470623D7E7000010B590F86B
:1015E0003430142B044629D017D8062B05D001D847
:1015F0001BB110BD093B022BFBD80021204601F096
:10160000E7F90021204601F0D9F963681B6813B19E
:10161000062120469847062319E0152BE9D10B2314
:1016200080F83430302383F3118800231A4619469A
:10163000FFF7DAFD002383F31188DAE7C3689B69BB
:101640005B68002BD5D1036C03B19847002384F865
:101650003430CEE700230375826803691B689968FC
:101660009142FBD25A680360426010605860704734
:1016700000230375826803691B6899689142FBD84F
:101680005A680360426010605860704708B50846A9
:10169000302383F311880B7D032B05D0042B0DD051
:1016A0002BB983F3118808BD8B6900221A604FF0B3
:1016B000FF338361FFF7CEFF0023F2E7D1E9003269
:1016C00013605A60F3E70000FFF7C4BF054BD96809
:1016D0000875186802681A60536001220275D860A4
:1016E000FEF710BE9823002030B50C4BDD684B1C74
:1016F00087B004460FD02B46094A684600F04EF9E1
:101700002046FFF7E3FF009B13B1684600F050F955
:10171000A86907B030BDFFF7D9FFF9E7982300208B
:101720008D160008044B1A68DB6890689B68984225
:1017300094BF00200120704798230020084B10B56B
:101740001C68D86822681A60536001222275DC6028
:10175000FFF78EFF01462046BDE81040FEF7D2BDE0
:101760009823002038B5074C074908480123002575
:101770002370656001F044FB0223237085F3118818
:1017800038BD00BF00260020F43400089823002054
:1017900000F044B9034A516853685B1A9842FBD879
:1017A000704700BF001000E08B60022308618B824D
:1017B000084670478368A3F1840243F8142C026939
:1017C00043F8442C426943F8402C094A43F8242C3E
:1017D000C26843F8182C022203F80C2C002203F8EC
:1017E0000B2C044A43F8102CA3F12000704700BFD3
:1017F0001D0300089823002008B5FFF7DBFFBDE8B4
:101800000840FFF761BF0000024BDB6898610F20C2
:10181000FFF75CBF98230020302383F31188FFF784
:10182000F3BF000008B50146302383F31188082078
:10183000FFF75AFF002383F3118808BD064BDB68CE
:1018400039B1426818605A60136043600420FFF7A2
:101850004BBF4FF0FF307047982300200368984239
:1018600006D01A680260506099611846FFF72CBFD5
:101870007047000038B504460D462068844200D108
:1018800038BD036823605C608561FFF71DFFF4E7E6
:1018900010B503689C68A2420CD85C688A600B6033
:1018A0004C602160596099688A1A9A604FF0FF3342
:1018B000836010BD1B68121BECE700000A2938BFCB
:1018C0000A2170B504460D460A26601901F092FA05
:1018D00001F07EFA041BA54203D8751C2E4604466F
:1018E000F3E70A2E04D9BDE87040012001F0C8BA20
:1018F00070BD0000F8B5144B0D46D96103F110011D
:1019000041600A2A1969826038BF0A220160486072
:101910001861A818144601F05FFA0A2701F058FA76
:10192000431BA342064606D37C1C281901F062FA29
:1019300027463546F2E70A2F04D9BDE8F8400120D2
:1019400001F09EBAF8BD00BF98230020F8B5064606
:101950000D4601F03DFA0F4A134653F8107F9F429F
:1019600006D12A4601463046BDE8F840FFF7C2BF1F
:10197000D169BB68441A2C1928BF2C46A34202D94E
:101980002946FFF79BFF224631460348BDE8F84051
:10199000FFF77EBF98230020A823002010B4C0E9E1
:1019A000032300235DF8044B4361FFF7CFBF000022
:1019B00010B5194C236998420DD0D0E900328168E6
:1019C00013605A609A680A449A60002303604FF0DB
:1019D000FF33A36110BD2346026843F8102F536004
:1019E0000022026022699A4203D1BDE8104001F052
:1019F000FBB9936881680B44936001F0E9F92269AF
:101A0000E1699268441AA242E4D91144BDE8104049
:101A1000091AFFF753BF00BF982300202DE9F047B4
:101A2000DFF8BC8008F110072C4ED8F8105001F0F8
:101A3000CFF9D8F81C40AA68031B9A423ED8144438
:101A4000D5E900324FF00009C8F81C4013605A6015
:101A5000C5F80090D8F81030B34201D101F0C4F9B4
:101A600089F31188D5E9033128469847302383F359
:101A700011886B69002BD8D001F0AAF96A69A0EB34
:101A800004094A4582460DD2022001F0F9F90022EC
:101A9000D8F81030B34208D151462846BDE8F04787
:101AA000FFF728BF121A2244F2E712EB090938BFE8
:101AB0004A4629463846FFF7EBFEB5E7D8F810301E
:101AC000B34208D01444211AC8F81C00A960BDE82C
:101AD000F047FFF7F3BEBDE8F08700BFA823002062
:101AE0009823002000207047FEE7000070470000A8
:101AF0004FF0FF307047000002290CD0032904D0BA
:101B00000129074818BF00207047032A05D8054857
:101B100000EBC2007047044870470020704700BFC8
:101B2000CC350008202200208035000870B59AB01E
:101B30000546084601A9144600F0C2F801A8FFF7BF
:101B4000BFF8431C5B00C5E9003400222370032367
:101B50006370C6B201AB02341046D1B28E4204F1BA
:101B6000020401D81AB070BD13F8011B04F8021C5E
:101B700004F8010C0132F0E708B5302383F3118833
:101B80000348FFF759FA002383F3118808BD00BF0B
:101B90000826002090F8443003F01F02012A07D1E4
:101BA00090F845200B2A03D10023C0E90E3315E03D
:101BB00003F06003202B08D1B0F848302BB990F81F
:101BC0004520212A03D81F2A04D8FFF717BA222A52
:101BD000EBD0FAE7034A82630722C2630364012061
:101BE000704700BF1822002007B5052917D8DFE885
:101BF00001F0191603191920302383F31188104AB4
:101C000001900121FFF7BAFA01980E4A0221FFF76D
:101C1000B5FA0D48FFF7DCF9002383F3118803B010
:101C20005DF804FB302383F311880748FFF7A6F91A
:101C3000F2E7302383F311880348FFF7BDF9EBE7A0
:101C400020350008443500080826002038B50C4D22
:101C50000C4C0D492A4604F10800FFF767FF05F117
:101C6000CA0204F110000949FFF760FF05F5CA72C6
:101C700004F118000649BDE83840FFF757BF00BF20
:101C8000D02A002020220020003500080A35000854
:101C90001535000870B5044608460D46FFF710F8E4
:101CA000C6B22046013403780BB9184670BD3246DF
:101CB0002946FEF7F1FF0028F3D10120F6E70000E6
:101CC0002DE9F04705460C46FEF7FAFF2B49C6B250
:101CD0002846FFF7DFFF08B10636F6B22849284646
:101CE000FFF7D8FF08B11036F6B2632E0BD8DFF835
:101CF0008C80DFF88C90234FDFF894A02E7846B9C3
:101D00002670BDE8F08729462046BDE8F04701F07F
:101D10009DBB252E2ED1072241462846FEF7BCFF4B
:101D200070B9194B224603F10C0153F8040B42F829
:101D3000040B8B42F9D11B78137007350D34DDE7A6
:101D4000082249462846FEF7A7FF98B90F4BA21C68
:101D5000197809090232C95D02F8041C13F8011B45
:101D600001F00F015345C95D02F8031CF0D118348E
:101D70000835C3E704F8016B0135BFE7EC3500080F
:101D80001535000802360008F4350008107AFF1FE8
:101D90001C7AFF1FBFF34F8F024AD368DB03FCD4CA
:101DA000704700BF003C024008B5094B1B7873B96F
:101DB000FFF7F0FF074B1A69002ABFBF064A5A60B7
:101DC00002F188325A601A6822F480621A6008BDF3
:101DD0002E2D0020003C02402301674508B50B4B27
:101DE0001B7893B9FFF7D6FF094B1A6942F00042FE
:101DF0001A611A6842F480521A601A6822F48052FA
:101E00001A601A6842F480621A6008BD2E2D002004
:101E1000003C02400B28F0B516D80C4C0C49237836
:101E20007BB90C4D0E460C234FF0006255F8047B35
:101E300046F8042B013B13F0FF033A44F6D101238B
:101E4000237051F82000F0BD0020FCE7602D002039
:101E5000302D002014360008014B53F82000704745
:101E6000143600080C2070470B2810B5044601D921
:101E7000002010BDFFF7CEFF064B53F82430184466
:101E8000C21A0BB90120F4E712680132F0D1043B09
:101E9000F6E700BF143600080B2810B5044621D819
:101EA000FFF778FFFFF780FF0F4AF323D360C300EB
:101EB000DBB243F4007343F002031361136943F48C
:101EC00080331361FFF766FFFFF7A4FF074B53F85A
:101ED000241000F0D9F8FFF781FF2046BDE810403C
:101EE000FFF7C2BF002010BD003C024014360008BE
:101EF000F8B512F00103144642D18218B2F1016F15
:101F000057D82D4B1B6813F0010352D02B4DFFF710
:101F10004BFFF323EB60FFF73DFF40F20127032C5B
:101F200015D824F001046618244C401A40F2011719
:101F3000B142236900EB010524D123F001032361A1
:101F4000FFF74CFF0120F8BD043C0430E7E78307AE
:101F5000E7D12B6923F440732B612B693B432B6141
:101F600051F8046B0660BFF34F8FFFF713FF036850
:101F70009E42E9D02B6923F001032B61FFF72EFF6E
:101F80000020E0E723F44073236123693B4323618E
:101F90000B882B80BFF34F8FFFF7FCFE2D8831F8A5
:101FA000023BADB2AB42C3D0236923F001032361EE
:101FB000E4E71846C7E700BF00380240003C024093
:101FC000084908B50B7828B11BB9FFF7EDFE0123CE
:101FD0000B7008BD002BFCD0BDE808400870FFF76F
:101FE000FDBE00BF2E2D002010B50244064BD2B21C
:101FF000904200D110BD441C00B253F8200041F8BB
:10200000040BE0B2F4E700BF502800400F4B30B59E
:102010001C6F240407D41C6F44F400741C671C6FED
:1020200044F400441C670A4C236843F48073236023
:102030000244084BD2B2904200D130BD441C00B2E1
:1020400051F8045B43F82050E0B2F4E70038024056
:10205000007000405028004007B5012201A900206F
:10206000FFF7C2FF019803B05DF804FB13B5044607
:10207000FFF7F2FFA04205D0012201A90020019440
:10208000FFF7C4FF02B010BD70470000034B1A6891
:102090001AB9034AD2F874281A607047642D0020D8
:1020A0000030024008B5FFF7F1FF024B1868C0F39B
:1020B000407008BD642D002070470000FEE700005E
:1020C0000A4B0B480B4A90420BD30B4BDA1C121AEB
:1020D000C11E22F003028B4238BF00220021FEF70E
:1020E000F7BD53F8041B40F8041BECE7C0370008A9
:1020F000602E0020602E0020602E002070B5D0E9F8
:1021000015439E6800224FF0FF3504EB4213510146
:10211000D3F800090028BEBFD3F8000940F0804082
:10212000C3F80009D3F8000B0028BEBFD3F8000B9A
:1021300040F08040C3F8000B013263189642C3F8A8
:102140000859C3F8085BE0D24FF00113C4F81C38FB
:1021500070BD0000890141F02001016103699B0607
:10216000FCD41220FFF716BB10B5054C2046FEF735
:10217000E5FF4FF0A0436365024BA36510BD00BFB0
:10218000682D00206836000870B50378012B0546DD
:1021900050D12A4B446D98421BD1294B5A6B42F0C7
:1021A00080025A635A6D42F080025A655A6D5A692C
:1021B00042F080025A615A6922F080025A610E216F
:1021C00043205B6900F022FC1E4BE3601E4BC4F809
:1021D00000380023C4F8003EC02323606E6D4FF426
:1021E0000413A3633369002BFCDA012333610C2051
:1021F000FFF7D0FA3369DB07FCD41220FFF7CAFAE5
:102200003369002BFCDA0026A6602846FFF776FF2C
:102210006B68C4F81068DB68C4F81468C4F81C68FC
:102220004BB90A4BA3614FF0FF336361A36843F0DE
:102230000103A36070BD064BF4E700BF682D0020CA
:10224000003802404014004003002002003C30C02F
:10225000083C30C0F8B5446D054600212046FFF724
:1022600079FFA96D00234FF001128F68C4F834384C
:102270004FF00066C4F81C284FF0FF3004EB431207
:1022800001339F42C2F80069C2F8006BC2F8080926
:10229000C2F8080BF2D20B686A6DEB65636210231B
:1022A0001361166916F01006FBD11220FFF772FABF
:1022B000D4F8003823F4FE63C4F80038A36943F46B
:1022C000402343F01003A3610923C4F81038C4F875
:1022D00014380A4BEB604FF0C043C4F8103B084B76
:1022E000C4F8003BC4F81069C4F80039EB6D03F181
:1022F000100243F48013EA65A362F8BD4436000877
:1023000040800010426D90F84E10D2F8003823F44F
:10231000FE6343EA0113C2F8003870472DE9F84321
:1023200000EB8103456DDA68166806F00306731E3C
:10233000022B05EB41130C4680460FFA81F94FEA58
:1023400041104FF00001C3F8101B4FF0010104F1E0
:10235000100398BFB60401FA03F391698EBF334EA0
:1023600006F1805606F5004600293AD0578A04F156
:102370005801490137436F50D5F81C180B43C5F875
:102380001C382B180021C3F8101953690127611E4E
:10239000A7409BB3138A928B9B08012A88BF5343A3
:1023A000D8F85C20981842EA034301F1400205EB9B
:1023B0008202C8F85C00214653602846FFF7CAFE37
:1023C00008EB8900C3681B8A43EA845348346401DC
:1023D0001E432E51D5F81C381F43C5F81C78BDE8A4
:1023E000F88305EB4917D7F8001B21F40041C7F823
:1023F000001BD5F81C1821EA0303C0E704F13F03D2
:1024000005EB83030A4A5A6028462146FFF7A2FEDD
:1024100005EB4910D0F8003923F40043C0F8003927
:10242000D5F81C3823EA0707D7E700BF0080001063
:1024300000040002826D1268C265FFF75FBE0000F3
:102440005831436D49015B5813F4004004D013F434
:10245000001F0CBF02200120704700004831436D6F
:1024600049015B5813F4004004D013F4001F0CBF63
:10247000022001207047000000EB8101CB68196A3F
:102480000B6813604B6853607047000000EB8103DA
:1024900030B5DD68AA691368D36019B9402B84BFD1
:1024A000402313606B8A1468426D1C44013CB4FBEA
:1024B000F3F46343033323F0030302EB411043EAD5
:1024C000C44343F0C043C0F8103B2B6803F0030340
:1024D000012B09B20ED1D2F8083802EB411013F4E7
:1024E000807FD0F8003B14BF43F0805343F000538B
:1024F000C0F8003B02EB4112D2F8003B43F004432A
:10250000C2F8003B30BD00002DE9F041244D6E6D56
:1025100006EB40130446D3F8087BC3F8087B380762
:102520000AD5D6F81438190706D505EB84032146D9
:10253000DB6828465B689847FA071FD5D6F8143839
:10254000DB071BD505EB8403D968CCB98B69488AB6
:102550005A68B2FBF0F600FB16228AB91868DA68EE
:1025600090420DD2121AC3E90024302383F311885C
:102570000B482146FFF78AFF84F31188BDE8F081FC
:10258000012303FA04F26B8923EA02036B81CB680F
:10259000002BF3D021460248BDE8F041184700BFA8
:1025A000682D002000EB810370B5DD68436D6C6918
:1025B0002668E6604A0156BB1A444FF40020C2F870
:1025C00010092A6802F00302012A0AB20ED1D3F8D8
:1025D000080803EB421410F4807FD4F8000914BFFC
:1025E00040F0805040F00050C4F8000903EB421264
:1025F000D2F8000940F00440C2F80009D3F83408CA
:10260000012202FA01F10143C3F8341870BD19B96F
:10261000402E84BF4020206020682E8A8419013C0F
:10262000B4FBF6F440EAC44040F000501A44C6E758
:102630002DE9F8433B4D6E6D06EB40130446D3F88D
:102640000889C3F8088918F0010F4FEA40171AD01B
:10265000D6F81038DB0716D505EB8003D9684B692F
:102660001868DA68904230D2121A4FF000091A60E6
:10267000C3F80490302383F3118821462846FFF7DE
:1026800091FF89F3118818F0800F1CD0D6F83438E8
:102690000126A640334216D005EB84036D6DD3F8B6
:1026A0000CC0DCF814200134E4B2D2F800E005EBF1
:1026B00004342F445168714515D3D5F8343823EAD2
:1026C0000606C5F83468BDE8F883012303FA04F26E
:1026D0002B8923EA02032B818B68002BD3D0214660
:1026E00028469847CFE7BCF81000AEEB01038342C1
:1026F00028BF0346D7F8180980B2B3EB800FE2D8A1
:102700009068A0F1040959F8048FC4F80080A0EB88
:1027100009089844B8F1040FF5D818440B449060A8
:102720005360C7E7682D00202DE9F74FA24C656D77
:102730006E69AB691E4016F480586E6107D0204662
:10274000FEF764FD03B0BDE8F04F00F047BC002E7B
:1027500012DAD5F8003E98489B071EBFD5F8003E18
:1027600023F00303C5F8003ED5F8043823F0010335
:10277000C5F80438FEF774FD370505D58E48FFF718
:10278000BDFC8D48FEF75AFDB0040CD5D5F80838CD
:1027900013F0060FEB6823F470530CBF43F410538F
:1027A00043F4A053EB6031071BD56368DB681BB9AA
:1027B000AB6923F00803AB612378052B0CD1D5F866
:1027C000003E7D489A071EBFD5F8003E23F0030364
:1027D000C5F8003EFEF744FD6368DB680BB1764840
:1027E0009847F30274D4B70227D5D4F85490DFF891
:1027F000C8B100274FF0010A09EB4712D2F8003B9D
:1028000003F44023B3F5802F11D1D2F8003B002B05
:102810000DDA62890AFA07F322EA0303638104EB03
:102820008703DB68DB6813B1394658469847A36DC8
:1028300001379B68FFB29F42DED9F00617D5676D5E
:102840003A6AC2F30A1002F00F0302F4F012B2F572
:10285000802F00F08580B2F5402F08D104EB830370
:102860000022DB681B6A07F5805790426AD130036B
:10287000D5F8184813D5E10302D50020FFF744FE30
:10288000A20302D50120FFF73FFE630302D5022019
:10289000FFF73AFE270302D50320FFF735FE750345
:1028A0007FF550AFE00702D50020FFF7C1FEA1077A
:1028B00002D50120FFF7BCFE620702D50220FFF718
:1028C000B7FE23077FF53EAF0320FFF7B1FE39E7E0
:1028D000636DDFF8E4A0019300274FF00109A36DB9
:1028E0009B685FFA87FB9B453FF67DAF019B03EB3F
:1028F0004B13D3F8001901F44021B1F5802F1FD1FB
:10290000D3F8001900291BDAD3F8001941F09041DF
:10291000C3F80019D3F800190029FBDB5946606D94
:10292000FFF718FC218909FA0BF321EA030323813D
:1029300004EB8B03DB689B6813B1594650469847FC
:102940000137CCE7910708BFD7F80080072A98BF66
:1029500003F8018B02F1010298BF4FEA182884E7BF
:10296000023304EB830207F580575268D2F818C08F
:10297000DCF80820DCE9001CA1EB0C0C00218842EB
:102980000AD104EB830463689B699A6802449A60E5
:102990005A6802445A606AE711F0030F08BFD7F87B
:1029A00000808C4588BF02F8018B01F1010188BFCE
:1029B0004FEA1828E3E700BF682D0020436D03EBC2
:1029C0004111D1F8003B43F40013C1F8003B7047BC
:1029D000436D03EB4111D1F8003943F40013C1F802
:1029E00000397047436D03EB4111D1F8003B23F4EC
:1029F0000013C1F8003B7047436D03EB4111D1F860
:102A0000003923F40013C1F80039704700F1604326
:102A100003F561430901C9B283F80013012200F0F4
:102A20001F039A4043099B0003F1604303F5614390
:102A3000C3F880211A60704730B5039C01720433DB
:102A400004FB0325C0E90653049B03630021059B97
:102A5000C160C0E90000C0E90422C0E90842C0E941
:102A60000A11436330BD0000416A0022C0E904112D
:102A7000C0E90A22C2606FF00101FEF7FBBE000050
:102A8000D0E90432934201D1C2680AB9181D7047D7
:102A90000020704703691960C2680132C260C269D0
:102AA000134482690361934224BF436A0361002196
:102AB000FEF7D4BE38B504460D46E3683BB1626903
:102AC000131D1268A3621344E362002007E0237A17
:102AD00033B929462046FEF7B1FE0028EDDA38BDAD
:102AE0006FF00100FBE70000C368C269013BC360EF
:102AF0004369134482694361934224BF436A43613B
:102B000000238362036B03B11847704770B530230D
:102B1000044683F31188866A3EB9FFF7CBFF05466A
:102B200018B186F31188284670BDA36AE26A13F8CB
:102B3000015BA362934202D32046FFF7D5FF002337
:102B400083F31188EFE700002DE9F84F04460E46A5
:102B5000174698464FF0300989F311880025AA4698
:102B6000D4F828B0BBF1000F09D141462046FFF749
:102B7000A1FF20B18BF311882846BDE8F88FD4E976
:102B80000A12A7EB050B521A934528BF9346BBF1D7
:102B9000400F1BD9334601F1400251F8040B43F8B2
:102BA000040B9142F9D1A36A40334036A362403509
:102BB000D4E90A239A4202D32046FFF795FF8AF30D
:102BC0001188BD42D8D289F31188C9E730465A46E8
:102BD000FEF758F8A36A5B445E44A3625D44E7E7EE
:102BE00010B5029C0172043303FB0421C0E90613F3
:102BF0000023C0E90A33039B0363049BC460C0E95C
:102C00000000C0E90422C0E90842436310BD00008F
:102C1000026AC260426AC0E904220022C0E90A22B4
:102C20006FF00101FEF726BED0E904239A4201D1DC
:102C3000C26822B9184650F8043B0B607047002365
:102C40001846FAE7C368C2690133C3604369134495
:102C500082694361934224BF436A43610021FEF7C6
:102C6000FDBD000038B504460D46E3683BB123695D
:102C70001A1DA262E2691344E362002007E0237A8E
:102C800033B929462046FEF7D9FD0028EDDA38BDD4
:102C90006FF00100FBE7000003691960C268013AA8
:102CA000C260C269134482690361934224BF436ACC
:102CB000036100238362036B03B118477047000070
:102CC00070B530230D460446114683F31188866A99
:102CD0002EB9FFF7C7FF10B186F3118870BDA36A44
:102CE0001D70A36AE26A01339342A36204D3E169CF
:102CF00020460439FFF7D0FF002080F31188EDE76C
:102D00002DE9F84F04460D46904699464FF0300A9B
:102D10008AF311880026B346A76A4FB94946204670
:102D2000FFF7A0FF20B187F311883046BDE8F88F88
:102D3000D4E90A073A1AA8EB0607974228BF1746B4
:102D4000402F1BD905F1400355F8042B40F8042B04
:102D50009D42F9D1A36A4033A3624036D4E90A23E5
:102D60009A4204D3E16920460439FFF795FF8BF3BB
:102D700011884645D9D28AF31188CDE729463A46CB
:102D8000FDF780FFA36A3B443D44A3623E44E5E770
:102D9000D0E904239A4217D1C3689BB1836A8BB1EF
:102DA000043B9B1A0ED01360C368013BC360C36928
:102DB0001A44836902619A4224BF436A0361002373
:102DC00083620123184670470023FBE700F030B907
:102DD0004FF08043586A70474FF080430022586399
:102DE0001A610222DA6070474FF080430022DA60F5
:102DF000704700004FF0804358637047FEE70000C3
:102E000070B51B4B01630025044686B0586085628F
:102E10000E4600F0BFF804F11003C4E904334FF08C
:102E2000FF33C4E90635C4E90044A560E562FFF755
:102E3000CFFF2B460246C4E9082304F134010D4AB2
:102E4000256580232046FEF7AFFC0123E0600A4A97
:102E50000375009272680192B268CDE90223074BB4
:102E60006846CDE90435FEF7C7FC06B070BD00BF6B
:102E7000002600207436000879360008FD2D000871
:102E8000024AD36A1843D062704700BF98230020DB
:102E90004B6843608B688360CB68C3600B69436198
:102EA0004B6903628B6943620B68036070470000E3
:102EB00008B5264B26481A6940F2FF110A431A61E9
:102EC0001A6922F4FF7222F001021A611A691A6B60
:102ED0000A431A631A6D0A431A651E4A1B6D11468E
:102EE000FFF7D6FF02F11C0100F58060FFF7D0FF6D
:102EF00002F1380100F58060FFF7CAFF02F15401CA
:102F000000F58060FFF7C4FF02F1700100F58060FA
:102F1000FFF7BEFF02F18C0100F58060FFF7B8FFFC
:102F200002F1A80100F58060FFF7B2FF02F1C401D1
:102F300000F58060FFF7ACFF02F1E00100F5806072
:102F4000FFF7A6FFBDE8084000F0EEB800380240E9
:102F5000000002408036000808B500F059FAFEF77C
:102F600001FCFFF793F8BDE80840FEF76FBE0000D4
:102F700070470000EFF3098305494A6B22F0010214
:102F80004A63683383F30988002383F31188704709
:102F900000EF00E0302080F3118862B60C4B0D4A40
:102FA000D96821F4E0610904090C0A43DA60D3F816
:102FB000FC20094942F08072C3F8FC200A6842F004
:102FC00001020A602022DA7783F82200704700BFEE
:102FD00000ED00E00003FA05001000E010B530231A
:102FE00083F311880E4B5B6813F4006314D0F1EE89
:102FF000103AEFF30984683C4FF08073E361094BAA
:10300000DB6B236684F30988FEF78CFB10B1064B5B
:10301000A36110BD054BFBE783F31188F9E700BFFF
:1030200000ED00E000EF00E02F030008320300088D
:103030000F4B1A6C42F001021A641A6E42F0010240
:103040001A660C4A1B6E936843F0010393604FF0BD
:10305000804353229A624FF0FF32DA6200229A6173
:103060005A63DA605A6001225A611A60704700BFE1
:1030700000380240002004E04FF0804208B511699A
:10308000D3680B40D9B2C9439B07116107D53023E0
:1030900083F31188FEF77CFB002383F3118808BDBE
:1030A0001F4B1A696FEAC2526FEAD2521A611A694B
:1030B000C2F308021A614FF0FF301A695A69586169
:1030C00000215A6959615A691A6A62F080521A627B
:1030D0001A6A02F080521A621A6A5A6A58625A6A66
:1030E00059625A6A1A6C42F080521A641A6E42F09F
:1030F00080521A661A6E0B4A106840F48070106095
:10310000186F00F44070B0F5007F1EBF4FF48030A0
:1031100018671967536823F40073536000F054B9BB
:103120000038024000700040334B4FF080521A6468
:10313000324A4FF4404111601A6842F001021A60AD
:103140001A689107FCD59A6822F003029A602A4B0C
:103150009A6812F00C02FBD1196801F0F9011960AC
:103160009A601A6842F480321A601A689203FCD599
:103170005A6F42F001025A671F4B5A6F9007FCD5F5
:103180001F4A5A601A6842F080721A601B4A5368DC
:103190005904FCD5184B1A689201FCD5194A9A605B
:1031A000194B1A68194B9A42194B21D1194A1168C7
:1031B000194A91421CD140F205121A60144A136850
:1031C00003F00F03052BFAD10B4B9A6842F0020271
:1031D0009A609A6802F00C02082AFAD15A6C42F4FA
:1031E00080425A645A6E42F480425A665B6E70475F
:1031F00040F20572E1E700BF003802400070004075
:103200000854400700948838002004E0116400202E
:10321000003C024000ED00E041C20F41074A08B502
:10322000536903F00103536123B1054A13680BB1DD
:1032300050689847BDE80840FFF7D0BE003C014009
:10324000E02D0020074A08B5536903F002035361DB
:1032500023B1054A93680BB1D0689847BDE8084090
:10326000FFF7BCBE003C0140E02D0020074A08B536
:10327000536903F00403536123B1054A13690BB189
:1032800050699847BDE80840FFF7A8BE003C0140E0
:10329000E02D0020074A08B5536903F00803536185
:1032A00023B1054A93690BB1D0699847BDE808403E
:1032B000FFF794BE003C0140E02D0020074A08B50E
:1032C000536903F01003536123B1054A136A0BB12C
:1032D000506A9847BDE80840FFF780BE003C0140B7
:1032E000E02D0020164B10B55C6904F478725A6129
:1032F000A30604D5134A936A0BB1D06A98476006B7
:1033000004D5104A136B0BB1506B9847210604D5B6
:103310000C4A936B0BB1D06B9847E20504D5094A70
:10332000136C0BB1506C9847A30504D5054A936CF8
:103330000BB1D06C9847BDE81040FFF74FBE00BFFF
:10334000003C0140E02D0020194B10B55C6904F4ED
:103350007C425A61620504D5164A136D0BB1506D5B
:103360009847230504D5134A936D0BB1D06D984748
:10337000E00404D50F4A136E0BB1506E9847A104B8
:1033800004D50C4A936E0BB1D06E9847620404D5F5
:10339000084A136F0BB1506F9847230404D5054AB0
:1033A000936F0BB1D06F9847BDE81040FFF716BE82
:1033B000003C0140E02D002008B5FFF75DFEBDE8B0
:1033C0000840FFF70BBE0000062108B50846FFF7CE
:1033D0001DFB06210720FFF719FB06210820FFF738
:1033E00015FB06210920FFF711FB06210A20FFF734
:1033F0000DFB06211720FFF709FB06212820FFF708
:1034000005FBBDE8084007211C20FFF7FFBA0000BC
:1034100008B5FFF745FE00F00BF8FDF78DFEFDF750
:1034200065FDFFF7A5FDBDE80840FFF7CFBC000034
:103430000023054A19460133102BC2E9001102F19D
:103440000802F8D1704700BFE02D0020034611F8B4
:10345000012B03F8012B002AF9D1704753544D3347
:1034600032463F3F3F0053544D33324634307800AC
:1034700053544D3332463432780053544D33324630
:103480003434365858000000012033000010410049
:1034900001105A000310590007103100000000000D
:1034A0005C340008130400006634000819040000AE
:1034B00070340008210400007A3400080000000085
:1034C000690E0008550E0008910E00087D0E0008D8
:1034D000890E0008750E0008610E00084D0E0008E8
:1034E0009D0E000800000000010000000000000028
:1034F00063300000F0340008F02300200026002094
:103500004172647550696C6F740025424F4152449A
:10351000252D424C002553455249414C25000000C1
:10352000020000000000000085100008F1100008F3
:1035300040004000A02A0020B02A00200200000025
:10354000000000000300000000000000351100082A
:103550000000000010000000C02A00200000000051
:103560000100000000000000682D002001010200A1
:10357000E91B0008F91A0008951B0008791B0008D0
:10358000430000008835000809024300020100C022
:1035900032090400000102020100052400100105A7
:1035A000240100010424020205240600010705820B
:1035B000030800FF09040100020A000000070501DA
:1035C00002400000070581024000000012000000D8
:1035D000D4350008120110010200004009124157C1
:1035E00000020102030100000403090425424F41C7
:1035F000524425007370656564796265656634764A
:10360000340030313233343536373839414243446F
:10361000454600000040000000400000004000005F
:103620000040000000000100000002000000020055
:103630000000020000000200000002000000020082
:103640000000020000000000791200083115000897
:10365000DD15000840004000C82D0020C82D0020C6
:1036600001000000D82D0020800000004001000073
:10367000030000006D61696E0069646C6500000004
:103680000001812A00000000AAAAAAAA00010024C1
:10369000FFFE00000000000000A00A000000000182
:1036A00000000000AAAAAAAA00000001FFFF000073
:1036B00000000000000000000000001000000000FA
:1036C000AAAAAAAA00000010FFFF00000000000044
:1036D000000000000000000000000000AAAAAAAA42
:1036E00000000000FFFF00000000000000000000DC
:1036F0000000000000000000AAAAAAAA0000000022
:10370000FFFF0000000000000000000000000000BB
:1037100000000000AAAAAAAA00000000FFFF000003
:103720000000000000000000000000000000000099
:10373000AAAAAAAA00000000FFFF000000000000E3
:103740000000000000000000000000000A0000006F
:103750000000000003000000000000000000000066
:103760000000000000000000000000000000000059
:103770000000000000000000000000000000000049
:10378000700400000000000000400F000000000076
:10379000FF009600000000080096000000000800EE
:1037A00004000000E83500080000000000000000F0
:1037B0000000000000000000000000000000000009
:1037C000FFFFFFFFFFFFFFFFFFFFFFFFFFFFFFFF09
:1037D000FFFFFFFFFFFFFFFFFFFFFFFFFFFFFFFFF9
:1037E000FFFFFFFFFFFFFFFFFFFFFFFFFFFFFFFFE9
:10C000000006002099D20008B17006080D700608DD
:10C01000797006080D700608457006089BD2000866
:10C020009BD200089BD200089BD20008457D0808DF
:10C030009BD200089BD200089BD200089BD200082C
:10C040009BD200089BD200089BD200089BD200081C
:10C050009BD200089BD20008DD88080805890808E3
:10C060002D890808558908087D8908088D30080839
:10C07000B5300808E13008080D31080839310808E2
:10C08000613108088D310808113008089BD200087A
:10C090009BD200089BD200089BD20008A589080803
:10C0A000F18A0808F58A0808098B08080D8B08082A
:10C0B000118B0808258B0808398B080819370808E0
:10C0C000C13808089BD200089BD200089BD2000808
:10C0D0009BD20008798A08088D8A0808A18A080876
:10C0E000098A08089BD200089BD200085D8B0808CB
:10C0F000618B0808758B0808798B0808B931080826
:10C100009BD200089BD200084D8B08089BD20008E8
:10C11000B58A0808C98A08089BD200089BD2000883
:10C12000E53108080D320808393208086532080878
:10C13000913208089BD200089BD200089BD20008CD
:10C140009BD200089BD200089BD20008718408088B
:10C15000B9320808E532080811330808DD8A0808F2
:10C160009BD200089BD200089BD200089BD20008FB
:10C170009BD200089BD200089BD200089BD20008EB
:10C180009BD200089BD200089BD200089BD20008DB
:10C190009BD200089BD200089BD200089BD20008CB
:10C1A0009BD200089BD200089BD200089BD20008BB
:10C1B0009BD200089BD200089BD200089BD20008AB
:10C1C0009BD200089BD200089BD200089BD200089B
:10C1D0009BD200089BD200089BD200089BD200088B
:10C1E0002DE700080DF70008D95B0108A9AD02088A
:10C1F000712B0408094A04085DA9040821B1040848
:10C2000059B40408ED130508692F0508B1A2050803
:10C2100009B00508A96106082D6706082DF0060873
:10C220008110070871650708498C0708D5A207081F
:10C2300081D0070849D60708000000000000000070
:10C2400081F0004102E000BF83F0004330B54FEAC7
:10C2500041044FEA430594EA050F08BF90EA020F34
:10C260001FBF54EA000C55EA020C7FEA645C7FEAC7
:10C27000655C00F0E2804FEA5454D4EB5555B8BFEA
:10C280006D420CDD2C4480EA020281EA030382EA5B
:10C29000000083EA010180EA020281EA0303362DED
:10C2A00088BF30BD11F0004F4FEA01314FF4801CC0
:10C2B0004CEA113102D0404261EB410113F0004FD2
:10C2C0004FEA03334CEA133302D0524263EB430389
:10C2D00094EA050F00F0A780A4F10104D5F1200E27
:10C2E0000DDB02FA0EFC22FA05F2801841F1000182
:10C2F00003FA0EF2801843FA05F359410EE0A5F156
:10C3000020050EF1200E012A03FA0EFC28BF4CF086
:10C31000020C43FA05F3C01851EBE37101F000453C
:10C3200007D54FF0000EDCF1000C7EEB00006EEB49
:10C330000101B1F5801F1BD3B1F5001F0CD34908D3
:10C340005FEA30004FEA3C0C04F101044FEA44522A
:10C3500012F5800F80F09A80BCF1004F08BF5FEAB1
:10C36000500C50F1000041EB045141EA050130BD91
:10C370005FEA4C0C404141EB0101013C28BFB1F5A3
:10C38000801FE9D291F0000F04BF01460020B1FAEE
:10C3900081F308BF2033A3F10B03B3F120020CDAC1
:10C3A0000C3208DD02F1140CC2F10C0201FA0CF09F
:10C3B00021FA02F10CE002F11402D8BFC2F1200C04
:10C3C00001FA02F120FA0CFCDCBF41EA0C019040BA
:10C3D000E41AA2BF01EB0451294330BD6FEA040403
:10C3E0001F3C1CDA0C340EDC04F11404C4F12002EE
:10C3F00020FA04F001FA02F340EA030021FA04F300
:10C4000045EA030130BDC4F10C04C4F1200220FA56
:10C4100002F001FA04F340EA0300294630BD21FA94
:10C4200004F0294630BD94F0000F83F4801306BF5A
:10C4300081F480110134013D4EE77FEA645C18BF4E
:10C440007FEA655C29D094EA050F08BF90EA020FE5
:10C4500005D054EA000C04BF1946104630BD91EADD
:10C46000030F1EBF0021002030BD5FEA545C05D1E0
:10C470004000494128BF41F0004130BD14F580041F
:10C480003CBF01F5801130BD01F0004545F0FE4193
:10C4900041F470014FF0000030BD7FEA645C1ABFC8
:10C4A000194610467FEA655C1CBF0B46024650EAFF
:10C4B000013406BF52EA033591EA030F41F400212B
:10C4C00030BD00BF90F0000F04BF0021704730B5B1
:10C4D0004FF4806404F132044FF000054FF0000186
:10C4E00050E700BF90F0000F04BF0021704730B547
:10C4F0004FF4806404F1320410F0004548BF40421C
:10C500004FF000013EE700BF42004FEAE2014FEA70
:10C5100031014FEA02701FBF12F07F4393F07F4F4B
:10C5200081F06051704732F07F4208BF704793F04E
:10C530007F4F04BF41F40021704730B54FF4607461
:10C5400001F0004521F000411CE700BF50EA010264
:10C5500008BF704730B54FF000050AE050EA01020D
:10C5600008BF704730B511F0004502D5404261EB7D
:10C5700041014FF4806404F132045FEA915C3FF4BE
:10C58000D8AE4FF003025FEADC0C18BF03325FEA5B
:10C59000DC0C18BF033202EBDC02C2F1200300FA0C
:10C5A00003FC20FA02F001FA03FE40EA0E0021FA31
:10C5B00002F11444BDE600BF70B54FF0FF0C4CF41F
:10C5C000E06C1CEA11541DBF1CEA135594EA0C0FD1
:10C5D00095EA0C0F00F0DEF82C4481EA030621EA0C
:10C5E0004C5123EA4C5350EA013518BF52EA033547
:10C5F00041F4801143F4801338D0A0FB02CE4FF0F9
:10C600000005E1FB02E506F00042E0FB03E54FF028
:10C610000006E1FB03569CF0000F18BF4EF0010E20
:10C62000A4F1FF04B6F5007F64F5407404D25FEA1C
:10C630004E0E6D4146EB060642EAC62141EA5551CF
:10C640004FEAC52040EA5E504FEACE2EB4F1FD0C11
:10C6500088BFBCF5E06F1ED8BEF1004F08BF5FEA8F
:10C66000500E50F1000041EB045170BD06F0004641
:10C6700046EA010140EA020081EA0301B4EB5C04EE
:10C68000C2BFD4EB0C0541EA045170BD41F48011E6
:10C690004FF0000E013C00F3AB8014F1360FDEBF0B
:10C6A000002001F0004170BDC4F10004203C35DAE7
:10C6B0000C341BDC04F11404C4F1200500FA05F36A
:10C6C00020FA04F001FA05F240EA020001F000420B
:10C6D00021F0004110EBD37021FA04F642EB060181
:10C6E0005EEA430E08BF20EAD37070BDC4F10C04AB
:10C6F000C4F1200500FA04F320FA05F001FA04F26F
:10C7000040EA020001F0004110EBD37041F100015A
:10C710005EEA430E08BF20EAD37070BDC4F1200565
:10C7200000FA05F24EEA020E20FA04F301FA05F2CD
:10C7300043EA020321FA04F001F0004121FA04F275
:10C7400020EA020000EBD3705EEA430E08BF20EA45
:10C75000D37070BD94F0000F0FD101F0004640007F
:10C7600041EB010111F4801F08BF013CF7D041EA01
:10C77000060195F0000F18BF704703F00046520005
:10C7800043EB030313F4801F08BF013DF7D043EAD6
:10C790000603704794EA0C0F0CEA135518BF95EA8C
:10C7A0000C0F0CD050EA410618BF52EA4306D1D113
:10C7B00081EA030101F000414FF0000070BD50EA32
:10C7C000410606BF1046194652EA430619D094EABC
:10C7D0000C0F02D150EA013613D195EA0C0F05D1A6
:10C7E00052EA03361CBF104619460AD181EA0301FA
:10C7F00001F0004141F0FE4141F470014FF00000B2
:10C8000070BD41F0FE4141F4780170BD70B54FF04C
:10C81000FF0C4CF4E06C1CEA11541DBF1CEA1355CC
:10C8200094EA0C0F95EA0C0F00F0A7F8A4EB0504AE
:10C8300081EA030E52EA03354FEA013100F08880A5
:10C840004FEA03334FF0805545EA131343EA12636E
:10C850004FEA022245EA111545EA10654FEA002623
:10C860000EF000419D4208BF964244F1FD0404F5DC
:10C87000407402D25B084FEA3202B61A65EB030538
:10C880005B084FEA32024FF480104FF4002CB6EBF5
:10C89000020E75EB030E22BFB61A754640EA0C0075
:10C8A0005B084FEA3202B6EB020E75EB030E22BFB5
:10C8B000B61A754640EA5C005B084FEA3202B6EBF6
:10C8C000020E75EB030E22BFB61A754640EA9C00B5
:10C8D0005B084FEA3202B6EB020E75EB030E22BF85
:10C8E000B61A754640EADC0055EA060E18D04FEA43
:10C8F000051545EA16754FEA06164FEAC30343EAE3
:10C9000052734FEAC2025FEA1C1CC0D111F4801FAF
:10C910000BD141EA00014FF000004FF0004CB6E7A8
:10C9200011F4801F04BF01430020B4F1FD0C88BF47
:10C93000BCF5E06F3FF6AFAEB5EB030C04BFB6EB52
:10C94000020C5FEA500C50F1000041EB045170BD45
:10C950000EF0004E4EEA113114EB5C04C2BFD4EB72
:10C960000C0541EA045170BD41F480114FF0000EF6
:10C97000013C90E645EA060E8DE60CEA135594EA72
:10C980000C0F08BF95EA0C0F3FF43BAF94EA0C0F75
:10C990000AD150EA01347FF434AF95EA0C0F7FF4EA
:10C9A00025AF104619462CE795EA0C0F06D152EA3E
:10C9B00003353FF4FDAE1046194622E750EA410622
:10C9C00018BF52EA43067FF4C5AE50EA41047FF433
:10C9D0000DAF52EA43057FF4EBAE12E74FF0FF3C98
:10C9E00006E000BF4FF0010C02E000BF4FF0010C69
:10C9F0004DF804CD4FEA410C7FEA6C5C4FEA430CE2
:10CA000018BF7FEA6C5C1BD001B050EA410C0CBF30
:10CA100052EA430C91EA030F02BF90EA020F002092
:10CA2000704710F1000F91EA030F58BF994208BFF9
:10CA300090422CBFD8176FEAE37040F001007047B6
:10CA40004FEA410C7FEA6C5C02D150EA013C07D10D
:10CA50004FEA430C7FEA6C5CD6D152EA033CD3D058
:10CA60005DF8040B704700BF8446104662468C4652
:10CA70001946634600E000BF01B5FFF7B7FF002885
:10CA800048BF10F1000F01BD4DF808EDFFF7F4FFAE
:10CA90000CBF012000205DF808FB00BF4DF808ED39
:10CAA000FFF7EAFF34BF012000205DF808FB00BF5C
:10CAB0004DF808EDFFF7E0FF94BF012000205DF87E
:10CAC00008FB00BF4DF808EDFFF7CEFF94BF012033
:10CAD00000205DF808FB00BF4DF808EDFFF7C4FF2C
:10CAE00034BF012000205DF808FB00BF4FEA410C75
:10CAF0007FEA6C5C02D150EA013C0AD14FEA430C58
:10CB00007FEA6C5C02D152EA033C02D14FF0000094
:10CB100070474FF0010070474FEA410212F50012D2
:10CB200015D211D56FF47873B3EB625212D94FEA74
:10CB3000C12343F0004343EA505311F0004F23FA5E
:10CB400002F018BF404270474FF00000704750EAB3
:10CB5000013005D111F0004008BF6FF00040704770
:10CB60004FF00000704700BF4A0011D212F50012CA
:10CB700011D20DD56FF47873B3EB62520ED44FEA35
:10CB8000C12343F0004343EA505323FA02F07047B5
:10CB90004FF00000704750EA013002D14FF0FF30F3
:10CBA00070474FF0000070474FEA4102B2F1E04396
:10CBB00024BFB3F5001CDCF1FE5C0DD901F0004C84
:10CBC0004FEAC0024CEA5070B2F1004F40EB8300D4
:10CBD00008BF20F00100704711F0804F21D113F100
:10CBE0003872BCBF01F00040704741F480114FEA39
:10CBF0005252C2F11802C2F1200C10FA0CF320FAC2
:10CC000002F018BF40F001004FEAC1234FEAD323DE
:10CC100003FA0CFC40EA0C0023FA02F34FEA430348
:10CC2000CCE77FEA625307D150EA01331EBF4FF0D1
:10CC3000FE4040F44000704701F0004040F0FE40EC
:10CC400040F40000704700BF80F0004002E000BFE9
:10CC500081F0004142001FBF5FEA410392EA030FE7
:10CC60007FEA226C7FEA236C6AD04FEA1262D2EB31
:10CC70001363C1BFD218414048404140B8BF5B4236
:10CC8000192B88BF704710F0004F40F4000020F0CF
:10CC90007F4018BF404211F0004F41F4000121F0E5
:10CCA0007F4118BF494292EA030F3FD0A2F101022F
:10CCB00041FA03FC10EB0C00C3F1200301FA03F16D
:10CCC00000F0004302D5494260EB4000B0F5000F90
:10CCD00013D3B0F1807F06D340084FEA310102F14F
:10CCE0000102FE2A51D2B1F1004F40EBC25008BF01
:10CCF00020F0010040EA03007047490040EB0000CB
:10CD0000013A28BFB0F5000FEDD2B0FA80FCACF1CB
:10CD1000080CB2EB0C0200FA0CF0AABF00EBC250F8
:10CD200052421843BCBFD0401843704792F0000FE6
:10CD300081F4000106BF80F400000132013BB5E739
:10CD40004FEA41037FEA226C18BF7FEA236C21D0AF
:10CD500092EA030F04D092F0000F08BF0846704714
:10CD600090EA010F1CBF0020704712F07F4F04D1E2
:10CD7000400028BF40F00040704712F100723CBFF5
:10CD800000F50000704700F0004343F0FE4040F41F
:10CD9000000070477FEA226216BF08467FEA2363DD
:10CDA0000146420206BF5FEA412390EA010F40F4C8
:10CDB000800070474FF0000304E000BF10F0004314
:10CDC00048BF40425FEA000C08BF704743F09643FB
:10CDD00001464FF000001CE050EA010208BF704716
:10CDE0004FF000030AE000BF50EA010208BF70479D
:10CDF00011F0004302D5404261EB41015FEA010CB2
:10CE000002BF84460146002043F0B64308BFA3F1A9
:10CE10008053A3F50003BCFA8CF2083AA3EBC2538B
:10CE200010DB01FA02FC634400FA02FCC2F12002AA
:10CE3000BCF1004F20FA02F243EB020008BF20F0E1
:10CE40000100704702F1200201FA02FCC2F1200247
:10CE500050EA4C0021FA02F243EB020008BF20EA3C
:10CE6000DC7070477BB972B90029BEBF00204FF05B
:10CE7000004106E008BF00281CBF6FF000414FF0E2
:10CE8000FF3000F007BAADF1080C6DE904CE0029BF
:10CE900009DB002B1ADB00F095F8DDF804E0DDE992
:10CEA000022304B07047404261EB4101002B1BDBC1
:10CEB00000F088F8DDF804E0DDE9022304B0404228
:10CEC00061EB4101524263EB43037047524263EB13
:10CED000430300F077F8DDF804E0DDE9022304B055
:10CEE000404261EB41017047524263EB430300F063
:10CEF00069F8DDF804E0DDE9022304B0524263EB97
:10CF00004303704753B94AB9002908BF00281CBF22
:10CF10004FF0FF314FF0FF3000F0BCB9ADF1080C1D
:10CF20006DE904CE00F04EF8DDF804E0DDE90223FF
:10CF300004B07047430803F05533C01A830803F068
:10CF4000333300F03330184400EB101000F00F3092
:10CF500000EB002000EB0040000E704707EE900A47
:10CF6000F5EEC07AF1EE10FA01D400F00BB8F1EE54
:10CF7000677A08B517EE900A00F004F8404261EBBA
:10CF8000410108BDD0B5FFF7BFFA0C4B00220646A1
:10CF90000F46FFF711FBFFF7E7FD0446FFF792FA94
:10CFA000074B0022FFF708FB02460B463046394686
:10CFB000FFF74AF9FFF7D8FD2146D0BD0000F03D4C
:10CFC0000000F0412DE9F047089D04468E46002BF5
:10CFD0004DD18A42944669D9B2FA82F252B101FA2D
:10CFE00002F3C2F1200120FA01F10CFA02FC41EA3D
:10CFF000030E94404FEA1C48210CBEFBF8F61FFAC2
:10D000008CF708FB16E341EA034306FB07F199425C
:10D010000AD91CEB030306F1FF3080F01F8199420F
:10D0200040F21C81023E63445B1AA4B2B3FBF8F0E9
:10D0300008FB103344EA034400FB07F7A7420AD970
:10D040001CEB040400F1FF3380F00A81A74240F298
:10D0500007816444023840EA0640E41B00261DB103
:10D06000D4400023C5E900433146BDE8F0878B4238
:10D0700009D9002D00F0EF800026C5E900013046F7
:10D080003146BDE8F087B3FA83F6002E4AD18B42D1
:10D0900002D3824200F2F980841A61EB030301207B
:10D0A0009E46002DE0D0C5E9004EDDE702B9FFDE67
:10D0B000B2FA82F2002A40F09280A1EB0C014FEA12
:10D0C0001C471FFA8CFE0126200CB1FBF7F307FB6F
:10D0D000131140EA01410EFB03F0884208D91CEB12
:10D0E000010103F1FF3802D2884200F2CB804346AF
:10D0F000091AA4B2B1FBF7F007FB101144EA01448E
:10D100000EFB00FEA64508D91CEB040400F1FF311C
:10D1100002D2A64500F2BB800846A4EB0E0440EA0A
:10D1200003409CE7C6F12007B34022FA07FC4CEA13
:10D13000030C20FA07F401FA06F31C43F9404FEA06
:10D140001C4900FA06F3B1FBF9F8200C1FFA8CFE1B
:10D1500009FB181140EA014108FB0EF0884202FA6F
:10D1600006F20BD91CEB010108F1FF3A80F0888030
:10D17000884240F28580A8F102086144091AA4B2ED
:10D18000B1FBF9F009FB101144EA014100FB0EFE6E
:10D190008E4508D91CEB010100F1FF346CD28E459D
:10D1A0006AD90238614440EA0840A0FB0294A1EB2E
:10D1B0000E01A142C846A64656D353D05DB1B3EB8B
:10D1C000080261EB0E0101FA07F722FA06F3F140BB
:10D1D0001F43C5E9007100263146BDE8F087C2F162
:10D1E0002003D8400CFA02FC21FA03F391400143DA
:10D1F0004FEA1C471FFA8CFEB3FBF7F007FB103613
:10D200000B0C43EA064300FB0EF69E4204FA02F4BE
:10D2100008D91CEB030300F1FF382FD29E422DD911
:10D22000023863449B1B89B2B3FBF7F607FB163346
:10D2300041EA034106FB0EF38B4208D91CEB0101C6
:10D2400006F1FF3816D28B4214D9023E6144C91A46
:10D2500046EA004638E72E46284605E70646E3E656
:10D260001846F8E64B45A9D2B9EB020864EB0C0E60
:10D270000138A3E74646EAE7204694E74046D1E76F
:10D28000D0467BE7023B614432E7304609E764441D
:10D29000023842E7704700BF02E000F000F8FEE706
:10D2A00072B6374880F30888364880F309883648D4
:10D2B0003649086040F20000CCF200004EF63471AE
:10D2C000CEF200010860BFF34F8FBFF36F8F40F2C3
:10D2D0000000C0F2F0004EF68851CEF20001086066
:10D2E000BFF34F8FBFF36F8F4FF00000E1EE100AD6
:10D2F0004EF63C71CEF200010860062080F31488DF
:10D30000BFF36F8F7AF07CFD79F054FE4FF055300B
:10D310001F491B4A91423CBF41F8040BFAE71D49E3
:10D32000184A91423CBF41F8040BFAE71A491B4ADC
:10D330001B4B9A423EBF51F8040B42F8040BF8E72E
:10D3400000201849184A91423CBF41F8040BFAE703
:10D350007AF05AFD79F082FE144C154DAC4203DA96
:10D3600054F8041B8847F9E701F0D0F9114C124D2D
:10D37000AC4203DA54F8041B8847F9E77AF042BD5F
:10D38000000600200022002000C0000808ED00E098
:10D390000000002000060020F8A30A080022002058
:10D3A000E8250020E825002090340120E0C1000895
:10D3B00038C2000838C2000838C200082DE9F04F12
:10D3C0002DED108AC1F80CD0C3689D46BDEC108AC3
:10D3D000BDE8F08F002383F311882846A047002082
:10D3E00079F06EFBFEE779F0DBF900DFFEE7000085
:10D3F00001F0FF01102A2BDB10F0070F08D010F806
:10D40000013B013A8B422DD010F0070F42B3F6D109
:10D41000F0B441EA012141EA014122F007047FF022
:10D4200000070023F0E80256083C85EA010586EA79
:10D43000010685FA47F5A3FA87F586FA47F6A5FAB5
:10D4400087F68EB9EED1F0BC01F0FF0102F00702C1
:10D4500032B110F8013B013A83EA010313B1F8D16C
:10D460000020704701387047002D06BF354603384D
:10D47000073815F0010F07D1013015F4807F02BF86
:10D48000013015F4C03F0130F0BC0138704700BFD7
:10D4900010F8012B11F8013B012A28BF9A42F7D05E
:10D4A000D01A7047034613F8012B002AFBD1181A33
:10D4B0000138704738B50022002304460D46FFF7B7
:10D4C000EDFA28B920462946BDE8384000F00AB8F0
:10D4D000204605F1004100F005F8404261EB4101B2
:10D4E00038BD00BFD0B50C4B002206460F46FFF7F3
:10D4F00063F8FFF739FB0446FEF7E4FF074B002211
:10D50000FFF75AF802460B4630463946FEF79CFEB6
:10D51000FFF72AFB2146D0BD0000F03D0000F0419E
:10D5200000207047704700007047000070470000FF
:10D53000002070470020704700207047012070478E
:10D54000002070477047000000207047002070479F
:10D5500070470000704700000020704700207047AF
:10D5600070B5154ED6F8D00203681B68984704289A
:10D570001ADC01281DDC002814BF012441240F4BB4
:10D580001D68E86A0368DB69984701280AD0D6F865
:10D59000D0220B4B9A4205D0EB6A93F89C300BB12A
:10D5A00044F08004204670BD0A2814BF01241924C9
:10D5B000E5E71924E3E700BFF0550020EC25002043
:10D5C000C8580020044BD3F8D00203F536729042BD
:10D5D00014BF042002207047F0550020014B93F83F
:10D5E000E0017047F04500207047000038B5C5786D
:10D5F0000B461C2D044628BF1C251C220021184662
:10D600007EF03AFB2A4604F10C01BDE838407EF07A
:10D61000E9BA000038B5C5780B46102D044628BF7E
:10D6200010251022002118467EF026FB2A4604F120
:10D630000C01BDE838407EF0D5BA000008B53FF0D7
:10D64000CDFD30B9034A92F8643343F0040382F805
:10D65000643308BDF055002038B591ED000AF7EEAF
:10D66000000A0D4618F08EFB20B10B4801F0D8FEE1
:10D67000002038BDD5ED007A9FED087AF0EEE77A0C
:10D68000F4EEC77AF1EE10FA03D5034801F0DAFEA2
:10D69000EEE70320EDE700BFF02500200000003496
:10D6A00010B5044608F0A6FA204610BD13B58B8BC2
:10D6B000B72B0C4607D0B3F5967F22D002B0BDE859
:10D6C000104043F029BA12491E22A1F54C5001F036
:10D6D000E1FED4ED017A94ED007A0D48FCEEE77A94
:10D6E000BCEEC77A17EE903A8DED017A9DF80410E2
:10D6F0009AB201F071FB002814BF0020042002B090
:10D7000010BD04480449022201F0C4FE0020F6E7DF
:10D71000F0580020F0250020C458002000B51F4A12
:10D72000DFED1F6AD2EDD77A92EDD67AD2F84C139C
:10D73000007CA2F580538BB093F902320491002B48
:10D7400018BFB0EE677AD2EDD17A8DED057AFDEE95
:10D75000E77A3E2117EE903AD2EDD27AF4EEE67AED
:10D76000F1EE10FA58BFF0EE667AFCEEE77A1BB2E3
:10D77000ADF82030ADF8223017EE903A0022039237
:10D7800006920792ADF82430B7221A23CDE9003271
:10D7900003AA3CF0A7FF0BB05DF804FBF055002096
:10D7A00000FF7F4770B5154C94F86A238AB022B900
:10D7B0000AB0BDE870403EF061BA057C59F0AEFC9D
:10D7C000D4E9B261D4F8C432A4F50054CDE905130C
:10D7D000B4F8C024ADF826200023CDE90733ADF816
:10D7E000243068221C23CDE90306CDE90032212133
:10D7F00003AA28463CF076FF0AB070BDF055002021
:10D80000F0B53B4CB4F82432DE078DB0054637D571
:10D81000D4F8D832089302238DF82430D4F8E832B3
:10D82000D4F8DC02CDF82530D4F8E432D4F8D012A4
:10D83000D4F8D4220590CDF8293062202123D4F8E1
:10D84000C862D4F8C4720691CDE90030C221192310
:10D85000287C079203AA049603973CF043FF287C98
:10D860003CF0D6FE0646287C3DF0D6FD00F12103B3
:10D870009E4205D2287C0DB0BDE8F0403CF044B992
:10D88000B4F82432990731D5D4F8C0330893032370
:10D890008DF82430D4F8D033D4F8BC23CDF825301B
:10D8A000D4F8CC33D4F8C403D4F8B8130792CDF825
:10D8B000293062222123D4F8B063D4F8AC730590E8
:10D8C000CDE90032287C0691192303AAC2210397CF
:10D8D00004963CF007FF287C3CF09AFE0446287C26
:10D8E0003DF09AFD00F121039C42C3D30DB0F0BD81
:10D8F000F045002005207047024BD3F8D0020368A2
:10D900001B681847F055002030B5CD788BB0272D17
:10D9100028BF27250C462722002168467EF0ACF957
:10D920002A4604F10C0168467EF05CF91A4BD3F8E4
:10D93000D01203F5387291422BD1DDED057A9FEDBF
:10D94000177AF0EEE77AF4EEC77AF1EE10FA20D506
:10D950009DF8262002F0410141291AD1110618D460
:10D9600002F01801182914D00199C3F8E41282F0CA
:10D9700004020299C3F8E812C2F380020399C3F8C3
:10D98000EC1283F8F4220499079AC3F8F012C3F852
:10D99000F8220BB030BD00BFF0550020000000346D
:10D9A00030B5194D95F8693385B00C464BBBCA7834
:10D9B0008DF80C30092A28BF09220C3101A8CDE9C5
:10D9C00001337EF00FF99DF808305A1F012A18D94B
:10D9D00003F0F703122B14D0A5F58053B3F9E2211D
:10D9E00012B9E279A3F8E221227AE179074800F03E
:10D9F000B1F9227AE179054800F0E4F9012385F8CC
:10DA0000693305B030BD00BFF055002068510020DB
:10DA1000F0B51B4BB3F9E23189B005460E4614460A
:10DA20003BB1D779BB4204D009B0BDE8F04041F02A
:10DA3000FDBBA27A637A43EA0223E27A43EA024315
:10DA40001D2B13D0212B08D01BB921462846FFF7E8
:10DA5000A7FF224631462846E6E701A92046FFF700
:10DA6000C5FD084801A901F093FFF2E701A920468E
:10DA7000FFF7D0FD034801A901F0E0FFE9E700BF8F
:10DA8000F0450020F025002013B5CA78072A4FF092
:10DA90000003044628BF07220C3168460093CDF8E6
:10DAA00003307EF09FF8BDF900304BB901231C21F3
:10DAB000204684F80F3302B0BDE8104042F0E4BFC6
:10DAC00002B010BD30B5CD7889B01E2D28BF1E25FF
:10DAD0000C461E22002168467EF0CEF82A4604F14C
:10DAE0000C0168467EF07EF80248694601F0F2FFBC
:10DAF00009B030BDF025002000B589B0084601A965
:10DB0000FFF774FD034801A901F042FF09B05DF879
:10DB100004FB00BFF02500201FB508466946FFF74B
:10DB200079FD0348694601F089FF05B05DF804FB03
:10DB3000F02500202DE9F041CC7894B0262C28BFA8
:10DB4000262488462622002107460AA87EF094F85B
:10DB500002AD224608F10C010AA87EF043F82846DF
:10DB600007F072FD9DF84A30022B06AC03D0032B60
:10DB700044D0002B66D1DFED357ADDED106A9FEDE4
:10DB8000346A9DED0F7A66EEA76ADDED0E7A27EE18
:10DB9000067A67EE867A0023FDEEE66ABDEEC77A66
:10DBA000FDEEE77A17EE102A17EE901A0093204642
:10DBB00016EE903A07F068FD94E80F0085E80F0034
:10DBC00097F80F3363BB012698F8083098F80720C0
:10DBD0008DF8193000238DF818208DF81B3099220C
:10DBE0000423CDE90032387C8DF81A6003232246E5
:10DBF0002F213CF077FD14B0BDE8F081DFED137A02
:10DC0000DDED106A9FED126A9DED0F7A66EEA76A50
:10DC1000DDED0E7A27EE067A67EE867A0123BBE702
:10DC2000BDF8446086B90B483246294601F0D2FB64
:10DC30000028C8D0084A062138463EF063FF87F81E
:10DC40000F63C1E70226BFE70026BDE70000C84218
:10DC50008096184BF025002010FF080838B58A7A06
:10DC60004B7A43EA0223CA7A43EA0243272B05464A
:10DC70000C460CD81C2B10D91D3B0A2B0DD8DFE805
:10DC800003F01E0C0C0C1B0C0C0C0C121500452B7D
:10DC90000FD0522B01D1FFF737FE21462846BDE8B1
:10DCA000384041F0D1BDFFF7EFFEF6E7FFF742FF46
:10DCB000F3E7FFF707FFF0E7FFF71EFFEDE7FFF7DA
:10DCC0002BFFEAE700207047C8207047012070470B
:10DCD00000207047002070470120704790F8903076
:10DCE0008B4286BF00EB8100D0F894000020704783
:10DCF00090F890308B4286BF00EB8100D0F8940002
:10DD000000207047014B93F8DE017047F04500207A
:10DD1000036A43F4E0530362436A43F4E05343620B
:10DD2000836A43F4E05383627047000013B54FF4F5
:10DD30004470CDE9002107F055FF044628B1DDE924
:10DD4000002142F0E5FA024B2360204602B010BDEC
:10DD5000AC0009082DE9F04FDFF8649085B0064665
:10DD60000F46904600254FF4837A96F89030ECB237
:10DD7000A34222D920463CF04BFC834620463DF08E
:10DD80004BFB031D9B4514D399F90332ADF80830C2
:10DD900094220623CDE90032422102AA20468DF8C2
:10DDA0000A708DF80B80ADF80CA03CF09BFC01359F
:10DDB000DBE720463BF0A8FEF9E705B0BDE8F08FB1
:10DDC000F04500202DE9F04FDFF8649085B006465D
:10DDD0000F469046002540F2011A96F89030ECB2BA
:10DDE000A34222D920463CF013FC834620463DF056
:10DDF00013FB031D9B4514D399F90332ADF808308A
:10DE000094220623CDE90032422102AA20468DF851
:10DE10000A708DF80B80ADF80CA03CF063FC013566
:10DE2000DBE720463BF070FEF9E705B0BDE8F08F78
:10DE3000F04500201FB500F540530021D3F84C23D6
:10DE40000191D3F84433029201A900F5965003934F
:10DE500001F0A0FF03F06CFB03F036F905B05DF8AC
:10DE600004FB000070B586B006461322002101A80D
:10DE700010EE105A10EE904A7DF0FEFEA3238DF8AE
:10DE8000043095238DF8053059F050F91322CDF860
:10DE90000700CDF80B1006F57C6001A9CDF80F50F6
:10DEA000CDF8134037F0B6FC06B070BD2DE9F04157
:10DEB0008AB00446884617460021232201A8109DF7
:10DEC0001E467DF0D9FEA3238DF8043095238DF8EE
:10DED000053001238DF8063059F028F92B68CDF86C
:10DEE0001B306B68CDF80700CDF80B10CDF81F3054
:10DEF0002322AB68CDF80F8001A904F57C60CDF832
:10DF00001370CDF81760CDF8233037F083FC0AB0DA
:10DF1000BDE8F0819720704710B500F540530446E6
:10DF2000D3F8D00203681B6898471A22C1B204F5DF
:10DF30007C6037F02FFE04F59070BDE8104010F0C3
:10DF400003B8000037B500F50751044601221C3123
:10DF500036F032FA012504F50251104A00950023EB
:10DF60000831DA2033F02EFE0D4A0095002304F527
:10DF70007C61FD2033F026FE0A4B1A68D20705D4D7
:10DF8000094A1D6004F58F540834146006480121C5
:10DF900003B0BDE8304033F067BE00BFFC5F0A0845
:10DFA000B8B70908E82500200022002000207047AB
:10DFB000002070470069C0F3401070470F299DBFD3
:10DFC000302303FB010050300020704700207047D1
:10DFD0000120704770470000036800221B68184743
:10DFE00000207047002070470020704700207047D5
:10DFF00000207047002070470020704700207047C5
:10E0000000207047002070477047000010207047C4
:10E0100000207047704700000320704701207047C0
:10E0200070470000012070470020704770470000D3
:10E0300000F508502C30704700487047D824090874
:10E0400008B500F54050D0F8D00203681B68984727
:10E05000C0B208BD034808600F2111704FF0FF32B5
:10E060001A607047683C090800207047002070471C
:10E070007047000015F02ABF37F032BD43F03EB8BC
:10E0800041F026BA05F0C0BB06F05EBA00F0D2BE81
:10E0900000F0CCBE00F0EABE01F018BC00F0B8BE43
:10E0A00000F0BEBE00F026BF70B51F4B036000F548
:10E0B00000530446D3F8280D1C4AC3F8782B08B146
:10E0C00007F09CFD1A4B236004F5805393F8C42E8F
:10E0D00042B9D3F8C05E2DB1284614F019FE284687
:10E0E00007F088FD04F58E500C3056F029F804F541
:10E0F0008650143045F0D4F804F6C44504F664465E
:10E10000B54204D0183D284614F072FAF8E7094BDE
:10E11000C4F8983804F694103AF0E6FC04F5106060
:10E120003AF0E2FC204670BD9C3D09080CD209087B
:10E1300094B009085C86090838B5474B044640F896
:10E14000043B45F025FA04F1100006F023FB04F12E
:10E15000680035F08BF904F590700FF0D7FA04F5EC
:10E16000866005F0C1F904F2545007F049FD04F649
:10E17000980015F04FFD04F5446045F091F904F561
:10E18000516034F095FE04F57C6037F077FA04F5C1
:10E190008650143045F06CF804F58850103006F0C5
:10E1A00007FC04F58E500C3055F0B6FF04F58F5087
:10E1B000083035F067FC04F591501C3046F0C6FB82
:10E1C00004F5805304F593520025104683F86052FD
:10E1D000224B10301A6030F097FF294604F5965014
:10E1E00001F0CEFE04F5C85010304EF03DFE04F5AF
:10E1F000EA50143052F0EEFF04F5F3500C3055F0B5
:10E20000E5F804F5F650103055F01AFD04F5F95014
:10E21000083001F015FD04F5025008304FF0F0FA17
:10E2200004F5035020304BF07FFA04F5005304F559
:10E23000065083F89C510A4D343056F0BDFA2B68D5
:10E2400013B1084858F038FF2046074933F032FF31
:10E250002C60204638BD00BF94B0090888640020B7
:10E26000045C0020683A0908CCAF090810B59FED9E
:10E27000225A9FED224A9FED222ADFED221A9FEDBE
:10E28000221A9FED220A86B00446F0EE453AB0EE1F
:10E29000453AF0EE452AF0EE450AF7EE004A5430D2
:10E2A0008DED054A8DED042ACDED031A8DED021A90
:10E2B0008DED015A8DED000A4EF076FB9DED015A71
:10E2C0009DED054A9DED042ADDED031A9DED021A30
:10E2D0009DED000AF7EE004AF0EE453AB0EE453A01
:10E2E000F0EE452AF0EE450A04F59E704EF05CFB18
:10E2F000204606B010BD00BF00000000CDCCCC3DD4
:10E3000000007A450AD7A33CCDCC4C3DCDCC4C3E49
:10E31000F0B500F50055224BB5F8DE211A7087B034
:10E32000044644F01BFE44F0D1FB204601F002FC01
:10E3300004F5805393F83C2512F001020FD102A896
:10E34000019207F081F902A904F5965002F0D2FE7D
:10E3500028B12368019ADB6C02A920469847114E28
:10E360003368DB6A93F89C7037B195F89E311BB91E
:10E3700058F0D4FEC5F8A001336885F89E71DB6AB9
:10E3800093F89C20084B5A7135F0E2FA35F034F8D6
:10E3900004F50C50183007B0BDE8F0404EF054BB07
:10E3A00028230020EC2500202D5B0020FFF7B0BFC4
:10E3B00010B50821044601F0A5F918B117F0E6F8E8
:10E3C00015F02CFB0121204601F09CF910B12046EC
:10E3D000FFF730FD0421204601F094F918B104F54F
:10E3E0007C6036F0C9FD1021204601F08BF928B180
:10E3F00004F57C60BDE8104036F058BE10BD00004A
:10E40000FFF7D6BF102925D8DFE801F0090D111953
:10E410001524242424241C2424242424200000F54E
:10E420004B501C30704700F54C500430704700F5DD
:10E430004B503C30704700F54B502030704700F592
:10E440004C50704700F54B501430704700F54B505E
:10E45000183070470020704708B54FF0D5FA044BCC
:10E460001B68DB6A93F89C10BDE808404FF0A8BA1F
:10E47000EC250020FFF7F0BF2DE9FF410446FFF730
:10E480005BFE884B236004F5075004F500551C30F3
:10E49000FFF7ECFE002304F51050C5F800340430FB
:10E4A00043F04AF8DFF860827F4BC5F8043442F24B
:10E4B000544642F25477A01943F0CCF944F8068050
:10E4C0003036BE42F7D1A01944F028FC04F52D5097
:10E4D0001C303AF04BFD04F52D5028303AF046FD43
:10E4E0000023A5F8743B714BC5F8783B04F52E501A
:10E4F00057F0DEFC04F52E5604F530572436083765
:10E50000304614363FF0F6F9BE42F9D10723C5F87C
:10E510002C3D0023A5F8303D4FF4CB7007F068FB8D
:10E52000C5F8280D04F53450343057F0C1FC04F51B
:10E530003550383057F0BCFC5D4A13681BB904F500
:10E540002D53383313605B4BC5F8783B00265A4B8C
:10E5500003930294009604AB04F5365013E90C00C3
:10E560004021143005F06EFC04F54B5007F06CF8B8
:10E5700004F5405504F54B531833C5F8D0324F4BD2
:10E58000C5F8D4324E4BC5F8D8324E4BC5F8DC3204
:10E590004D4BC5F8E0324FF07E53C5F8E4324B4B9B
:10E5A000C5F8FC3204F54C58494BC5F80033002738
:10E5B000484BC5F8043308F10808C5F8F072C5F8EF
:10E5C000EC72C5F8E87208F1040007F03DF808F1B4
:10E5D000140007F039F8404B4048C5F8347304F58F
:10E5E0004D52C5F83873C5F83C731860283233466D
:10E5F0004FF6FF774FF0140C9EB20CFB060101336F
:10E60000097C0029F8D1364B36491E800B6813B1BE
:10E61000354858F051FD85F8693304F54D50012314
:10E6200085F86A332C300A6056F074F92F4BC5F820
:10E630006C332F4BC5F8C043C5E9F1342D4B04F5BD
:10E640004F50C5E9F3342C4BC5F8D433283006F0CD
:10E65000FBFF04F55050043006F0F6FF04F550506F
:10E66000203006F0F1FF04F54E56244BC5F8343443
:10E67000A5F8387406F1BC0006F0E6FF4FF0FF3352
:10E680002436C5F898341E4B1E491E60304633F0C0
:10E6900011FD2046A5F8E073A5F8FC7304B0BDE8B1
:10E6A000F08100BF9C3D09084C3A09080CD20908CA
:10E6B000205F002080010908A5E00008103E09083D
:10E6C000F43A0908583E0908443E09086C3E090816
:10E6D000083B09081C3B0908C85B00208434090872
:10E6E000C45B0020845B00207C3A0908B43A090826
:10E6F00069E000086DE0000871E000080000FFFF1D
:10E70000FC5A002090920908A03A090838B5054B38
:10E710001C6823680A461D68034B01462046A8472B
:10E72000002038BDEC250020F025002010B557F062
:10E73000F9FF064C064B18602046FFF79DFE204669
:10E74000044A0549BDE810407AF068BDF025002074
:10E75000EC250020C0C00020A9E0000838B52DED50
:10E76000028B0D46F0EE608AB0EE408A144602F04D
:10E77000DFFE90ED937AD0ED957A67EE877A90ED93
:10E78000927A67EEA87AE7EE087AC5ED007AD0EDC6
:10E79000920AD0ED937A90ED957A67EEA07A67EEC3
:10E7A000A80AE7EE480ABDEC028BC4ED000A38BDAA
:10E7B00030B52DED068B83B0F0EE409AB0EE60AA36
:10E7C0000D46044602F0B4FED0ED7F7AD0F8000288
:10E7D000B8EEE79A17F0A2FB07EE900AF8EEE78A88
:10E7E00079EEC9AA3AEE688AFDEEEAAAB0EE480AC6
:10E7F00017F076FBBDEEC00A5DB110EE103ADFED0A
:10E80000190A002BCCBF38EE608A38EE208ABDEEA4
:10E81000C80AF8EEC00A01AAB8EEEA0A694620461C
:10E82000FFF79CFFDFED107A104B009AC3F85023DE
:10E8300069EEA79A019AC3F8542329EE279A2AEE83
:10E8400027AA68EEA78AA3F58053C3EDB19A83ED9A
:10E85000B29A83EDEBAAC3EDEC8A03B0BDEC068B54
:10E8600030BD00BF00A00C470AD7233CF055002064
:10E8700038B52DED028B0D46B0EE408AF0EE608A81
:10E88000144602F055FED0ED937A9FED147AF0EE27
:10E89000E77AF4EEC77AF1EE10FA1DD4D0ED957A4E
:10E8A00090ED927A67EEE87AE8EE077AC5ED007AA5
:10E8B00090ED937AD0ED957A90ED926AC7EE876AE3
:10E8C0000120C6EE077A67EEA80AE6EE880AC4EDD4
:10E8D000000ABDEC028B38BD0020FAE700000034CE
:10E8E00030B55F4C2DED068BB4F91C32DFED5D8A3F
:10E8F0005B4285B008EE103A054604F65C303AF00B
:10E9000039FBB8EEC88A90ED00AAB4F91C3228EEA3
:10E91000288AF6EE009A98EE29AA04F65C3008EEF2
:10E92000103A3AF027FBB8EEC88A90ED009AB4F995
:10E93000203228EE288A04F6683098EE299A08EEEC
:10E94000103A3AF017FBB4F92232D0ED009A04F6EF
:10E9500068300AEE903A3AF00DFBB8EEC88AF8EE4D
:10E96000EAAAD8EE289A6A4602A990ED008A8DEDAF
:10E9700000AA9AEEA88A2846F0EE4A0AB0EE690A82
:10E980008DED038A8DED019ACDED029AFFF770FFB0
:10E9900001AA03A9F0EE490AB0EE480A2846FFF79B
:10E9A00067FF02F0C5FDD0F8000217F0B7FA04F5D2
:10E9B0008053D4ED857A93EDD10A30EE270A08EE24
:10E9C000100A20EE280A17F08BFAB8EEC88A30EE4B
:10E9D000480A17F085FADFED247A9DED007AB5EE4E
:10E9E000C00AF1EE10FAACBF70EE676AF0EE406A52
:10E9F000B4EEE67AB4BF70EE277AF0EE407AF1EE2C
:10EA000010FA2ADD9DED016AB4EEE76AF1EE10FA24
:10EA100023D5B5EEC00AF1EE10FA08DD77EE665A9E
:10EA200037EEC65AF4EEC55AF1EE10FA13D4B5EE2D
:10EA3000C00AF1EE10FA10D537EE667A77EEC67A94
:10EA4000B4EEE77AF1EE10FACCBF0120002005B059
:10EA5000BDEC068B30BD0120F9E70020F7E700BFD1
:10EA6000F04500200000C84200A00C4770B5314CB2
:10EA70002DED028BA4F58055D5ED857A94EDD10A64
:10EA8000DFED2D8A30EE270A84B020EE280A0646F4
:10EA900017F026FAB5F92232D5ED867A01EE103A52
:10EAA000B5F92032B0EE408A00EE903A94EDD30AE8
:10EAB000B8EEC11A30EE270AF8EEE00A0C2017F083
:10EAC00063FA20EE280A30468DED010AFFF708FFB1
:10EAD0009DED010A0146F0EE480A3046FFF768FE58
:10EAE0009DED010A03AA02A9F0EE480A3046FFF79D
:10EAF00035FEB5F91E32002B0DDD07EE903A94ED90
:10EB0000D27AF8EEE77AB4EEE77AF1EE10FA02DAAA
:10EB100094F808334BB99DED020A084800F00AFB4F
:10EB20009DED030A054800F0E3FB04B0BDEC028B49
:10EB300070BD00BFF05500200000C842F025002045
:10EB400038B5484C94F8643313F00101054643D1BD
:10EB5000A4F580529FED447AB2F9F02194EDD10AE8
:10EB600007EE902AF8EEE77A13F0100F67EE877A37
:10EB7000F7EE006ABFEE007A08BFB0EE667AA7EE45
:10EB8000270AC3F30012DFED397A84EDD10AB5EE1E
:10EB9000C00AF1EE10FA0AD51AB161F3041384F831
:10EBA0006433B4EEE70AF1EE10FA06DC0BE0B4EEE3
:10EBB000E70AF1EE10FA06DD2AB994F8643343F05F
:10EBC000100384F864339FED291ADFED290A2C2005
:10EBD00017F0DAF984EDD10A94F864339807C3F397
:10EBE00040012ED4234A9FED207AB2F9F20107EEBC
:10EBF000900AB2F92002B2F92222F8EEE77A01EE89
:10EC0000102A00EE900A1A0767EE877AF8EEE00AFB
:10EC100094EDD37AB8EEC11A18D577EE677AF4EE90
:10EC2000E07AF1EE10FAC4EDD37A03D561F3C303B1
:10EC300084F8643394EDD30A3C2017F0A5F984EDF1
:10EC4000D30A2846BDE83840FFF710BF77EE877A31
:10EC5000F4EEC17AF1EE10FAC4EDD37AEADD43F0B6
:10EC60000803E5E7F05500200AD7A33C0000B443B1
:10EC700000000000F04500200A2070470120704786
:10EC8000094B93F80813024609B1FFF7EFBE93F85A
:10EC9000691329B9A3F5805393F82832DB0702D50D
:10ECA0001046FFF74DBF7047F05500200420704715
:10ECB0000120704730B52DED028B8BB0044658F023
:10ECC0002DFA07AB054606AA05A9201D18F062FE1D
:10ECD000274A9FED288A136841F28831EB1A8B424C
:10ECE0001CD9156041F0F6FADDED067A67EE887AF8
:10ECF000054617EE900AFDF707FCDDED077A67EE93
:10ED0000887ACDE9020117EE900AFDF7FDFB1A4A59
:10ED1000CDE90001062128463AF0ECFCDDED067A4B
:10ED2000DDED070A9FED150A60EE880A27EE888A56
:10ED300060EE800A204628EE000A0021FFF738FD29
:10ED4000DDED070A9DED060A09AA08A92046FFF78E
:10ED500005FD9DED080A0A4800F0ECF99DED090A51
:10ED6000074800F0C5FA0BB0BDEC028B30BD00BF08
:10ED7000905A0020E02E65421C3E09080000C8425F
:10ED8000F02500200020704701207047024B01460B
:10ED90001868026812681047285F002008B5002034
:10EDA000FFF7F4FFC188472043F044FF472043F0BA
:10EDB0000DFE0120FFF7EAFFC188482043F03AFF2B
:10EDC000BDE80840482043F001BE00000220704723
:10EDD00001207047FFF7B4BE08B50B46013BDBB21C
:10EDE000012B114611D85BB9472043F023FF472080
:10EDF00043F0ECFD43F0E2FF43F0C8FC012008BD06
:10EE0000482043F017FF4820F2E70020F7E7000012
:10EE100008B542F0EBFCBDE8084042F0C7BB00007B
:10EE2000002100F5965002F009BB000000F254509A
:10EE300007F070BB10B5044607F05CFC90F9213078
:10EE40008BB190F8403373B194F978355BB1064BD0
:10EE50001B68DB6A93F89C302BB904F25450BDE870
:10EE6000104007F06FB910BDEC25002070B50446C6
:10EE700000F590700FF0C0FF94F8E4331B4904EBE9
:10EE80000312D2F894010A68824210D0B02202FB29
:10EE9000034294F8285492F8C12145B9022A06D9B0
:10EEA000134E08603278012A02D9013A327070BDDF
:10EEB000FDD104F54052D2F8C81229B9D2F8CC22BB
:10EEC00012B905233370F2E7B02202FB034303F5C6
:10EED000E6730FCB04F54B5585E80F00236800223D
:10EEE000DB6C2946204698470023EBE7945A002024
:10EEF0000C2200207047000037B5044644F02EF87D
:10EF000043F0E4FD04F500554721002043F0E0FE06
:10EF10004821012043F0DCFEB5F81C1201EB810111
:10EF200001EB8101490089B2472043F039FDB5F971
:10EF30002032B5F922120F4DC91A01EB810101EB04
:10EF40008101490089B2482043F02AFD43F036FF91
:10EF500043F01CFC04F52D5001A91C3001953AF03A
:10EF600067F804F52D5001A9283001953AF060F8B2
:10EF700003B030BDCDCCCC3DF0B52DED028B00F50E
:10EF8000005785B0B7F82022B7F82232044664252E
:10EF9000482012FB05F613FB05F543F0F1FC04F5E0
:10EFA000405304F508503030B0EE408ADFED230ABC
:10EFB00093EDD40A019000214DF0B0FE07EE906A67
:10EFC00038EE000AF8EEE77A0198B4EEE70AF1EEBF
:10EFD00010FA25D98DED020A07EE905A9DED027ABE
:10EFE000F8EEE77AF4EEC77AF1EE10FA03D8CDED39
:10EFF000027A4DF087FD48209DED020A43F0ACFCFB
:10F0000097F8753B04F52D50283083B10C4B0393D2
:10F0100003AA02A93AF010F805B0BDEC028BF0BDCE
:10F020000190CDED027A4DF06DFD0198D4E702A973
:10F0300039F0A2FF012387F8753BEDE70AD7A33C1F
:10F040000AD7A33C00F5405300F50050D0ED827A7A
:10F0500090ED846A93EDD47A67EE867AF0EEC76A13
:10F06000F4EEE76AF1EE10FA04D59FED180A482095
:10F0700043F072BCDFED167AB5EEC07AF1EE10FA0D
:10F0800020EE270A10DDB0F82032642213FB02F3D1
:10F0900007EE903AF8EEE77AF4EEC07AF1EE10FA65
:10F0A00002D59FED0C0AE2E7B0F82232642213FB8E
:10F0B00002F307EE903AF8EEE77AF4EEC07AF1EE5A
:10F0C00010FA02DD9FED040AD1E77047000000004E
:10F0D0000000C84200A00CC600A00C4610B50446B3
:10F0E00000F5405304F5005400F50850DFED100A18
:10F0F00093EDD40A002130304DF010FEB4F9220215
:10F10000B4F920323221C21A1B1A4A434B4301EE92
:10F11000102A00EE903A8020B8EEC11AF8EEE00A0C
:10F1200016F032FFBDE81040482043F015BC00BF88
:10F130000AD7A33C00F5005393F90032012B03D00A
:10F14000022B03D0FFF718BFFFF77CBFFFF7C6BF46
:10F15000F0B52DED028B00F500573223B7F81C52A5
:10F16000DFED310A00F50C5615FB03F5183600F5F6
:10F17000405393EDD50A83B00021044630464DF04C
:10F18000CDFD9FED2A1ADFED2A0ABF2016F0FCFE06
:10F190004720B0EE408A43F0F3FB9FED241ADFEDE9
:10F1A000240A30EE080AC02016F0EEFE6B4207EE8D
:10F1B000903AF8EEE77AB4EEE70AF1EE10FA26D9C3
:10F1C0008DED000A07EE905A9DED007AF8EEE77A91
:10F1D000F4EEC77AF1EE10FA04D83046CDED007A9D
:10F1E0004DF090FC47209DED000A43F0B5FB97F8E9
:10F1F000743B04F52D501C307BB10E4B019301AADA
:10F20000694639F019FF03B0BDEC028BF0BD304602
:10F21000CDED007A4DF076FCD4E7694639F0ACFECE
:10F22000012387F8743BEEE70AD7A33C00A08C4685
:10F2300000A08CC60AD7A33C00F540539FED117A7D
:10F24000D3EDD57A00F5005067EE877A90ED836AAA
:10F2500090ED817A27EE067AF0EEE76AF4EEC76A5F
:10F26000F1EE10FA04D59FED080A472043F074BB75
:10F27000F5EEC07AF1EE10FACCBF9FED040A9FEDD7
:10F28000040AF2E70AD7233C0000000000A08C46E5
:10F2900000A08CC610B5044600F5405304F5005498
:10F2A00000F50C50DFED110A93EDD50A002118305E
:10F2B0004DF034FDB4F91C324FF6CE71322213FBFF
:10F2C00002F213FB01F301EE102A00EE903AF12056
:10F2D000B8EEC11AF8EEE00AB1EE400A16F054FE9C
:10F2E000BDE81040472043F037BB00BF0AD7A33C1E
:10F2F00000F5005393F90132012B03D0022B03D008
:10F30000FFF726BFFFF798BFFFF7C4BFFEF704BEA5
:10F3100070B500F5005088B090F929020C46D8B1BC
:10F3200005210E4843F0D8FE092106460B4843F05C
:10F33000D3FE01210390094843F0CEFE04AD002125
:10F340000346039A00912846314606F09DF995E858
:10F350000F0084E80F00012008B070BD985A00200B
:10F3600037B50C460022054611460F4843F0C0FE53
:10F3700062680D48012143F0D3FEA2680A480521C6
:10F3800043F0CEFEE2680848092143F0C9FE05F5C6
:10F39000085001240DF1070129308DF8074033F0A2
:10F3A00081FC204603B030BD985A002037B5036871
:10F3B0000191DD6C04460FF05DFD90F8C412019AD6
:10F3C000B02303FB0101AC3120462B4603B0BDE85E
:10F3D000304018477FB5044604F5965668460D46FA
:10F3E00006F032F96946304601F0A8FE48B92946D0
:10F3F0002046FFF7B5FF064650B90026304604B058
:10F4000070BD2946304601F063FD0028EFD1F4E7D6
:10F4100095E80F0004F54B5484E80F00EEE7000078
:10F4200010B5074B1B680446D86A036801211B68A6
:10F43000984704F57C600121BDE8104036F0CEB954
:10F44000EC25002010B5074B1B680446D86A0368FA
:10F4500000211B68984704F57C600021BDE810403E
:10F4600036F0BCB9EC25002010B5044657F056FE26
:10F4700004F500540021C4F80004472043F0F8FBD1
:10F480000021482043F0F4FB43F098FCBDE8104015
:10F4900043F07CB970B5044604F5005304F54055BB
:10F4A00083F89C21D5F8D0328B420846164625D0E9
:10F4B000C5F8D0120B685B68984700B32046FFF789
:10F4C000AFFFD5F8D00203681B6898473246C1B237
:10F4D00004F57C6036F05EFB04F52D5000213830D9
:10F4E00041F0F2FA04F5A653D3ED007A9FED067AC7
:10F4F000F8EEE77A67EE877AC5EDD17A70BD2046DF
:10F50000FFF7A0FFDDE700BF0AD7233CF7B50446AD
:10F5100000F5935010302FF087FF5E4B04F5365006
:10F52000012214309A71DA7104F5866604F036FD12
:10F5300004F52D550823C4F844343046383504F01A
:10F54000E3FB28463EF020FA284641F0D7FD07F0BD
:10F55000D1F82023036307F0CDF808F043F9022324
:10F56000C4F8743104F5907004F596570EF04AF91A
:10F57000384600F073FE04F58053002283F8C92555
:10F58000B4F9A43004F698001BB9B4F8A230A4F87A
:10F59000A430B4F8A41016F067F8384600F058FF0D
:10F5A0003046012104F040FA3B4B00933B4B019362
:10F5B00002AB13E9060004F57C6036F003F942F073
:10F5C00015F99922292143F021F842F00FF942F070
:10F5D000B5F804F500562046FFF78EFC96ED7D7ACF
:10F5E000DFED2F7AF0EEC76AF4EEE76AF1EE10FA7B
:10F5F00004F5405746D8D6ED7E7ADFED2A6AB0EEA4
:10F60000E76AB4EEE66AF1EE10FA3BD8DFED266A5F
:10F6100027EE267A67EEA67ABDEEC77AFDEEE77A88
:10F6200087EDB27AC7EDB37AD7F8C8323BB9D7F8CD
:10F63000CC3223B904F54B512046FFF769FE1B4B32
:10F640001B68986A03684FF47A715B68984796F96B
:10F6500026122046FEF7D6FE014610B904F54B519E
:10F660001C311F222046FFF715FFD6ED7F7AF5EEFD
:10F67000C07AF1EE10FA0BDD204603B0BDE8F04091
:10F68000FFF7F2BE0A4A052128463AF033F8CBE7E5
:10F6900003B0F0BD2D5B0020F02500200DF3000825
:10F6A0000000B442000034438096184BEC25002043
:10F6B000783E090808B50A2921D8DFE801F00D18BD
:10F6C00011151C2020202020060000F54B5114317C
:10F6D000FFF7E0FE012008BD00F54B511C31F7E7B4
:10F6E00000F54B513C31F3E700F54C51F0E700F5E4
:10F6F0004C510431ECE700F54B512031E8E7002094
:10F70000E9E7000000F57C6036F092BE0148032175
:10F7100043F044BC985A002070B505462DED028B8D
:10F7200005F5405457F0EEFCD4F82C33DFED1D7A8C
:10F73000C31A08EE103AB8EE488A28EE278AF1EE8E
:10F74000047AB4EEE78AF1EE10FA29D504F5437392
:10F750000FCB04F5477686E80F00D4EDCE0A94ED82
:10F76000CD0A05F54C5068EE200A28EE000A1C3040
:10F7700006F02CFADFED0C7A94EDCF7A27EE277A9B
:10F78000D4EDC87AF8EEE77A0123E7EE087AFDEEC9
:10F79000E77AC4EDC87A84F80833BDEC028B70BDFB
:10F7A0000023F8E7BD3786350000C84230B585B084
:10F7B0006D460446284605F047FF294604F5965055
:10F7C00001F098FC50B104F54053002283F86A23FD
:10F7D00095E80F0004F54B5484E80F0005B030BDE8
:10F7E00070B52DED028B00F5405482B094F80833CB
:10F7F0000546002B5BD000F54B50D4F8D0220346D1
:10F800003C3305F54C569A4206F11C0618D094F884
:10F810006433DA0714D43146019006F0C5F89FED41
:10F82000277A0198F6EE007AE0EE077A9FED247AC7
:10F83000FDEEE77AF8EEE77A67EE877AC4EDD17AE3
:10F84000314606F053F905F5005584EDD20A95F9D5
:10F850000232DFED1C6AD4F8D002012B05BFD4F8C8
:10F860002033D4F8C422D4EDD07A9B1A08BF07EE17
:10F87000903AF8EEE77A87EEA67A84EDD77A0368B5
:10F880001B689847022812D094F864339B070ED463
:10F8900095F90232D4EDD20A9FED0B8A5BB994ED53
:10F8A000D60A7AF003F820EE080A84EDD30A02B0F3
:10F8B000BDEC028B70BD94EDD70AF2E7A00CB34506
:10F8C0000AD7233C0000C842E02E654273B50446C7
:10F8D000FFF722FF2046FFF769FF04F50055204699
:10F8E000FFF77EFFD5ED7F7AF5EEC07AF1EE10FAE4
:10F8F00009DC244B1E68F06A0368DB69984701281D
:10F9000016D102B070BD57F009FCD5F8003495ED62
:10F910007F7ADFED1D6AC01A07EE900A27EE267A7D
:10F92000F8EE677AF4EEC77AF1EE10FAE1D5E8E77F
:10F93000F36A93F89C10E9B995F92732012B10D19D
:10F940009FED120A472043F007F89FED100A482068
:10F9500043F002F843F032FA02B0BDE8704042F0E2
:10F9600015BF4720019143F065F90199482043F004
:10F9700061F9EFE704F54054D4F8D00203689B68BE
:10F980009847E7E7EC25002000007A4400000000DB
:10F9900037B54B68054613B98A68002A49D005F582
:10F9A00040540A20C4F814338B68C4F81833CA686A
:10F9B00092FBF0F2C4F810230B6993FBF0F3C4F848
:10F9C0004033B1F91630DFED1C7A07EE103AB1F989
:10F9D0001830B8EEC77A87EE276A07EE103AB1F909
:10F9E000143084EDCE6AB8EEC77AC7EE276A07EE08
:10F9F000103AB8EEC77AC4EDCF6AC7EE275AC4ED05
:10FA0000CD5A57F07FFBC4F82C0357F087FB022137
:10FA1000C4F830032846FFF775FE50B105F54C5386
:10FA200034330093D4E9C512D4F810332846FEF7D6
:10FA30003DFA03B030BD00BF0000C84210B52DED47
:10FA4000028B044691ED018ADFED207A94F841346F
:10FA500028EE278A00F58660242202FB0303F0EEDD
:10FA6000480A93ED090A03F087FCB4EE400AF1EE70
:10FA700010FAF0EE400A1FD69FED157AF0EEC07A2C
:10FA8000F4EE477AF1EE10FA16DC04F54053D3EDAC
:10FA9000D87A93F8642377EE807A5107C3EDD67A4B
:10FAA0000AD5F1EE407A00216FF38202C3EDD87AD5
:10FAB000C3F8581383F86423B0EE480ABDEC028BF8
:10FAC0002046BDE81040FEF7CDB900BF0000C84297
:10FAD000FFFF7F7FB1F9003007EE903AF8EEE77A4A
:10FAE00000F5405010B5C0EDD17AB1F9023007EE03
:10FAF000903AF8EEE77A0023C0F84833C0EDD37AA5
:10FB0000B1F9002090F8643347F6FF74121B18BF58
:10FB1000012262F3000380F86433B1F9023090F8F7
:10FB200064231B1B18BF012363F3410280F8642385
:10FB300010BD000010B500F54054D4F8300350B1AA
:10FB400057F0ECFAD4F83033C01A41F287339842B8
:10FB50008CBF00200120014B187110BD2D5B0020CF
:10FB600070B52DED028B00F500541646B4F9222233
:10FB700094ED860A01EE102AB4F9202200F54053D4
:10FB8000D3EDD37AD3EDD18A00EE902ADA20B8EE05
:10FB9000C11AF8EEE00A30EE270A0D4616F0F4F925
:10FBA000B4F92022B4F9223207EE902AF8EEE77A6F
:10FBB0009B1A30EE670A07EE903A30EE000AF8EE34
:10FBC000E77AB7EE008A80EE277A37EE487A86ED3C
:10FBD000007A94ED850A38EE800A16F041F9B4F9FE
:10FBE0001C3207EE103A30EE000AB8EEC77A012058
:10FBF000C0EE077A77EEC87ABDEC028BC5ED007ACD
:10FC000070BD000070470000002070477047000082
:10FC10000020704700207047002070470020704788
:10FC20009FED010A704700BF000000009FED010A30
:10FC3000704700BF000000000020704770470000C0
:10FC400010B50446143000F019F804F12C0000F04F
:10FC500015F804F1740057F06DFA04F1F40057F050
:10FC600069FA4FF0FF33C4F85031204610BD000050
:10FC7000014B1868704700BF9C5A00207047000075
:10FC8000F0B52DED048B91B004466D46284605F085
:10FC9000DBFC94F8BC33002B72D004F57A730FCBE5
:10FCA00085E80F0094F8F833D4EDEC8A94EDED8AF2
:10FCB00094EDEE9A002B63D094F8D033002B5FD0F4
:10FCC0002D22002104A8D4F8C073D4F8C463D4F85A
:10FCD000C853D4F8CC437BF0CFFFA3238DF810306A
:10FCE00095238DF8113046238DF8123057F01EFA07
:10FCF0009FED250A9FED257ACDF8171068EE807AE2
:10FD0000CDF8130067EE877AFDEEE77A17EE903AAA
:10FD100068EE007A29EE000A67EE877AADF81B30AC
:10FD2000FDEEE77A20EE070A17EE903AADF81D30A7
:10FD300016F0C0F8DDED017A9FED157ACDF82D7043
:10FD4000BCEEC00AF8EEE77A10EE103A67EE877A5A
:10FD5000ADF81F3017EE903ACDF82130029BCDF868
:10FD60002530039BCDF82930CDF83160CDF83550E2
:10FD7000CDF8394036F036FD2D2204A935F04AFD84
:10FD800011B0BDEC048BF0BDE02E65420000C8420E
:10FD90000AD7233C30B52DED028B8BB004462422CC
:10FDA0000D4601A800217BF067FFA3238DF80430E6
:10FDB00095238DF8053048239FED1F8A8DF8063076
:10FDC00057F0B4F9D4ED817A2B68CDF80F3067EE97
:10FDD000887A95ED020ACDF80B1017EE903AD4ED23
:10FDE000827ACDF8133067EE887A6B68CDF81730D9
:10FDF00017EE903ACDF80700CDF81B3016F030F82A
:10FE000010EE103A94ED830ACDF81F3020EE080A68
:10FE100016F026F810EE103ACDF8233094F80C3393
:10FE20008DF8273036F0DEFC242201A935F0F2FCF3
:10FE30000BB0BDEC028B30BDE02E654230B587B013
:10FE400014460D461822002168467BF015FFA323B7
:10FE50008DF8003095238DF8013049238DF802305C
:10FE600057F064F9A3680393E36804936368CDF8DB
:10FE700007100593CDF803008DF80B5036F0B2FC57
:10FE80001822694635F0C6FC07B030BD10B58EB0FB
:10FE9000044602A805F0D8FB02A9204601F02AF981
:10FEA000002845D001F044FB694600F0BBFF1F224B
:10FEB000002106A87BF0E0FEA3238DF818309523DF
:10FEC0008DF819304A238DF81A3057F02FF9DDEDEF
:10FED000037A9FED1B7A049BCDF82330F8EEE77A86
:10FEE000059BCDF8273067EE877ACDF81B0017EE1B
:10FEF000903ADDED007ACDF82B30F1EE677A17EE0F
:10FF0000903ACDF81F10204601A9CDF82F3000F00F
:10FF1000FDFB78B1DDED017AF1EE677A17EE903AEC
:10FF2000CDF8333036F05EFC1F2206A935F072FCA6
:10FF30000EB010BD36F056FCDFED027AEEE700BFE2
:10FF40000AD7233C5241C07F002303604360836093
:10FF5000C360036143618361C36103627047000052
:10FF600090F8C432B02202FB030390F8082393F800
:10FF7000A13012B1012B28BF0123184670470000A1
:10FF80002DE9F04F04468BB04FF0000A0D461BF0F0
:10FF9000F7FF84F814A204F506704FF07E5755F071
:10FFA00087FF4FF47A73A4F8623284F86852C4F879
:10FFB0004872C4F84C72C4F8507204F51B700025E6
:10FFC00005F042FB04F52B790323C4F8803204F5D5
:10FFD0003476C4F89452C4F89852C4F89C52C4F8C9
:10FFE000A052C4F8A452C4F8A8524846FFF7ACFF88
:10FFF00004F5487B3046FFF7A7FFC4F81453C4F854
:020000040801F1
:100000001853C4F81C535846FFF79EFFC4F84453D6
:10001000C4F84853C4F84C53C4F85053C4F854536C
:10002000C4F85853C4F85C53C4F86053C4F864531C
:10003000C4F86853C4F86C53C4F87053C4F88C53B4
:10004000C4F89053C4F89453C4F8A853C4F8A45304
:10005000C4F8A053C4F8B053C4F8B453C4F8B853A8
:10006000C4F8CC53C4F8C853C4F8C453C4F89C7340
:10007000C4F8C07304F5757005F0E6FA04F57A70FB
:1000800005F0E2FA04F58063C4F8FC531D6004F542
:10009000816304F583601D605D609D6005F0D4FAA6
:1000A00004F22C4304F264481D605D609D60684B5F
:1000B000C4F83C3404F50D73C4F8403404F50E73F1
:1000C000C4F8443404F50F73C4F8483404F51073CD
:1000D000C4F84C3404F24523C4F8503404F51173C9
:1000E000C4F8543404F58B6340461D605D609D6028
:1000F000FFF72AFF04F59160FFF726FF04F59763E9
:1001000004F23C421D605D609D6004F2C44304F251
:10011000A4501D605D609D6004F59A631D605D6084
:100120009D6004F2DC431D605D609D6004F2EC4361
:100130001D605D609D6004F2FC431D605D609D601C
:1001400004F5A463C2F8D470C2F8D8701D605D6075
:100150009D6004F22C531D605D609D6004F5A963F1
:100160001F605D6004F26C531D605D609D6004F56E
:10017000AF631D605D609D6004F5B2631D605D60EE
:100180009D6005F061FA04F2B45324221D605D60A5
:1001900004F2BC5351461D605D6004F2C4534046F6
:1001A0001D605D607BF068FD04F2E450C8F82070CB
:1001B000C8F81070C8F80070FFF7C6FE04F5C163F8
:1001C00004F5C7601D605D609D6004F214631D60EE
:1001D0005D609D6004F5C4631D605D609D6004F218
:1001E0002C631D605D609D6005F02EFA194B1A4965
:1001F0001C60204631F05EFF5146242258467BF0B9
:100200003BFDC4F84073C4F83073C4F8207304F5A0
:10021000257207CA04F5287383E80700484694ED61
:10022000AA1AD4EDA90A94EDA80A16F059FA35468F
:10023000494668466E4616F075F90FCE0FC50FCECB
:100240000FC533682B6020460BB0BDE8F08F00BFB0
:10025000B8400908A05A0020683F090810B50446B4
:1002600088B001F0EFF994F93232012B02D127481E
:1002700004F080FB022B0AD1032384F8323204A954
:10028000012304F111008DF8103032F0CDFC94F808
:10029000323284F8903204F23C4001F089F994F94A
:1002A0003132642B30D1652304A904F231208DF85A
:1002B000103032F0F7FC04A9204631F0D1F918B320
:1002C00004238DF818300023CDE9013303930F2365
:1002D0000593694604A831F095FB059B28B108AA4F
:1002E00002EB8302009942F8581C0133112B05934D
:1002F000EFD954F0F3FA9DED031ADDED020A9DEDFE
:10030000010A652154F0A8FA08B010BDC83E0908DA
:1003100070B500F5257600F528758CB00446314699
:10032000284617F0C9FDE0B996E8070085E8070000
:1003300004F52B7194EDAA1AD4EDA90A94EDA80A3C
:100340000191084616F0CCF902AD019902A816F009
:10035000E9F80FCD04F534740FC40FCD0FC42B682A
:1003600023600CB070BD000013B540F2411200F5DF
:100370000671044601A812F087FA04F23C4001F02D
:10038000FFFA20461BF0DAFF01A812F09FFA02B034
:1003900010BD0000F8B50B68C0F804324B68C0F817
:1003A00008328B68C0F80C3201F10C0607460C4687
:1003B00000F548750FCE0FC50FCE0FC533682B6003
:1003C00004F1300207CA07F5457383E8070004F11A
:1003D0003C0207CA07F5517383E8070004F148029D
:1003E00007CA07F5547383E80700543494E80700FC
:1003F00007F5577383E80700384601F037FA3846A7
:10040000BDE8F84001F01ABA13B5044600F23C40CA
:10041000019002F0ABFE04F5BB610198009102F07F
:1004200003FA0099204602B0BDE81040FFF7B2BFC2
:100430004A78064BC2F340121A754A78C2F380120A
:100440005A750A78C2F300129A7570472D5B002026
:1004500013B540F2F522044600F5067101A812F02A
:1004600013FA002104F23C4001F0FCFC94F86032E5
:1004700023B120461CF00EF984F8600201A812F0A6
:1004800025FA02B010BD000038B590F80C330546CF
:100490000C462BB1032B0BD095F86832DB070CD43C
:1004A00005F5C7630FCB84E80F0095F8480603E015
:1004B0001BF09AFF0028EFD038BD0020FCE70000B9
:1004C00000F23C4090ED350A7047000000F23C40DD
:1004D00090ED360A7047000010B490F80C230C46DB
:1004E0002AB1032A0AD000205DF8044B704700F5BA
:1004F000B26007C884E807000120F5E75DF8044B07
:100500001BF05ABF90F88403431E5842584170476D
:1005100038B590F80C330D468BB900F23C4001F031
:10052000A1FA044610B90024204638BD01F0EEF9C6
:10053000D5ED007A27EE800A85ED000AF4E7D0EDCC
:10054000E07AC1ED007A90F87C43002CEBD090ED7E
:10055000DE7ADFED086AB4EEE67AF1EE10FAF7EE35
:10056000006AB8BFB0EE667A67EE877AC1ED007AAE
:10057000DAE700BF0000003490F80C33032B01D100
:100580001BF09ABE0020704790F80C23032A01D17B
:100590001BF0B4BF00F23C4001F0C6BE30B590F88D
:1005A0000C3385B004460D468BB1032B18D004F5EF
:1005B000257017F0BBFC284601A98DED010ACDED91
:1005C000020A8DED031A17F00BFB012006E000F282
:1005D0003C4001F0F1F90028E9D1002005B030BD20
:1005E00090F86032002BF8D01BF070FFDFE70000BE
:1005F0007FB590F80C2332B1032A4FF0000309D0E5
:10060000039304930CE000F23C4007B05DF804EB68
:1006100001F0ACBA03A90393049305931BF042FEC7
:100620009DED030ADDED040A07B05DF804FB000050
:1006300007B590F80C3333B100F57F7003B05DF867
:1006400004EB17F0D9BB00F23C4001F08FFA68468A
:100650008DED000ACDED010A17F0CEFB03B05DF879
:1006600004FB000090F80C03003818BF012070470D
:1006700008B590F80C23032A05D0BDE8084000F225
:100680003C4001F05DBA1BF00DFE012008BD0000EA
:1006900010B590F80C230C461AB1032A07D000209D
:1006A00010BDBDE8104000F23C4001F0EDB91BF078
:1006B0000FFE012084ED000AF2E7000030B590F84B
:1006C0000C3385B005460C4623B1032B09D000201E
:1006D00005B030BD00F23C4005B0BDE8304002F04E
:1006E000D3B8002302A9029303931BF0C3FD002893
:1006F000EDD001A928461BF0C9FD0028E7D0029BD8
:100700002360039B6360019BA360E1E790F80C23E7
:100710001AB1032A05D00020704700F23C4002F0D5
:10072000D9B81BF0B3BD000090F932323BB990F854
:10073000683213F0010F14BF03200020704703201C
:1007400070470000F7B50446FFF7EEFF05460028A6
:1007500062D0032839D194F860326BB394F86832D0
:10076000D8072BD501A920461CF0BEF8BDF80430EF
:10077000002B18BF002594F8146206F0FD06012E28
:100780004AD10023032D019307D101A920461CF073
:10079000B7F820461BF0BEFE064604F23C4002F0CD
:1007A00025F908B994F809039DF80430D90703D551
:1007B0005A0701D59F0632D400252DE020461BF0B4
:1007C00033FD002808BF0025D5E70025D3E713F047
:1007D000020F2EE094F9443223B99DF80430DB096E
:1007E0002FD0E9E7002EF8D00EF044FBFFF7B8FB5E
:1007F000022807D99DF805309806DDD59DF804300C
:10080000D906D9D5FB6A93F89C30002BE5D118E0C6
:10081000DA0601D41B0718D5284603B0F0BD00281E
:10082000FAD094F80923B4F94C36002ACFD013F04B
:10083000010FF1D1154B1F68FB6A93F89C30002B18
:10084000C8D19DF804309C07E2D405F053FF05F0B1
:100850004FFE0028B0D10EF00DFBFFF781FB022800
:10086000AAD90EF007FB90F8C432B02202FB0300B5
:1008700090ED2F7AF0EE007AB4EEE77AF1EE10FA0E
:100880009AD59DF80530DB09C6D195E7EC25002007
:100890002DE9F04790F8603292B00446002B00F04A
:1008A000948020461CF02CF92046FFF74BFF0328CC
:1008B0007BD104F5487800274146204600970197F0
:1008C00002971BF0F9FD694620461BF0EBFD009BEB
:1008D000C4F80432019BC4F80832029BC4F80C32FD
:1008E000204600F0C3FF204600F0A8FF14F04EFEA3
:1008F000054620461BF0B0FC0028A8BFC6B203AADC
:100900004FF0FF312046BCBF95F8129395F8136362
:100910000397A8BFB146049705971BF0E7FC03A80F
:1009200017F004FB4FF00C0A0AFB095084EDD10AC2
:10093000C4EDD20A84EDD31A04F5517100F511709B
:1009400017F004FB04F557770AFB065584EDC50A3A
:10095000C4EDC60A84EDC71A3A464FF0FF3120466F
:1009600005F5C4751BF0D6FC95E8070006AE86E8D1
:1009700007003946304617F04FFB04F52B7241460D
:1009800009A815F05FFD314609A815F0DDFC09A99D
:10099000204684EDD40AC4EDD50A84EDD61A1BF0A6
:1009A000AFFF09A92046FFF743FD94F84E36002B10
:1009B0003AD109A804F048FE09A920461BF020FD01
:1009C00090B3012384F84E362EE0D0F864321BB980
:1009D00056F0A4FBC4F86402154B1B68D86A036880
:1009E0005B68984788B156F099FBD4F86432C01A16
:1009F000B4F86232984204D920461BF04BFE84F8CA
:100A0000600294F860327BB14BE756F087FBD4F874
:100A10006432C01A41F287339842E4D835F0E2FEDE
:100A200035F022FD0028DED112B0BDE8F08700BF0E
:100A3000EC25002090F80C3323B1032B4FF000007D
:100A400007D0704790F93222032A04D10A7001209E
:100A500070470870FBE718467047000073B50D46F5
:100A60000DF107010446FFF7E5FF064628B19DF8A2
:100A700007302BB1032B09D00026304602B070BDE1
:100A800004F5C7630FCB85E80F00F6E7294620463B
:100A90001BF0AAFC94F86062EFE700007FB50E46F9
:100AA0000DF103010446FFF7C5FF054618B90025FF
:100AB000284604B070BD9DF8033083B1032B16D0D7
:100AC00004F5257017F032FA01A930468DED010AC0
:100AD000CDED020A8DED031A17F082F8E8E73146F2
:100AE00004F23C4000F068FF0028E9D1DFE794F809
:100AF0006032002BDBD0314620461BF0E7FCDFE7FD
:100B000037B50D460DF107010446FFF793FF28B1F5
:100B10009DF8073023B1032B0FD0002003B030BD68
:100B200004F5BB631B682B6004F2DC5304F5BC6462
:100B30001B686B602368AB60F0E7204629461BF01A
:100B4000B1FC94F86002E9E710B50446FFF7ECFD4C
:100B500018B1032807D0002010BD04F23C40BDE8C6
:100B6000104000F053BF94F86032002BF3D02046C1
:100B70001BF05AFB0028EED094F8143203F0FD036A
:100B8000012BE9D194F80C03C31E58425841E3E706
:100B900010B50446FFF7C8FD80B1032810D194F8C2
:100BA000600250B156F0BAFAD4F86432C01A44F672
:100BB0002063984294BF0020012010BD0120FCE773
:100BC0000020FAE708B50246FFF7AEFD032804D17E
:100BD00010461BF095FE012008BD0020FCE7000038
:100BE00030B585B004460191FFF742F801990546FA
:100BF00010B9002005B030BD0191FFF70BF8019945
:100C00000028F6D02846FFF709F80028F1D0B4F8FC
:100C10004C365907EED494F80933002BEAD00B4A2E
:100C20001268D26A92F89C506DB103A92046FFF772
:100C3000C9FF30B19DF80E309A07DBD5C3F38000B1
:100C4000D8E72846D6E71846D4E700BFEC250020B1
:100C50002DE9F04190F80C338CB00027032B0646A9
:100C60000C46154600970197029719D11BF0F4FA2C
:100C70006A4680464FF0FF3130461BF04BFBB8F11F
:100C8000FF3FA760676027600DD114F07FFC2B4603
:100C900090F81313224613F007FD0CB0BDE8F08165
:100CA0004FF0FF38EBE714F071FC2B4622465FFA59
:100CB00088F113F0F9FC95ED000A684617F072F917
:100CC00003A920468DED051A8DED030ACDED040A2A
:100CD00017F0A2F906F52B7206F5487103A815F076
:100CE000B1FB214603A815F02FFB84ED021A84ED19
:100CF000000AC4ED010A95ED007ADFED037AA7EE54
:100D0000271A84ED021AC8E70AE81C4137B50546E0
:100D100000F5067140F6033201A811F0B5FD284632
:100D2000FFF702FD044640B103280AD0002401A8C1
:100D300011F0CCFD204603B030BD28461BF018FB57
:100D4000F5E728461BF014FB0446F0E708B5024619
:100D5000FFF7EAFC10B1032806D008BDBDE8084043
:100D600002F23C4000F01CBEBDE8084010461BF0FB
:100D7000D3BD00000B4610B411462BB1032B09D094
:100D800000205DF8044B70475DF8044B00F23C40D6
:100D900000F01CBE5DF8044B1BF032BB13B50446DB
:100DA000FFF7C2FC0A46014620460192FFF7E2FF28
:100DB00070B9084B019A1B68DB6A93F89C0038B144
:100DC00094F80C13204602B0BDE81040FFF7D2BFE4
:100DD00002B010BDEC25002037B504460D4640F2A8
:100DE000B25200F5067101A811F04EFD29462046C9
:100DF0001BF024FB94F80C33032B054610D148B1AB
:100E000004F583612046FFF7C9FF84F828042046D3
:100E100000F05CFD01A811F059FD284603B030BD7B
:100E20000025F7E770B590F87C32DB0786B0044602
:100E30000D460CD402F04EFF437C242202FB03003B
:100E4000D0ED0B7AF1EE677AC5ED007A3BE002A8AF
:100E500004F0FAFB01A92046FFF758FCE8B90EF0B0
:100E600009F894F94432022B0646E3D1FFF778F8EB
:100E70000228DFD996F8C4029FED147AB02303FB51
:100E80000066D4F87032D6F8B0209B1A07EE903A7C
:100E9000F8EEE77A67EE877AD6E702A92046FFF7F1
:100EA0007DFF0028DBD0D4F87022039BDFED076ABA
:100EB0009DED017A9B1A07EE903AF8EEE77AA7EEDD
:100EC000E67A85ED007A06B070BD00BF0AD7233CF4
:100ED000F0B50C4687B000F50671064640F686323E
:100EE00001A811F0D1FCA36853B9E36843B9636862
:100EF00033B9002701A811F0E9FC384607B0F0BD6E
:100F0000204604F0A9FC0028F3D094E80F0002ADBD
:100F100085E80F000021284604F060FC0746002801
:100F2000E7D096F87C32DB0704D435F05BFC19215E
:100F300035F0F0F995E80F0006F51B7C8CE80F0002
:100F400096F87C3243F0010386F87C32304600F09C
:100F5000BDFC3FF0BFF946213FF0B6FD3FF0BAF9C6
:100F600045213FF0B1FD054BA2681B68DB6A1A61A1
:100F7000E2685A6162689A61BCE700BFEC25002014
:100F800038B5144B1B68DD6A2B6804465B6828463D
:100F90009847F0B12B690BB96A69D2B1C4F87432C1
:100FA0006B69C4F87832A969002204F51B7004F05B
:100FB00051FB94F87C3223F0030343F0030384F8DD
:100FC0007C323FF087F9BDE83840034A062138F00B
:100FD00091BB38BDEC250020F03E090810B588B063
:100FE00004460593FFF7A0FB0328059B4FF0000084
:100FF0000AD10690079006A802900B9801900A98D3
:10100000009020461BF06CFA08B010BD38B50446BD
:10101000FEF72EFE0546D0B194F80C33032B03D017
:1010200095F84E41204638BD20461BF0D1F9FF28E7
:101030000446F5D001462846FEF7F0FD0028EFD023
:1010400021462846FEF7E6FD0028E9D0EAE70446F7
:10105000E8E7000008B590F80C33032B05D014F036
:1010600095FA90F91203C0B208BD1BF0F5F8431CC5
:10107000F9D1F4E708B590F80C3383B1032B03D111
:10108000BDE808401BF0E0B833F02AFE40F6ED4220
:101090004FF4801133F0DCFD4FF0FF3008BD1846EF
:1010A000FCE7000090F80C33032B01D11BF074BE59
:1010B0007047000090F80C33032B01D11BF012B8DD
:1010C000704700001BF098B810B504461DF0A6FE4E
:1010D0002046FEF7D5FD2046BDE81040FEF7D6BEFF
:1010E00090F80C330BB1032B01D11BF0D1BE0020C3
:1010F0007047000030B500F5757304460D460FCB00
:1011000085E80F0094F8E40330BD0000D0F8803388
:101110000B6090F87C037047D0F888330B6090F830
:101120008503704730B500F5677304460D460FCB55
:1011300085E80F0094F8AC0330BD000030B500F531
:10114000836304460D460FCB85E80F0094F828040E
:1011500030BD000010B500F22C4203460C4607CA11
:1011600084E8070093F8380410BD00002DE9F0432F
:101170002DED028B8BB005460E461746FFF746FF56
:10118000014680462846FFF72BFD0446002848D03C
:10119000FEF76EFD4146FEF743FD86ED000A95F928
:1011A0003032002B3ADD0DF065FEFEF7D9FE012846
:1011B00034D90DF05FFE90F8C432D5EDDE7ADFED64
:1011C0005D8A96ED000AB02202FB030095F93032E9
:1011D000D0ED2F0A07EE103AF4EEE87AB8EEC77AAF
:1011E000F1EE10FAB7EE008AB8BFF0EE487A37EEAB
:1011F000201A20EE270A70EEC70A40F2B63014F02B
:10120000C3FED5EDDE7AF4EEE87AF1EE10FAB8BF5F
:10121000F0EE487A80EE277A86ED007A01233B7063
:1012200003E095F8083333B9387020460BB0BDECB5
:10123000028BBDE8F08395F80C334FF00009CDF830
:101240000490CDF80890CDF80C9043B1032B10D04A
:10125000CDF81090CDF81490CDF818907CB90223F9
:101260003B703246414605F23C4001F083FB0446A8
:10127000DBE701A928461BF09FF80446E8E795F84C
:101280000C33002BEBD004A92846FFF763FF04467C
:101290000028E4D001A904A816F06EFE07A8CDED41
:1012A000080A8DED091A8DED070A17F079FA04A8DE
:1012B000B0EE408A17F074FA95F93032002B30DD29
:1012C00007EE903AF8EEE77A4FF47F7070EE670A17
:1012D00037EE801AF5EEC00AF1EE10FA48BFDFEDE6
:1012E000160AF4EE410AF1EE10FAB0EE480AC8BF51
:1012F000B0EE601A14F048FEB0EE408AD5EDDE7A0A
:101300009FED0C7AF4EEC77AF1EE10FAB7EE007AA0
:10131000B8BFF0EE477A88EE277A032386ED007A8D
:101320007DE7B5EEC08AF1EE10FA48BF9FED028A64
:10133000E4E700BF000000340000000010B50446E0
:10134000FFF788FE84F80D032046FFF783FE84F83C
:101350000E032046FFF77EFE84F80F032046FFF7BA
:1013600089FE04F55A7184F810032046FFF7B4F89B
:1013700084F8740300F0CAFA04F5617284EDDE0AA1
:1013800004F560712046FFF7F1FE04F5627184F800
:101390007C032046FFF7BCF804F5637184F88503ED
:1013A0002046FFF7E9F804F5677184F898032046B2
:1013B000FFF7F4F804F56C7184F8AC032046FFF7EE
:1013C0009FFB04F5707184F8BC032046FFF766FBB1
:1013D00004F5757184F8D0032046FFF755F804F53D
:1013E0007A7184F8E4032046FFF738FB84F8F803A9
:1013F0002046FFF7FDF804F5806384EDFF0A2046E0
:10140000C3ED000AFFF714F904F2044383ED000A68
:1014100004F2144204F581612046FFF719FC04F53B
:1014200083612046FFF7BAFC04F22C4184F82804BB
:101430002046FFF71DF984F8380410BD37B50D4676
:10144000044600F0FFF81DB914F0A0F813F05CF8A2
:101450004FF4BE7204F5067101A811F015FA94F864
:1014600069322BB92046FFF78BFD012384F86932DE
:10147000224B1D68A86A03689B6998472046FEF7BF
:1014800047FF2046FEF7C0FF204600F051FA2046F5
:10149000FFF7FEF9286B30B10368D4EDD20ADB68A0
:1014A00094EDD10A9847D4F8100208B156F0A4FD83
:1014B000204600F07DF82046FFF744F994F890327A
:1014C00084F80C0383420ED084F8900298B10C4D3E
:1014D0000C4B032808BF1D463EF0FCFE0A4A2B4673
:1014E000062138F007F92046FFF728FF01A811F080
:1014F000EDF903B030BD054DEEE700BFEC2500204F
:1015000037120908E73E0908083F0908EC3E0908B8
:10151000D0EDDE7A9FED057AF4EEC77AF1EE10FA9F
:10152000B7EE000AA8BFB0EE670A704700000034AB
:10153000014B1868704700BFA05A00204FF0FF30E1
:10154000704700000120704770470000002070477E
:10155000002070477047000070470000002070476F
:10156000002070470020704700207047002070471F
:101570000020704700207047012070470368D3F8AF
:1015800094301847002070470020704700207047B3
:1015900000207047002070470020704700207047EF
:1015A00000207047002070470020704770470000FF
:1015B0007047000008B513F0E9FF90F8130308BD69
:1015C00008B513F0E3FF90F8120308BD30B52DED18
:1015D000028B9FED1A1ADFED1A0A91ED000A87B00F
:1015E00005462D200C468DED011ACDED000A14F0B4
:1015F000CBFC9DED011ADDED000AF0EE408A2E20B5
:1016000094ED010A14F0C0FC9DED011ADDED000A15
:10161000B0EE408A2F2094ED020A14F0B5FC03A925
:1016200005F52570CDED038A8DED048A8DED050A53
:1016300031F01CFC07B0BDEC028B30BDC2B8323EAD
:10164000C2B832BE10B5044655F068FDD4F8F43285
:101650001BB1C21AB2F57A7F12D30A4A1268D26A53
:1016600092F89C2002B15BB9C4F8F40294F83142BC
:1016700013F08CFF80F80D4305F03CF880F825400E
:1016800010BD00BFEC2500202DE9F0432DED028BAD
:1016900091ED007AD1ED037A87B08DED047AB0EE4A
:1016A000C77AB5EEC07AF1EE10FADDE91087DDF801
:1016B0004C90CDED057A0C4615461E4606DCF0EE44
:1016C000E77AF5EEC07AF1EE10FA02DD04A816F022
:1016D000E5FB6B20B7EE001AFFEE000A9DED050A50
:1016E00014F052FC6C2089ED000AB7EE001AFFEEF0
:1016F000000A9DED040A14F047FC04A888ED000AD6
:1017000016F054FBB7EE008A002852D00023C9F827
:10171000003088ED008AD4ED067A67EEA77AF4EE01
:10172000C87AF1EE10FA4ADB0023336085ED008AB7
:10173000DFED3F0A96ED000A7C20B7EE001A14F0A8
:1017400023FC86ED000A95ED000A7D20B7EE001A15
:10175000FFEE000A14F018FC85ED000AD4ED067ABD
:10176000129BDFED346AF1EE677AC3ED007A96EDF5
:10177000007AF0EEC77AF4EEE67AF1EE10FA2BD5A5
:1017800003AB02AA01A9204615F00AF89DED018AD3
:10179000B0EE480A77F068FE85ED000AB0EE480A20
:1017A00077F0B8FF87ED000A07B0BDEC028BBDE80B
:1017B000F08304A816F0E6FA0028A7D1ABE738EECC
:1017C000670A14F013FB86ED000A94ED087AC7EE61
:1017D000007AC5ED007AABE794ED076AC6EE077AAA
:1017E000C7ED007A96ED007AB0EEC77AB4EEE67AED
:1017F000F1EE10FAC4D495ED007ADFED0F6AB0EE89
:10180000C76AB4EE666AF1EE10FAB9DCB4EE477A54
:10181000F1EE10FAB4D6B0EEE77AB4EE667AF1EEF5
:1018200010FAADDCF4EE677AF1EE10FABCD7A7E758
:101830000000000000000034FFFF7F7F1FB500F5AF
:101840001773039300F51673029300F51573019354
:1018500000F51473009300F5127200F5137300F590
:101860004871FFF711FF05B05DF804FB9FED156AA5
:1018700090ED817ADFED146AD0ED837A27EE067A57
:1018800067EE867A27EE267A67EEA67ABDEEC77AED
:10189000FDEEE77A80ED7E7A90ED827A27EE067A89
:1018A00017EE903A27EE267A002BB8BF03F50C43CB
:1018B000BDEEC77AB8BFA03380ED7F7AC0F80032A2
:1018C000704700BFE02E65420000C8421FB50E4BB6
:1018D0001B680446B3B1684603F0B6FE694620466D
:1018E000FFF72CFC20B16A4600212046FEF7A6FA3D
:1018F00094F87C32DB0705D504F51B7201212046E4
:10190000FEF79CFA04B010BD505D002008B502F04F
:10191000E1F9BDE8084001F06FBD000010B580F8A6
:10192000F812044655F0FAFBC4F8FC0210BD0000A2
:1019300010B590F8F832044653B155F0EFFBD4F8E7
:10194000FC32C01AB0F57A7F84BF002384F8F832E5
:1019500094F8003353B155F0E1FBD4F80433C01AC6
:10196000B0F57A7F84BF002384F8003310BD0000F7
:1019700000F5AA700B4607C883E8070001207047EE
:101980000023C0F89C30C0F89830C0F89430C0F8FC
:10199000A830C0F8A430C0F8A030C0F8AC30704710
:1019A00070470000024B0B604FF07C531360704790
:1019B000000048427047000008B50B4600F12801BE
:1019C000184615F057FD012008BD000010B500F5C0
:1019D000B4700C460FC884E80F00204603F024FEC4
:1019E00030B1FFF7A5FD00F51B700FC884E80F00AC
:1019F000204603F019FE80F00100C0B210BD0000C7
:101A000010B5044604F0F6F8204610BD10B5D0F825
:101A1000603104465BB155F081FBD4F86031C01AE7
:101A200041F28833984294BF0020012010BD01206C
:101A3000FCE7000013B5009303680192D3F89030DF
:101A40009847DDE90021044628B90448044B0068A2
:101A5000C06A11F0F7F8204602B010BDEC25002056
:101A60002840090813B504460191FEF701F92368DF
:101A7000019A1B6D014608B190F84E11204602B044
:101A8000BDE810401847000030B585B00023019331
:101A90000293039303680D46DB6D01A99847044642
:101AA00020B1039B2B60204605B030BD02F012F937
:101AB000417C01F0DDFD04460028F4D002F00AF973
:101AC00001F03CFDB1EE400A85ED000AEBE70000B5
:101AD00090ED007ADFED0F7AB0EEC77AB4EEE77AD8
:101AE000F1EE10FA14D590ED017AB0EEC77AB4EEAB
:101AF000E77AF1EE10FA0BD590ED027AB0EEC77AE4
:101B0000B4EEE77AF1EE10FA4CBF012000207047E6
:101B1000002070470000003410B5FEF7A9F8044615
:101B200058B190F84E11FEF775F830B194F84E1197
:101B30002046BDE81040FEF771B8002010BD00003F
:101B400038B50D460DF096F90446FEF709FA02285D
:101B500081BF94F8C402B02303FB0040D43089BF96
:101B600007C8002085E80700012038BD2DE9F043B3
:101B70002DED028B8FB003680025DB6C0395049577
:101B800005950695029502A904469847064638B180
:101B9000FFF7BCFEDDED027A27EE800A8DED020A2A
:101BA0000DF068F9FEF7DCF90746002E50D0DDEDA8
:101BB000027AD4ED646A94ED657A23680B9527EE7A
:101BC000877A67EEA67A8DED097ACDED0A7A0C95C3
:101BD0000D959B6C0BA9204609AD98470BA928468B
:101BE00016F05AF8012F8DED030ACDED040A40F2EC
:101BF000B3800DF03FF990F8C432DFED5B7AB02589
:101C000005FB030090ED308A28EE278AB0EE480AE3
:101C100077F02AFCF0EE408AB0EE480A77F07AFDC1
:101C2000CDED0B8A8DED0C0A0DF024F990F8C4323D
:101C300005FB030090ED2F0A0BA816F04DF809AD37
:101C40008DED050ACDED060A05A896BB03C885E013
:101C50000128CED89DED020AB5EEC00AF1EE10FAC9
:101C60007FDD07AED4F89421D4F890310792304646
:101C7000089316F04FF823680B950C950D959B6C07
:101C80000BA920469847DDED077A9DED0B7A77EE9C
:101C9000877A9DED0C7ACDED077ADDED087A77EE47
:101CA000877A09ABCDED087A96E8030083E8030054
:101CB00049E0236993ED000AB7EE008A38EE408AC6
:101CC00016F00AF804F5BC798DED090A4846B0EE25
:101CD000480ACDED0A0A15F0FFFF0BA92846CDED05
:101CE0000C0A8DED0B0A15F0D7FF04F5C47603AF8F
:101CF000C4ED5F0A314684ED5E0A384615F0DCFF1C
:101D000004F5C0788DED090A4046B0EE480ACDEDE5
:101D10000A0A15F0E1FF0BA928468DED0B0ACDED5F
:101D20000C0A15F0B9FF97E8030084ED600AC4EDD2
:101D3000610A86E803004946404615F0ADFF8DED87
:101D4000090ACDED0A0A9DED090ADDED0A0A0FB078
:101D5000BDEC028BBDE8F083DDE9030185E80300FB
:101D6000F1E709950A95EEE735FA8E3C10B590F843
:101D70004213044604F0D8F87C23C0B203FB0044AD
:101D8000D4F8A00010BD0000044B026F1B68DB6A92
:101D90005A60426F9A60826FDA607047EC250020CB
:101DA000F0B58FB0044613F0F1FB002302930393C8
:101DB000049390F8121301AB02AA054612F01AFC24
:101DC00004F19407D8B39DED010AB5EEC00AF1EE17
:101DD00010FA34DD02A816F0F5F804F1B00684ED2F
:101DE0002C0AC4ED2D0A84ED2E1A3946304616F021
:101DF000F9F804F17C01304616F0A8F804F18801E6
:101E000005A88DED050ACDED060A8DED071A16F031
:101E10009DF808A88DED080A9DED010ACDED090A8F
:101E20008DED0A1A16F0BEF80BA904F128008DED0D
:101E30000B0ACDED0C0A8DED0D1A14F05DFD95F831
:101E400012030C2303FB0050394600F5117016F005
:101E50007DF884ED2C0AC4ED2D0A84ED2E1A0FB006
:101E6000F0BD00002DE9F047824B00251F682DEDE5
:101E7000028BC0F89C50C0F89850C0F89450C0F83D
:101E80008450C0F88050C567C0F89050C0F88C509E
:101E9000C0F88850C0F8B850C0F8B450C0F8B0507E
:101EA0000446F86A03688AB05B680E46984704F1F6
:101EB0002809002854D055F031F942F20F739842A6
:101EC0004ED8FB6A9FED6C8A93ED010A84ED1C0AE3
:101ED000D3ED020AC4ED1D0A93ED031A484684EDC2
:101EE0001E1A14F0FDFB3EF0F5F9D4ED1E7A67EEF4
:101EF000887A054617EE900AFAF706FBD4ED1D7AAC
:101F000067EE887ACDE9040117EE900AFAF7FCFA39
:101F1000D4ED1C7A67EE887ACDE9020117EE900ABB
:101F2000FAF7F2FA554ACDE900010621284637F0C2
:101F3000E1FB94ED1E8AB0EE480A77F095FA84ED45
:101F4000650AB0EE480A77F0E5FB84ED640A55F0C7
:101F5000E5F8C4F864010AB0BDEC028BBDE8F08777
:101F6000A6B194ED1C0AB4EE400AF1EE10FA0DD6BB
:101F7000D4ED1D0AF4EE600AF1EE10FA06D694EDE7
:101F80001E1AB4EE411AF1EE10FA52D713F0FEFA0F
:101F900090F813334FF00C0A0AFB030303F5C473E4
:101FA000074693E8070007AE86E807004FF01508DC
:101FB000B2EE028AF2EE068A304616F0F1FBB4EE7B
:101FC000C80AF1EE10FA38D508F1FF3818F0FF080A
:101FD0003CD1304616F0E4FBF1EE047AB4EEE70AA9
:101FE000F1EE10FA43DD9DED090ADDED087A9DED75
:101FF000078A20EE000AA7EEA70A77F0A1FDF0EE0F
:10200000400AB0EE480A77F051FCDDED090A84ED94
:102010001D0A9DED080AF1EE600AB1EE400A77F064
:1020200045FC84ED1C0A9FED161AD4ED1D0A94EDB3
:102030001C0A484614F054FB7BE7304616F0B0FB10
:10204000B4EEE80AF1EE10FABEDCC2E7384612F050
:1020500093F9384612F058FA97F813330AFB0373D2
:1020600003F5C47393E8070086E80700A4E7256733
:102070006567D8E7EC250020E02E6542344009086A
:10208000000000000021FFF7EDBE000037B5044658
:1020900008461546019116F083FBB7EE007AC7EEAD
:1020A000007AB4F8D03001980133A4F8D03094ED20
:1020B000337A37EE277A84ED337AB0EE007AF4EE95
:1020C000C77AF1EE10FA06D5B6EE007AF4EEC77ACA
:1020D000F1EE10FA0DDC9FED0E7AF4EEC77AF1EE18
:1020E00010FA13D59FED0B7AF4EEC77AF1EE10FAE1
:1020F0000CDDB0EE670A15F055FF012085ED000AF2
:10210000C5ED010A85ED021A03B030BD0020FBE7E2
:1021100000247449BD37863570B52DED028B00F172
:10212000280600F134058AB029460446304615F0E9
:10213000B5FFB6EE008A20EE088A2846B0EE480ABF
:1021400015F030FF07A93046CDED080A8DED091ACC
:102150008DED070A15F010FF30468DED010AB0EE47
:10216000480ACDED020A8DED031A15F01BFF07A9F1
:1021700028468DED070ACDED080A8DED091A15F0F8
:10218000FBFE04A901A88DED040ACDED050A8DED35
:10219000061A15F097FF324601A920468DED070A71
:1021A000CDED080A8DED091AFFF770FF58B954F00C
:1021B000B5FF0121C4F860012046FFF753FE0AB0C5
:1021C000BDEC028B70BD2A4604A92046FFF75EFFD6
:1021D0000028ECD004F1400207A92046FFF756FF83
:1021E0000028E4D0EBE7000030B52DED028B0D4662
:1021F00083B091F842130446284603F095FEC1B21D
:102200007C2000FB0151903104F1280014F0F8F813
:1022100068468DED000ACDED010A15F0EDFDDFED0C
:102220001C7AB4EEE70AF1EE10FA05D59FED190A13
:1022300003B0BDEC028B30BD684615F02FFE68463A
:1022400015F0B4FD0028F1D1284694ED428A03F040
:10225000DFFFF0EE400AB0EE480A13F093FD80B9BC
:10226000284603F0D5FF84ED420AB0EE408A77F0AD
:10227000FBF884ED430AB0EE480A77F04BFA84EDA0
:10228000440A04F58671684615F06EFDD0E700BF7C
:1022900000000034000000009FED0C7AB4EEC70A85
:1022A000F1EE10FA0BD4DFED0A7AB4EEE70AF1EEA4
:1022B00010FA07DCC0EE077AB0EE670A7047F7EE57
:1022C000007AF9E7F2EE047AF6E700BFF3665F3FC3
:1022D00058A00B4108B51C3015F08EFDF1EE007AC8
:1022E000B4EEE70AF1EE10FA9DBFF1EE027A37EE96
:1022F000C00ADFED047A9FED040A98BF20EE270A9A
:1023000008BD00BFCDCC4C3ECDCCCC3D08B58369DB
:1023100093F9000038B10CF0ADFDFDF721FE012866
:1023200094BF0020012008BDF8B52DED028B0546B5
:1023300004F0E0F904F0DCF80446B8B3FFF7F8F86D
:1023400090F8093393B32846FFF7E0FF064668B3D9
:102350000CF090FD90F8C432B02707FB030090ED1D
:102360002F7AF0EE087AB4EEE77AF1EE10FA1DD487
:1023700095ED1E8A0CF07EFD90F8C432DFED1E7ADA
:1023800007FB030090ED300A98EE270A13F07EFD5C
:10239000DFED1A7AB0EEC00AB4EEE70AF1EE10FAF9
:1023A00008DC54F0BBFE3446C5F85001BDEC028B8E
:1023B0002046F8BD05F5AA7016F0F2F9B0EE408A95
:1023C0000CF058FD90F8C4329FED0D7A07FB030323
:1023D000D3ED2F7A67EE877AB4EEE78AF1EE10FA42
:1023E000DFD554F09BFED5F85041001BB0F5FA6FD5
:1023F0008CBF00240124D9E7E02E6542000034425E
:10240000CDCC4C3F10B50A4B1B68DB6A93F89C306F
:1024100004465BB954F082FED4F86431C01A44F625
:102420001F6398428CBF0020012010BD0020FCE7F4
:10243000EC250020F8B52DED068B04460CF01AFDB6
:10244000054604F057F9064606F040FE002840F025
:10245000AA802046FFF768FF002800F0A7803046DA
:10246000FFF784FCD4F8DC30984200F01881304645
:10247000FFF77CFCD4F8DC30DFED8E7AC31A08EE6F
:10248000903AF8EE688A304668EEA78AFFF76EFC4D
:1024900094F8BC30C4F8DC00F3B9304604F03AF8E4
:1024A000D0B104F1280796F842233946304603F0AC
:1024B000B3FED4ED1D0AB0EE401A384694ED1C0A66
:1024C00014F00EF90023C4F89030C4F88C30C4F82E
:1024D0008830012384F8BC3020463146FFF784FE63
:1024E00095F8C40205EB0015B0EE408A2B6FC4F8D6
:1024F000E03004F1B000D4ED129A16F051F963689F
:10250000DFED6D7A93ED007AB4EEE77AF1EE10FA32
:1025100068EE299AB0EE40AA01D5C3ED007A2046B4
:10252000B0EE4A0AFFF7B8FE636820EE299A93EDF1
:10253000000A29EE009AFFF7CDFE29EE009A204608
:1025400084ED249AFFF75EFF38B1D4ED247AB2EE21
:10255000007A67EE877AC4ED247AF0EE007AF4EE22
:10256000E78AF1EE10FA10D5DFED547AB4EEE7AA5F
:10257000F1EE10FA09D5DFED527A69EEA79AD4EDA3
:102580002A7AE9EEA87AC4ED2A7A9FED4E0A94EDF4
:10259000367ADFED4D7AB0EEC88A28EE008AA7EED3
:1025A000278A84ED368ABDEC068BF8BDFEF7C0FFA6
:1025B00090F80933002B72D02046FFF7A7FE0028C1
:1025C0006DD095F8C42205EB0213196FD4F8E030F2
:1025D0008B4264D0B02606FB025292ED2F7AF0EEC9
:1025E000087AB4EEE77AF1EE10FA58DBCB1AC4F8A9
:1025F000E01008EE903A95F8C4329FED341A94ED4D
:102600001E0ADFED337A06FB0353D3ED309A69EEF1
:10261000819AF8EE688A39EEC00A68EEA78A13F04C
:102620009FFCB0EE409A77F075F894F8BC30B0EEAD
:10263000408AF3B1F3EE047AF4EEE78AF1EE10FA91
:1026400017DC95F8C40206FB005595ED2F7AF2EEE3
:10265000027AB4EEE77AF1EE10FAFFF64AAFDFED58
:102660001D7AB0EEC99AB4EEE79AF1EE10FAFFF6D1
:1026700040AF9FED198AD4ED1D0A94ED1C0AB0EE0F
:10268000691A04F1280014F02BF8012384ED248A40
:1026900084ED238A84ED228A84F8BC3029E7BDECDE
:1026A000068B04F188009FED0D0ABDE8F84015F097
:1026B000CDBC00BFBD378635CDCC4C3DC2B8B23E97
:1026C0000AD7233CCDCC4C3ECDCC4C3F35FA8E3C8A
:1026D0006F12833A1904863F00000000EC51783FE6
:1026E00030B50C2303FB010101F1C003144693E84C
:1026F00007008BB004AD85E8070094E8070083E885
:1027000007002846FFF7E4F907AB58B194E8070043
:1027100083E807009DED070ADDED080A9DED091A23
:102720000BB030BD95E80700F2E70000F0B52DEDE5
:10273000028BD0F818318B60D0F81C31CB6085B09B
:1027400004460D4601F0C6FA06460CF093FBA36959
:1027500093F90030022B07464BD1FDF701FC02280C
:1027600047D997F8C432B02202FB0373D3F8B010F4
:102770000022284602F06EFFD4ED4A0A94ED490A81
:10278000284603F023FA94F82C3163B354F0C6FCC6
:102790009FED228A97F8C4128DED018A01AA0646A0
:1027A00038460BF0EBFBD4F820019FED1D0A361ADA
:1027B00007EE906AF8EE677A4FF4876027EE800A9A
:1027C000B6EE001AF0EE480A13F0DEFBDDED017AFA
:1027D00030EE270A04F1F0008DED010A15F07CFAC5
:1027E000284603F0F3F994F82C0105B0BDEC028BF8
:1027F000F0BD707C242303FB006696ED0B8AFEF788
:1028000097FED0ED9C7A9FED077AF8EEE77AE8EE36
:10281000077AFDEEE77A17EE901AA9E700000000AC
:102820006F12833A0000C842F8B5036F0B60436F24
:102830004B60836F8B6000F14C050E46074601F13B
:102840000C040FCD0FC40FCD0FC42B68236007F10C
:10285000B00207CA06F1300383E8070007F19402CB
:1028600007CA06F13C0383E8070007F11C0207CA08
:1028700006F1480383E8070006F160013846FFF7D8
:1028800055FF86F87000F8BD30B589B0044668463B
:102890000D4602F0D9FE69462046FFF797F818B9B1
:1028A0000024204609B030BD04A802F0CDFE204629
:1028B00004A9FFF73BFF04460028F1D004A96846AD
:1028C00003F0DCF885ED000AC5ED010A85ED021A7A
:1028D000E7E700001FB500230C4601A9019302930E
:1028E0000393FFF7D1FF08B1039B236004B010BD31
:1028F00030B585B001AD00230C4629460193029303
:102900000393FFF7C1FF034618B195E8030084E87D
:102910000300184605B030BDF8B506460F4615460B
:10292000FDF7A6F9044690B13946FDF773F970B189
:1029300020463946FDF772F9044640B1FDF798F993
:102940003946FDF76DF985ED000A2046F8BDFEF722
:10295000EFFD90F8083343B13046FFF7D7FC04464B
:1029600018B1D6F84C312B60EFE7D6F84C312B601C
:102970000024EAE770B52DED048B1646FFF7CCFF77
:10298000054670B3FEF7D4FD90F930424CB30CF01D
:1029900071FAFDF7E5FA012823D9E4B207EE904A6F
:1029A000B8EE678A0CF066FA90F8C43296ED009A99
:1029B000B02202FB0300D0ED2F8AFEF7A7FF38EE0E
:1029C000281A78EEC80A40F2614029EE000A13F096
:1029D000DBFAB0EE408AFEF799FFC8EE007AC6ED4A
:1029E000007ABDEC048B284670BD000008B503F0EA
:1029F00081FEBDE8084003F07BBD000010B5044631
:102A000015F07CFB50B904F10C0015F077FB28B9E8
:102A100004F11800BDE8104015F070BB012010BD96
:102A200038B500F1280504462846FFF7E7FF28B12E
:102A300020460121BDE83840FFF714BAD4ED107AE2
:102A4000B7EE007AF4EEC77AF1EE10FA06D5BFEED3
:102A5000007AF4EEC77AF1EE10FA12DC2046FFF7A6
:102A60005BFB2846FFF7CAFF0028E1D1D4ED107ABE
:102A7000B2EE047AF0EEE77AF4EEC77AF1EE10FAED
:102A8000D6DC38BD10B5044615F08AFE2046BDE8F8
:102A9000104015F0EFBA00002DE9F04F2DED048B3A
:102AA0009FEDC48A95B00446F0EE408A8DED028A0F
:102AB0008DED038A8DED048AFFF7BCFC12F066FDF4
:102AC0000023054695F87921012AA8BF01229342E7
:102AD0003FD20021284611F0BBFB01230028F1D092
:102AE00008AB0BAA002128468DED0B8A8DED0C8AD0
:102AF0008DED0D8A11F0D8FD9DED080AB5EEC00AE6
:102B0000F1EE10FA23DD0BA815F05CFA11A904F11F
:102B100028008DED110ACDED120A8DED131A13F078
:102B200013FC0EA88DED0E0AB0EE680ACDED0F0A6B
:102B30008DED101A15F036FA11A904F1E4008DEDAF
:102B4000110ACDED120A8DED131A15F04BFA01237F
:102B5000B8E795F813130C2303FB015104F1280B7C
:102B600001F5C471584613F0EFFB84ED070A94EDAC
:102B70003F0AC4ED080A70EE288A84ED091AC4EDF4
:102B80003F8A0CF077F90646FEF7D2FC90F809333D
:102B900000932046FFF7BAFB80B13046FDF7E0F91D
:102BA00002280BD996F8C4226169B02303FB0263A3
:102BB00091F9001093F8D20088425FDA94ED3F7AE1
:102BC000DFED7D7AB4EEE77AF1EE10FA5DD4D4ED64
:102BD000538AFEF7A1FF38B1FDF74AF890F84E117D
:102BE000FDF71EF8F0EE408A236C626BA16A139326
:102BF000B0EE680A11A81292119115F0D3F904F5FC
:102C0000AA7102A88DED020ACDED030A8DED041A1A
:102C100015F0E8F954F082FA0023074684F81431DD
:102C20002046FFF773FB002865D096F8C422B02336
:102C300002FB033232445268C4F8182196F8C422C9
:102C400002FB033333449B68C4F81C3154F066FA2A
:102C50000123C4F8200184ED498A84ED4A8A84F86E
:102C60002C31D4F80031002B58D102AB93E8070087
:102C7000C4F80071F03484E8070006E006EB0212A5
:102C8000176FD4F80021BA4204D115B0BDEC048B03
:102C9000BDE8F08FD43393E8070094F814310DF1B8
:102CA000080C8CE807001BB904F1F00383E8070067
:102CB0000123604684F8143104F5AA7115F05CF91B
:102CC00011A904F14C008DED110ACDED120A8DED24
:102CD000131A13F067FBB5EEC00AF1EE10FA8DED92
:102CE000110AD8BF9FED330ACDED120A8DED131AEC
:102CF00084ED530A94E794ED3F7AD4ED497ADDED03
:102D0000026AE6EE877ADDED036AC4ED497AD4ED16
:102D10004A7AE7EE267AC4ED4A7AA2E7D4ED3F7A02
:102D2000224B8DED058AF5EEC07AF1EE10FA8DEDAD
:102D3000068A0793A9D99FED1E7A94F8143167EE9D
:102D4000877AB7EE007AC7EE279A1BB9009B002B53
:102D500000F0AA80E36804F1F00102A8D3ED008A34
:102D600015F00AF969EEA88A8DED110A11A8B0EEE6
:102D7000680ACDED120A8DED131A15F013F90EA99C
:102D800005A88DED0E0ACDED0F0A8DED101A15F088
:102D900029F905A8FFF776FE05A815F0C9F9D8B1FD
:102DA00054F0BCF9C4F860016FE700BF000080BFB9
:102DB0000AE81C4100000000CDCC4C3ECDCC4C3F7D
:102DC000CDCC4C3D920A06BF920A063FC2B8B23E35
:102DD000728A0E3C5B821839012301930023CDE9EE
:102DE0000833CDE90A33CDE90C335FED0E8A4FF09D
:102DF000FF3A04F1E40895F87921012A1046A8BFAA
:102E00000120834257D20123002AFAD095F83513C6
:102E10000029F6D0B0EE690A404615F017F9019B7B
:102E20000DF12C09002B41D0424600212046FFF72E
:102E300057FC8DED0B0ACDED0C0A8DED0D1A4846B1
:102E4000FEF746FE70BB4846FFF71CFE484615F0ED
:102E50006FF938BB05A9484615F034F9484605A96D
:102E60008DED080ACDED090A8DED0A1A15F016F957
:102E700008A8B0EE409A15F093FCBAF1000F06D105
:102E8000F4EEC08AF1EE10FAD8BFB0EE680AB5EEE3
:102E9000C09AF1EE10FAF7EE008A58BFF0EE408AC1
:102EA0004FF0000A0123A6E7009B96E798E8070089
:102EB00089E80700C3E7BAF1000F7FF471AF002380
:102EC00084F804312046FFF72FFA38B12046FFF787
:102ED0001DFA002840F025818DED0A8A95F81233FD
:102EE00095F878219A4240F233812B4493F8343399
:102EF000002B00F02D8195F8133395F879219A4233
:102F000040F226812B4493F83533002B00F02081CA
:102F100008A9584613F046FA8DED080ACDED090AC6
:102F20008DED0A1A08A815F0E9F8002840F017817D
:102F300008A815F0FDF8002840F011815FED627AD5
:102F400094ED357A68EEA78A5FED647AE7EE278A1A
:102F500004F1B000C4ED358A15F022FCA3685FEDE2
:102F6000687A93ED007AB4EEE77AF1EE10FAF0EEBB
:102F7000408A00F1F8802046B0EE680AFFF78CF92D
:102F800008A815F00FF8A3688DED110ACDED120A0F
:102F90008DED131A93ED000A11A815F003F82046E1
:102FA00084ED1F0AC4ED200A84ED211AFFF72AFAE6
:102FB00028B1B2EE000A04F17C0015F047F8009B3E
:102FC000B3B33046FCF7CCFF012831D996F8C402E0
:102FD000B02303FB006696ED2F7AF0EE087AB4EE8C
:102FE000E77AF1EE10FA23D595F813030C2303FBCF
:102FF000005595ED627AF1EE0C7AB4EEE77AF1EED7
:1030000010FA15DBD4ED1D7A1FED927AF4EEC77A33
:10301000F1EE10FA0CDD1FED947AF4EEC77AF1EEC2
:1030200010FA05D5B6EE000A04F17C0015F00EF892
:103030005FED9A7AF4EEE78AF1EE10FA22D51FEDF1
:103040009C0A08A814F0AEFF0EA88DED0E0A94EDB0
:103050003F0ACDED0F0A8DED101A14F0A3FF11A950
:1030600004F1A0008DED110ACDED120A8DED131AB9
:1030700014F0B8FFD4ED2B7A94ED3F7A77EE877A8F
:10308000C4ED2B7A94ED2B7AF1EE047AB4EEE77A64
:10309000F1EE10FA3BDB12F079FA5FEDB27A94EDC3
:1030A0002B1A94ED280A21EE271A40F2C530F1EED2
:1030B000410A8DED011ACDED000A12F065FF9DED7C
:1030C000011ADDED000A84ED280A40F2C63094EDC5
:1030D000290A12F059FF9DED011ADDED000A84ED79
:1030E000290A40F2C73094ED2A0A12F04DFF04F18C
:1030F000A00184ED2A0A04F1940014F073FF84ED1A
:103100002A8A84ED298A84ED288A84ED2B8A00237B
:10311000C4F8E430C4F8E830C4F8EC3084ED3F8AF9
:10312000A3E5E368F7EE000A93ED000A12F02AFE29
:1031300000283FF4D1AE94ED1C0AB0EEC00A76F040
:10314000E9FADDED0A7A27EE800A8DED0A0AC5E676
:103150008DED0A8A8DED098A8DED088AE2E620461A
:10316000FFF75EFC1CE6C3ED007A04E72DE9F04DA5
:103170002DED048B9EB0044612F008FAD0EDC87A0B
:1031800090ED618AF4EE487AF1EE10FA48BFB0EEA5
:10319000678ADFED5C7AB4EEE78AF1EE10FA0EDDB5
:1031A0000023C4F8E430C4F8E830C4F8EC3000235D
:1031B000C4F8FC301EB0BDEC048BBDE8F08D204699
:1031C000FEF7EEFD2046FEF7A7FFB0EE480A2046C8
:1031D000FFF762FC2046FFF723FCFEF7A9F914ADC8
:1031E00000F5347204F1280114A813F02BF90FCD67
:1031F00004F14C060FC60FCD0FC62B68336004F1E7
:10320000740204F1780304F1700104F14C0013F02E
:10321000C7FA94ED1E8AB0EE480A76F025F984EDDF
:10322000650AB0EE480A76F075FA204684ED640A25
:10323000FEF7AAFDFEF77CF904F5B471FDF77EFFF9
:1032400053F06CFFD4F89831C31A632BB2D9C4F889
:10325000980133F0C7FA9FED2C9A054653F066FFAC
:10326000D4ED1C7A67EE897A074617EE900A0E466F
:10327000F9F74AF9D4ED1D7A67EE897A824617EE9E
:10328000900A8B46F9F740F994ED1E0A20EE090AE0
:1032900041EC180B12F0E4FDD4F85C0110EE108A3A
:1032A000F9F732F9CDE91201D4F85801F9F72CF900
:1032B000CDE91001D4F85401F9F726F9CDE90E0152
:1032C000D4F8D800F9F720F9CDE90C01D4F8D400EE
:1032D000F9F71AF9CDE90A014046F9F715F90B4B50
:1032E00001930B4B0093CDE908018DED068BCDE9E1
:1032F00004ABCDE90276074B074A0849284632F06D
:10330000B3FE57E7CDCC4C3EE02E6542994009080C
:10331000A3400908604009086A400908EC3E090812
:1033200008B52DED048BB0EE609AF0EE408A00F007
:1033300011F9B0EE408A89EE280A76F021FBDFED24
:103340000B7A20EE270A76F0B3FADFED097A38EE31
:10335000278ADFED087A28EE278AF7EE007A37EE23
:10336000C00A28EE000ABDEC048B08BD41D3423EE2
:1033700033938843A1D81943FFF7D2BF08B52DED89
:10338000048B9FED189AF0EEE07AF4EEC97AF1EE34
:1033900010FAF0EE408AB0EE608A1ED400F0DAF83F
:1033A000DFED117A9FED117A70EE277A9FED100A0A
:1033B000E8EEC77A9FED0F7A27EE800AC8EE007A12
:1033C00087EE270AB4EEC90AF1EE10FA05DBBDEC70
:1033D000048BBDE8084076F0B3BBBDEC048BB7EEC0
:1033E000000A08BD0000003433938843F4FDD43B49
:1033F00048A18F43CDCC9C3F427CD0ED257A24213F
:1034000001FB020292ED0B0AD2ED090A30EE270A07
:10341000FFF7B4BF38B52DED088BDFED21AA9FED86
:1034200021AA9FED21BA0546B0EE409AF0EE609ACF
:10343000B0EE408A1524013CA4B25CB3F0EE490A18
:103440002846B0EE480AFFF76BFFF0EE490A70EE2F
:10345000698A284638EE2A0AFFF762FFB0EEE87A5A
:1034600070EE697AB4EECA7AF1EE10FA77EEE87A85
:1034700010D468EEAA8A40F2631088EEA70AB0EE74
:103480004B1A38EE400AF0EE4A0A12F07DFDB0EE1B
:10349000408AD0E7B0EE480ABDEC088B38BD00BFCB
:1034A000CDCCCC3D0AD7233C002474490023436093
:1034B0008360C360036143618361C361002380F85B
:1034C0002030704790F82020531CDBB2062B80F888
:1034D000203000EB820288BF002382ED010A88BF02
:1034E00080F82030704700004FF0FF3310B5436183
:1034F0000E4BC0F8A8300023044680F8C830A8302E
:10350000FFF7D4FF0A4BC4F8A83004F5867052F0D8
:10351000CFFC084B08491C6020462EF0CBFDD4F8A8
:103520009030C4F89430204610BD00BFC042090856
:10353000D0420908A45A00206843090808B5A830F9
:1035400035F00AFADFED027A20EE270A08BD00BF47
:1035500000007A4490ED3C0ADFED057AB0EEC07AC7
:10356000B4EEE77AF1EE10FA48BF90ED3D0A7047ED
:103570000000003473B5D0F8A43004460E4663B1A1
:1035800053F0CCFDD4F8A430C01A42F20F73984225
:1035900003D894ED280A02B070BD114B1D687DB1AF
:1035A00095F84E112846FCF739FB48B195F84E11B5
:1035B00001AA2846FCF728FB10B19DED010AEAE7B5
:1035C000242101FB064494ED0A0ADFED067AB4EEED
:1035D000E70AF1EE10FA58BFB0EE670ADBE700BF6A
:1035E0009C5A002000000C4208B561B10378022B00
:1035F00002D9064853F060FD5A1C027000EB8300AC
:103600004160012008BD0846FCE700BF8841090869
:103610002DE9F84305460E469146002400F13C088A
:103620002B78A34211DD00234A46314601200EF0DB
:103630009FFF242363430746002158F803000EF040
:10364000A7FF874204D00134EAE70020BDE8F883F1
:103650000120FBE7054B1B682BB141694A1C02D0D6
:10366000184632F0E5BE0020704700BF505D0020D4
:1036700002290BD8242303FB010191F8390030B152
:1036800091F83A0018B191F83B007047002070475C
:103690002DE9F047044653F041FDD4F8F86042F2BA
:1036A0001073861B9E4288BFC4F8F80000274FF0B5
:1036B000240942F2107A237CFDB2AB421CD9294680
:1036C0002046FFF7D5FF70B109FB054898ED0D0ABC
:1036D000D8ED097AD4ED250A30EE270A2046FFF707
:1036E00099FE88ED0C0A564504D909FB0540303097
:1036F0002EF0B8FE0137DEE7617C2046FFF73AFF87
:1037000084ED3D0ABDE8F08770B5044686B053F0FD
:1037100005FDD4F89830C31AB3F57A7F05464FD328
:10372000344B94ED257A1B68DFED336ADB6AD4ED08
:10373000247A93F89C60B0EEC76AB4EEE66AF1EEC4
:1037400010FA32D5B0EEE76AB4EEE66AF1EE10FA9E
:103750002BD502A801F078FF96BBFDF7E9FE02A980
:10376000FDF7ECFC60B3DDED037A9FED247AF8EE13
:10377000E77A67EE877AC4ED257AC4F89850FDF7AA
:10378000D7FEFDF7C3FA2046FFF782FF3CF0A2FD0B
:103790000546D4F89400F8F7B7FE194ACDE90001C0
:1037A0000621284635F0A6FF0AE037EE676AF7EEF5
:1037B000005AB0EEC66AB4EEE56AF1EE10FA01DC2A
:1037C00006B070BDB0EEE76AB4EEE66AF1EE10FA4C
:1037D000F6D4002ECFD02046903080ED007A2EF027
:1037E00041FE3CF077FD074A012106B0BDE870407C
:1037F00035F080BFEC250020000000340AD7233CC0
:10380000C9410908A4410908F0B52DED048B85B024
:1038100004464FF4537200F5867103A80FF034F894
:10382000D4ED227AD4ED236A9FED796A637C37EE7A
:10383000E67A2422B0EEC77AB4EEC67AF1EE10FA38
:10384000C1BF9FED747A67EE877A9FED737AE6EEDB
:10385000877A02FB03430025C4ED237A93F839608D
:103860002378E9B28B4206D904EB8103013558680D
:1038700054F0B4FCF4E7DFED698A9FED698A9FEDAF
:10388000699A0027237CFDB2AB4264D9242303FB51
:10389000054393F83920002A5BD0D3ED0C7AF4EE7F
:1038A000E87AF1EE10FA0BDBF4EE677AF1EE10FA3B
:1038B00006D6F0EEE77AF4EE487AF1EE10FA04DD7F
:1038C000242303FB05435A6A1A63242303FB05439D
:1038D000D3ED090AD3ED0D7A93F8382070EEA70ADC
:1038E000A2B993ED0C0A2046FFF746FDD4ED257AE8
:1038F00030EE670AB4EE400AF1EE10FA16D7242330
:1039000003FB0545002385F83A3022E0012A09BF70
:10391000D3ED0C7A93ED0B0A77EEE00AD4ED3B7A07
:1039200004BF80EE897A87EE270AE3E7F0EEC07ADB
:10393000F4EE487A2423F1EE10FA03FB0545E1DCAE
:10394000012385F83A30D4ED237A37EE800A85EDED
:103950000B0A013796E7627C20461146FFF788FE86
:1039600048B1242101FB024292ED0B0AD16904F116
:10397000A80034F0D1FF94F99C10277C002907DBC4
:10398000B94205DACAB211462046FFF771FE68B99E
:1039900000226274D5B2AF4209D929462046FFF70A
:1039A00067FE01320028F5D0657400E0627420469D
:1039B000FFF7AAFE2046FFF74DFE10B1204654F057
:1039C00013FD637C242505FB034393F83930B34290
:1039D00016D032F007FF4FF6FF7132F029FD78B1B3
:1039E000607C05FB004494F83930002B14BF0022A2
:1039F0000422019232F0F6FE019A122132F0AAFC62
:103A000003A80EF063FF05B0BDEC048BF0BD00BF52
:103A10000AD7233C0AD7A33C48E17A3F0000003490
:103A2000FFFF7F7F002019462DE9F04F0446007C00
:103A30000F4687B004F13A0300220121D5B2A84213
:103A400003F1240305D903F8231C03F8241C0132D5
:103A5000F4E76F4B1E68F06A03685B68984740B1F3
:103A60003CF038FC6B4A062107B0BDE8F04F35F05A
:103A700041BE3CF02FFC684A062135F03BFE002396
:103A800003A904F1880003932FF0A2F80A2553F04C
:103A900045FB80462046FFF7B7FE53F03FFBA0EB07
:103AA0000800B0F5FA7F02D95C4800F063FFB06A05
:103AB00003680A215B689847617C2046FFF7D8FDC0
:103AC0000028E7D0B06A036864215B68013D98472D
:103AD00015F0FF05DBD1524B05951B888DF806507C
:103AE000CDE90355ADF80430052553F017FB8046AA
:103AF0002046FFF789FE53F011FBA0EB0800B0F55C
:103B0000FA7FD1D8617C2046FFF7B2FD0028EFD0C4
:103B100094F810B00DF10C08A14601AA4FF0000A6C
:103B20005FFA8AF18B4516D92046FFF7A1FD50B107
:103B3000D8ED007A99ED097A137877EE877A013318
:103B4000C8ED007A13700AF1010A08F1040809F1BE
:103B500024090132E4E7B06A036864215B68013D2F
:103B6000984715F0FF05C0D1A9464FF02408237CE3
:103B70005FFA89F6B34226D906AB334413F8143CF6
:103B800033B908FB064686F83B3009F10109EEE738
:103B9000002FFAD007EE903A06AA02EB8602F8EE62
:103BA000E77A12ED030AD4ED250A204680EE270AB3
:103BB000FFF730FC08FB064002A930308DED020A09
:103BC0002FF006F8E1E7617CDFF85C902046FFF714
:103BD000D1FC002684ED3D0A4FF02408237CF7B287
:103BE000BB420FD908FB074393F83B3043B13CF08D
:103BF00071FB7B1C4A46062135F07CFD0135EDB298
:103C00000136EBE70DB907484FE707B0BDE8F08F85
:103C1000EC250020E44109080F4209082542090863
:103C2000A4FD0808614209083F42090808B5037C61
:103C3000022B02D9034853F03FFA5A1C027418466B
:103C400008BD00BF8042090838B5057C0246002443
:103C5000E1B28D4206D91046FFF70AFD0134002873
:103C6000F6D138BD281E18BF0120FAE770B50D4601
:103C700009780729044606D8027E437E22B901222C
:103C80008A401343437670BD002BFCD00026227877
:103C9000F3B29A42F7D904EB8303294658680368C4
:103CA000DB6898470136F2E737B50D460192FFF71A
:103CB000CBFF0199044630B90448054B00682A46F9
:103CC000C06A0EF0BFFF204603B030BDEC250020D7
:103CD0008B6B0A08014B1868704700BFA45A00207C
:103CE00010B50446006810B103685B689847204629
:103CF00010BD000010B50446006810B103685B6891
:103D00009847204610BD000070B5D0ED247A9FED95
:103D1000427AF0EEE77AF4EEC77A0123F1EE10FA78
:103D20008AB00446037609D49030002309A905908F
:103D300009932EF04DFF05982EF094FB0026E663C4
:103D40002666C4F88460762231462046FFF760FC80
:103D5000054600283BD0CDE90666079A0992002364
:103D600009A92046CDE9073354F066FE01462046F6
:103D7000FFF73AFC09A8FFF7BDFF08A8FFF7BAFF55
:103D800007A8FFF7ADFF15B106A8FFF7A9FF237835
:103D9000032B3FD0237C032B3CD0D4F80031DA0432
:103DA00003D5637E0BB9012363760025637EEB4068
:103DB000DB07EAB21AD40135082DF7D123781BB1FD
:103DC000237C0BB163682BBB144800F0D3FD144B6C
:103DD0001B68596804220B68CDE90102114A009260
:103DE0001E680246762307A8B047B6E7382005923A
:103DF00001F0F8FE064618B1059A214654F068FB1A
:103E000031462046FFF7F0FB2378032B02D0237CBA
:103E1000032BD0D10AB070BD0000003494420908D1
:103E2000EC250020801A060090F81835934207D937
:103E300002F59E7250F8220010B103689B6A184781
:103E4000002070472DE9F34105466E4686E80C00D8
:103E5000134B45F8043B04460F4600F5C878284646
:103E60002C3500F08DFCA845F9D196E8030004F24A
:103E70001C53C4F8147583E80300089BC4F8243568
:103E8000084920462EF016F9074B1A6812B1074868
:103E900053F012F920461C6002B0BDE8F08100BF6B
:103EA0008846090850450908A85A00209444090882
:103EB0002DE9F041A2B00C4607A92DF0D1FB002856
:103EC00055D000210D220CA80591ADF818100B91CA
:103ED00077F0D2FE2B4B611C1F68C9B20BAD0129D4
:103EE000F86A0A9546D1284B062205A90EF0AAFECB
:103EF000264B019305AB0093002411222946244B45
:103F0000F86A8DF819400EF09DFE04AA0DF10F011C
:103F100028468DF83C4004942EF038FD38B31D49F6
:103F2000DFF86C80482210A877F05CFE062610AC03
:103F30002268531E049AC2F3513202EB8312237992
:103F40008DF82430A368019305AB00930892434693
:103F500011222946F86A0EF075FE0021B7EE000A1C
:103F600007A82DF07FFD013E04F10C04E0D122B042
:103F7000BDE8F0810091084B062205A90EF062FE13
:103F8000B6E700BFEC25002025340908C544090820
:103F9000BF440908A8FD0808B84409082DE9F04FF6
:103FA00090F8186585B00446002E59D17F2380F81B
:103FB00028350DF10F01042328308DF80F302EF035
:103FC00043FE04F5C87504F59E68271D5FFA86FA5E
:103FD0001822FF21284677F04FFE85F857A097F961
:103FE0002490B9F10A0F59D03DDCB9F1040F0FDC70
:103FF000B9F1020F0FDD442001F0F4FD834620B13A
:104000003B462A46214654F0C9FDC8F800B002E0FC
:10401000B9F1090F36D0D8F8000050B1E96DC5F8F4
:10402000589031B1244B43F826102EF051FA2EF05F
:1040300047FA58F8040B0AF101095FFA89F940B10F
:1040400003689B68984784F8189551462046FFF707
:104050002FFF0136092E05F1600507F12C07B5D1B8
:1040600005B0BDE8F08FB9F1190FD4D1482001F0A7
:10407000B9FD83460028C8D03B462A46214655F064
:1040800007FCC2E7382001F0ADFD83460028BCD014
:104090003B462A46214655F0DBF9B6E7302001F0D1
:1040A000A1FD83460028B0D0CDF800A03B462A46AB
:1040B000214655F06FFBA8E7AC5A002090F8183560
:1040C0008B4283BF602303FB010090F8D5010020E1
:1040D0007047000090F818358B4283BF602303FBC4
:1040E000010090ED6A0A9FED010A70470000000090
:1040F00090F818358B4206D901F59E7150F82100D1
:1041000008B154F0DFBE9FED010A704700000000C7
:1041100010B490F818458C420A4614D901F59E74E3
:1041200050F824407CB1E468246A640603D55DF845
:10413000044BFFF7DDBF602101FB020393ED6A0A28
:104140005DF8044B70479FED010AF9E7000000009D
:1041500090F818358B420BD901F59E7150F821006B
:1041600038B1C3681B6A1A4214BF0120002070478F
:104170000020704770B590F81835934204460E46FB
:10418000154601D8002070BD02F59E7350F823003B
:104190000028F7D003689B6998470028F2D0602276
:1041A00002FB0544D4F8AC313360ECE770B590F80D
:1041B0001835934204460E46154601D8002070BDBE
:1041C00002F59E7350F823000028F7D003689B691E
:1041D00098470028F2D0602202FB0544D4ED6C7AA7
:1041E000F4EE677AF1EE10FAE8D6C6ED007AE6E76B
:1041F00070B590F81835934204460E46154601D81E
:10420000002070BD02F59E7350F823000028F7D0FF
:1042100003685B6998470028F2D0602202FB0544DE
:10422000D4F8B4313360ECE790F8183593420ED9E6
:1042300002F59E7350F823305BB1602303FB02024A
:1042400092F8E40130B1D2F8E0310B607047002001
:10425000704718467047000008299DBF2C2303FBB8
:1042600001004068002070472DE9F04F4B4B2DEDC9
:10427000028B1B68DB6A93F89C3089B00446002BE4
:1042800000F08680DFF82CB19FED458A4FF00009E1
:1042900094F818355FFA89F5AB4279D905F59E7324
:1042A00054F8230000285DD003685B6B98476023B7
:1042B00003FB0543074693F8D431834252D20328C7
:1042C00061D8DFE800F04F025259364E4FF0000837
:1042D0003CF000F894F81825AA4284BF602202FB43
:1042E00005424FF0600105F1010301FB05458CBF5C
:1042F000D2F8A82118EE102A8246D5F8B001CDE9EF
:104300000632F8F701F9079ACDE904011046F8F7EB
:10431000FBF8069B0096CDE902015A46042150465F
:1043200035F0E8F90123204A84F8293585F8D4715D
:10433000D372D4F824354BB3002255B25957481CD8
:1043400003D0414502F10102F7D194F92835AB427F
:1043500008DBD4F82035D4F81C054246314698478E
:1043600084F8285509F1010992E72C2303FB054342
:104370000E4E93F92B80ABE72C2303FB05430C4E29
:1043800093F92C80A4E70026B046A1E71D46DCE7A0
:1043900009B0BDEC028BBDE8F08F00BFEC2500201A
:1043A00000000000D94409082D5B0020D2760A08DD
:1043B000D0440908E844090890F818358B4207D919
:1043C00001F59E7150F8210010B10368DB691847B0
:1043D0000020704708299CBF602303FB010000F503
:1043E000C870704790F81835934207D902F59E724D
:1043F00050F8220010B103685B6A1847002070472C
:104400002DE9F04F002493B005460E46174621468D
:104410002F2206A8059405F59E6977F02DFC05F17D
:10442000280A4FF02C0B05F5F4730BFB04F259F836
:10443000040B1AF90210E5B230B951B90134092C54
:10444000F3D14FF0010813E0602262439A58914281
:1044500012D01548154B006801930135EDB2009557
:10446000134BC06A324639460EF0ECFB4FF00008A1
:10447000404613B0BDE8F08F05A93322039354F0F2
:1044800003FE039B804605A90028D7D10648019169
:104490000135EDB200680095054BC06A32463946D9
:1044A0000EF0D0FBE4E700BFEC2500201E45090814
:1044B000104509082DE9F04FDFF88090DFF880A063
:1044C000DFF880B08DB00646002796F81835FCB2AC
:1044D000A3422ED9602505FB046595F8DC3133B382
:1044E00095F8DD1119BB4FF001082022444404A8BF
:1044F00089F8198077F0C0FB07EE904A4AF2104322
:10450000F8EEE77A03AA4C21ADF828305046242370
:10451000CDED037A36F0EEFF3BF0DCFE9BF8003089
:10452000054A0094042135F0E5F885F8DD8101376E
:10453000CBE70DB0BDE8F08F284509082D5B0020C2
:10454000DD5D0020282300202DE9F04F2F4B1E6851
:1045500085B0044646B1D0F81415304631F068FFF6
:1045600010B1304630F014FF52F0D8FD4FF0000883
:1045700001904FF02C0A4FF0600B94F818355FFA59
:1045800088F5AB4239D904EB8507D7F8F00488B336
:104590000AFB05430BFB054993F92820D9F8E811DC
:1045A0008A4227D132B30268D2689047D7F8F00424
:1045B0000268126B904799F8D52112B1019BC9F896
:1045C000D831BEB1D4F81415304631F031FF88B17E
:1045D00052F0ACFDCDE9021002460B46D7F8F004CC
:1045E000294654F049FFDDE90232D7F8F0042946A4
:1045F00054F0C0FF08F10108BFE72046FFF734FE82
:10460000204605B0BDE8F04FFFF754BF505D0020D5
:104610002DE9F0474FF000082DED028B0446894646
:10462000B0EE408A474601264FF0600A94F81835EC
:104630005FFA88F5AB421AD929FA05F3DB070AD5E8
:1046400005F59E7354F8230078B10368B0EE480A6C
:104650009B6B984706400AFB054508F1010895F851
:10466000D4319F4238BF1F46E0E70646F3E727B93B
:104670007F23A4F82835034BDF72BDEC028B304654
:10468000BDE8F0872D5B002090F818358B4207D9E4
:1046900001F59E7150F8210010B10368DB6B1847DB
:1046A000002070470B46114690F818259A4207D90A
:1046B00003F59E7350F8230010B103681B6C184774
:1046C0007047000070B504460E46002594F8183572
:1046D000E9B28B4205D932462046FFF7E3FF0135A8
:1046E000F4E770BD2DE9F84390F818550246002410
:1046F00000F128062C2700F5F4784FF06009E1B2AC
:104700008D420FD907FB04F309FB04F0F35658F868
:104710000000834209D11BB11046FFF7CFFC10B156
:104720000134ECE70120BDE8F8830020FBE700003E
:1047300010B590F818258A42044617D9602202FB6A
:10474000010393F8D431022B03D004D9032B18BFF3
:104750000023184610BDFFF797FF48B92046FFF722
:10476000C1FF00280CBF06230123F2E70023F0E776
:104770000623EEE7014B1868704700BFA85A0020D7
:1047800010B5034904462DF095FC204610BD00BF2E
:104790000047090810B50446203044F08BFE044B56
:1047A00004491C6020462DF085FC204610BD00BF4A
:1047B000D05A0020844809082DE9F3410022B7EEC1
:1047C000000A022105462DF065FA284655F0B0F89A
:1047D00044F054FF234B1E680446F06A03685B6A8A
:1047E00098470B46022102460091204644F078FE8D
:1047F000B5F94A70002F13DDD6F82C80D8F80030B8
:1048000040465B68BCB2984728B198F84D3013B168
:10481000C92FA8BFC824B06A036821465B689847BF
:1048200095F949002022002111F0ECFBC4B245F0BB
:104830003BFD45F0D9FC70B9B06A036801345B6890
:10484000E4B205219847072CF1D9074802B0BDE82A
:10485000F04151F02FBD072CF7D885F8494002B040
:10486000BDE8F081EC250020F047090810B50446AA
:1048700055F02CF82046BDE8104055F057B8000020
:104880002DE98048284BDFF8A490DFF8A4A0DFF8DA
:10489000A4B01446012293B005460E461A704FF09C
:1048A000000852F03BFCD9F800300393A0EB08025B
:1048B00041F287339A4207461FD9CDE90056039843
:1048C0005346342205A9C06A0EF0BCF9214605A85A
:1048D000049451F0DFFCCDE9005603985B46342286
:1048E00005A9C06A0EF0AEF904943BF0F3FC049BFA
:1048F00005AA022134F0E4FEB8463BF0EBFC3AF0A6
:10490000E7FD3BF0E7FC3CF0F9FB0A2105A80DF0C0
:10491000A1FF039B986A036805215B68984705A877
:104920000DF0A4FFBDE700BFD45A0020EC25002005
:10493000D1B90908F9850A080FB400B595B016AACF
:10494000002152F8043B039205A83C2201930491F4
:1049500077F092F9054A019B402104A851F042FCEE
:10496000039A034804A9FFF78BFF00BF0848090812
:104970001E4809080FB407B504AA034852F8041BDF
:104980000192FFF77DFF00BF304809080146D0E9DA
:10499000070300B11847002BFCD17047B0F9023073
:1049A00002889A4314BFC3F3C00000207047000080
:1049B00038B507230380022200230525C0E905320C
:1049C000C0E90D33C0E91033C0E92C330C49036250
:1049D000C0F89C5004462DF06DFB0A4B196811B1CC
:1049E000094852F069FB94F910001C602A4611F046
:1049F00009FB637C207403F010036361204638BD1B
:104A0000D4490908D85A00201449090801234361F0
:104A10000423C36470470000002343610423C3647C
:104A2000704700000123C364704700000223C36481
:104A3000704700000323C3647047000010B5C369CA
:104A400093B190F9514090F950309C4207DA074BEE
:104A500007480068C06A0EF0F5F8002010BD036A30
:104A6000012B01D8034BF3E70120F7E73049090890
:104A7000EC2500203C490908F8B504463CF0B6FE98
:104A80003CF0A0FE3DF05EFD07463CF0AFFE3CF082
:104A9000A3FE3DF057FD06463CF0A8FE3CF07EFE2E
:104AA0003DF050FD05463CF0A1FE3CF081FE3DF09E
:104AB00049FD0246606C50B101285FD1012E5DD1E5
:104AC000012A5BD1012D14BF00200820F8BD012F61
:104AD00028D176B9012A61D1012D63D1627CD70733
:104AE00005D494F9511094F95020914210DA022023
:104AF000ECE7022E16D1012A50D1012D52D1627C51
:104B0000D60741D494F9511094F9502091423BDBDF
:104B10006269216C8A421AD0002A33D0012A08BF68
:104B20000A20D3E7002D3BD0012E0BD1012A09D159
:104B3000022DEDD12046FFF731FF002814BF0420DD
:104B40000320C3E7E2B1022AE2D10620BEE7E26C0D
:104B5000A16B8A42BAD0012A1DD1617C0D0715D400
:104B6000617C490710D4022A12D1617C0B070DD455
:104B7000627C12F0040F18BF0220A7E70020A5E70F
:104B80000520A3E70920A1E701209FE710469DE744
:104B9000042A9BD1ECE7032AE5D1E1E7002DD1D12E
:104BA000072093E7002DB3D1FAE700004B6A022BF0
:104BB0004FF0000303D080F84830436470478A68A0
:104BC000032A05D0042A05D0002380F84830704716
:104BD0004364F9E70B680A7B5B78012A03F00F0353
:104BE00005D0022AF0D1002BEED00262ECE7002BB8
:104BF000EAD005230362E7E7FFF7D8BF037C033B56
:104C0000022B94BF0120032070470000037C033B6C
:104C1000022B94BF0120042070470000C06910B12E
:104C200003681B6A1847704770B50446C06903687B
:104C300000215B6C9847E069036801219B6C9847F1
:104C4000E06903680021DB6B9847E5692B6828461B
:104C5000D3E90D63984740F4407081B22846B047CD
:104C60000A23E0691A464FF4E1310DF0B9FEE0691C
:104C70000368BDE870401B6A184700000339042927
:104C80009ABF024B58560020704700BFCC49090814
:104C9000F7B5C36904466BB3E2B9012915BF002318
:104CA000012303270427CC208DF804008DF805107C
:104CB0000BB18DF80620002630467D1EF3B2AB42C4
:104CC00006F1010609DA02AA134413F8041C11F0D4
:104CD00045FAF3E701230427E5E702AB1D443A4612
:104CE00005F8040CE069036801A9DB689847E069EE
:104CF0000DF0D2FE03B0F0BD10B5C4693CB18469BB
:104D0000012C06D1C262CAB22146FFF7C1FF20467C
:104D100010BD0020FCE70000042910B5044604DCA7
:104D200002290DDC01290ED010BD0A29FCD1FFF7A4
:104D300065FFE26801462046FFF7DEFF032306E039
:104D4000437C9B07F0D5FF23A4F852300423236251
:104D5000EAE7000010B590F8513080F85030044672
:104D600044F0DEFD20B100F58050002380F884344B
:104D70006369012B0DD163885B060AD52046FFF7D6
:104D80003DFFE26801462046FFF7B6FF032323629A
:104D900010BD0223FBE70000013938B5044606299F
:104DA00069D8DFE801F0042031688B8BB60090F9F8
:104DB0005030002B5FDC013380F85030C268022194
:104DC000FFF79AFF94F95030002B0ADD44F0A8FD5C
:104DD00020B100F58050012380F88434052323623C
:104DE00049E00423FBE790F95030002B08DD013B3C
:104DF000C26880F850300221FFF77EFF0623EEE7FD
:104E0000BDE83840FFF7A6BF90F9503090F9521036
:104E1000012B20DD90F91000484D421EC2EBC2026A
:104E2000AB18AA5C2AB353FA81F394F853205B7849
:104E3000013B9A421DD105281BD0A26800212046C3
:104E4000FFF75AFF002384F8533094F85030013BA9
:104E500084F850300FE00CD190F910203748531EE1
:104E6000C3EBC303C35C23B1013B994201D1052AC3
:104E700002D100290BDA38BDE26800212046FFF795
:104E80003BFF94F85030013B84F85030B6E794F97A
:104E900010302A4A013BC3EBC30313440B445B7835
:104EA000002BE8D0A26800212046FFF725FF94F9E7
:104EB00050300133022BA8BF0223C9E701218268C9
:104EC000FFF71AFF94F950301C49012B94F9103068
:104ED00011DD013B94F8520094F85320C3EBC30357
:104EE0000B44034401325B78B2FBF3F103FB112264
:104EF00084F85320BFE7013BC3EBC30394F952206E
:104F0000CB5C013292FBF3F103FB112284F85220B7
:104F1000B1E790F95030002B09DD013B80F85030AB
:104F20000023C26880F853300221FFF7E5FE94F9B0
:104F30005030002B9FD194F85130A5E70D2200206E
:104F400010B54369012B044610D143885B060ED58A
:104F5000437CD90607D4FFF751FEE26801465200B0
:104F60002046FFF7C9FE0323236210BD0BB10223C5
:104F7000FAE743885A06FAD5437CDB06F7D5FFF7F4
:104F800045FEE268014652002046FFF7B5FEEEE717
:104F9000042910B5044604DC02290DDC01290ED0D9
:104FA00010BD0929FCD1FFF731FEE2680146204619
:104FB000FFF7A2FE02230EE0437C9B07F0D52046BC
:104FC000FFF724FEE26801462046FFF795FEFF2327
:104FD000A4F8523004232362E2E7000010B504462F
:104FE00052F09CF8A36AE26AC31A934207D3226A7A
:104FF000A0620023022AE36202D0032A10D010BD6F
:105000006269012A0AD1638813F0400F0CBF0021A6
:105010000A212046BDE81040FFF77EBE1946F8E79A
:10502000616949B9638813F0400F18BF0921204610
:10503000BDE81040FFF7ACBF1946F8E773B50B6841
:105040005B78836143885B045EBF0B685B88438049
:10505000B0F90230002B04461ADD012303623BF055
:1050600039F905462046B4F90260FFF797FC68B9A4
:105070002388B3430CBF022300230093094A33461D
:105080000621284634F036FB02B070BD0523F4E754
:105090003BF020F9044A042102B0BDE8704034F02E
:1050A00029BB00BF5049090881490908FFF7C6BF5D
:1050B00070B50446D0F8B8000E46E8B1D4F8A83070
:1050C00023B1D4F8A420CB1A934221D3B4F8AC5026
:1050D0009DB12046FFF7A8FDD4E9260194F8A02051
:1050E000FFF7D6FDB4F8AC30C4F8A8600020013B4F
:1050F00084F8A100A4F8AC3070BD042304F194003E
:10510000C4F8B830FFF742FCC4F8B8502846F3E7BB
:105110000120F1E738B50024054620466B7BA34209
:1051200005DD2B68195D11F019F80134F6E738BD7B
:105130002DE9F041C3690446002B43D051F0EEFF46
:1051400001462046FFF7B4FF00283BD0E069036822
:105150005B699847402828BF40200025064604F197
:105160009407A846AE422DD051F0D8FF0146204604
:10517000FFF79EFF30B3E06903689B69984794F896
:10518000A130C0B20BB9CC281AD1D4F89420D05495
:1051900094F8A13094F8A2200133DBB29A4284F84B
:1051A000A1300DD13846FFF7B5FF00280CBF022310
:1051B0000323C4F8B8303846FFF7E8FBC4F8B880DA
:1051C0000135CFE7BDE8F081074A002352F83300EC
:1051D000884203D102EBC303187970470133042BD3
:1051E000F4D10020704700BF3022002038B503738F
:1051F00000234373049B03611546BDF8143085609A
:1052000001F154020446C0E90021038300F11C03AC
:10521000DDE9060183E803000123636251F07EFFAC
:10522000294660612046FFF7CFFFA073204638BDB6
:105230002DE9F0438FB016AC064634F8049B0F46B8
:1052400090461D46FFF7EAFC94E8030002AB83E8B2
:1052500003003A46CDE900594346314604A804AC60
:10526000FFF7C4FF0FCC06F194050FC50FCC0FC597
:1052700094E80300424685E80300394630460FB003
:10528000BDE8F043FFF704BD10B586B0094B0593A8
:10529000049006AA12E9030001AB83E80300002290
:1052A0004FF6FF73009311464FF47A63FFF7C0FF88
:1052B00006B010BDAD50010813B51A4B044618686E
:1052C00020B100221A212EF0BDFCE061E36953B148
:1052D00001230DF1070104F110008DF807302DF0C6
:1052E000B3FC2DF0EDF894F9103013B9E36102B07E
:1052F00010BDE269002AFAD0022B01D0052B03D1A0
:105300004FF6FF73A4F850302046FFF78DFC51F0A4
:1053100005FF6368A0622046E36202B0BDE810406A
:10532000FFF7B2BFFC5B002030B587B004AB83E869
:105330000600054693E8030001AC022384E805005B
:105340000421009301224FF4C8732846FFF770FF31
:1053500007B030BD30B587B004AB83E80600054622
:1053600093E8030001AC84E80500022200924FF4A8
:10537000C87304212846FFF75BFF07B030BD00006B
:1053800010B586B006AC04E90C0061B10124446498
:1053900001AC84E80C000224CAB200944FF4C87334
:1053A0002146FFF745FF06B010BD000070B586B07E
:1053B00004AB83E8060002254564044693E8030035
:1053C00001AE86E805004FF4C87300950022032162
:1053D0002046FFF72DFF06B070BD000010B5012379
:1053E00080F848304B1E88B00446C262072B31D883
:1053F000DFE803F0040E181818181825164B009053
:105400001A460146019308B0BDE81040FFF78CBF73
:10541000114B02901A460146039308B0BDE81040B4
:10542000FFF798BFFFF72AFC0B4B04940146224676
:105430002046059308B0BDE81040FFF7A1BF064B1A
:105440000793069008AB13E9060008B0BDE81040CA
:10545000FFF7ACBF08B010BDF94B01084B1E10B5EB
:105460000446092B20D8DFE803F00C233636363605
:1054700036053636642208212046BDE81040FFF785
:10548000ADBF90F9503083B944F04AFA20B100F52D
:105490008050012380F88434642201212046FFF7E4
:1054A0009DFF012384F8503010BD64220321E3E7FF
:1054B00090F95030002BF7DD44F032FA20B100F5BE
:1054C0008050002380F88434642202212046FFF7B4
:1054D00085FF0023E6E76422CEE7000013B504460B
:1054E0000191FFF75BFA019928B1204602B0BDE8AF
:1054F0001040FFF7B3BF2388B4F90220934305D1CE
:10550000204602B0BDE81040FFF746BC02B010BD17
:1055100070B5044651F002FE94F8482022B9A36AFF
:10552000E16AC31A8B4202D20023236370BDC4E92F
:105530000A022046FFF7A0FA236B62698342014604
:10554000236AE06C0ED1656BAB420BD1A56B854233
:1055500008D194F93C6094F95050AE4202D1256CC8
:105560009542E3D0C4E90C13A063013B94F85000CA
:1055700084F83C002264052BD8D8DFE803F0030848
:105580000D1213182046BDE87040FFF7D9BC204625
:10559000BDE87040FFF7C0BB2046BDE87040FFF794
:1055A000F7BC01212046BDE87040FFF797BF0221FC
:1055B000F8E7000010B50D4B1B68DB6A93F89C30D0
:1055C000044623B12046BDE81040FFF707BD44F074
:1055D000A7F928B100F5805393F86434032BF1D870
:1055E0002046BDE81040FFF793BF00BFEC25002028
:1055F00038B5C36904467BB190F9103063B1FFF749
:1056000097FD51F08BFD636AC31A642B054603D9DD
:105610002046FFF7CFFF656238BD0000014B1868D8
:10562000704700BFD85A002008B50449102276F010
:10563000C9FAB0FA80F0400908BD00BFDC5A00206A
:105640001022002176F018BB10B50446FFF7F8FFD2
:10565000204610BD0378416023F00D03022A037039
:1056600008D0032A0AD0012A03D1DBB243F0010398
:1056700003707047037843F00803F9E7037823F0D9
:10568000050343F00503F3E773B504460E461546DC
:105690000193FFF7D5FF2046C4E90265069A0199F8
:1056A000FFF7D8FF02B070BD0078420704D40307AB
:1056B00004D400F0010070470320704702207047B7
:1056C000F0B587B004461546FFF7EEFF88420F4657
:1056D000064605D163682B600126304607B0F0BD51
:1056E00000230328019301D0032913D12EF05EFE7D
:1056F00008B90026F1E7012301AA21462EF092FC09
:105700000028F6D0DDED017A9FED337A67EE877AD7
:10571000CDED017A032E32D8DFE806F00209162417
:105720006468032FE5D8DFE807F02C2E3C49FBF72F
:10573000FFFE90F87C32DB07DBD56468FBF7F8FEF0
:10574000D0F870321C44ECE702A8FFF779FFFBF7B2
:10575000EFFE02A9FBF7F2FC06460028BDD0646804
:10576000039BEFE7D4ED017A9DED017AF8EEE77A3D
:1057700077EE877AFDEEE77A17EE904AD1E70024BC
:10578000CFE72C60A8E7FBF7D3FE90F87C6216F019
:105790000106AED0FBF7CCFED0F87032E41A2C60D4
:1057A0009BE702A8FFF74CFFFBF7C2FE02A9FBF73D
:1057B000C5FC0646002890D0039BEFE707EE904A11
:1057C0009DED017AF8EEE77A77EEC77AFDEEE77A9B
:1057D000C5ED007A80E700BF0000C84273B501AA9A
:1057E00005460E46FFF76CFF044620B1019932468C
:1057F0002846FFF72FFF204602B070BD13B51446B0
:1058000001AAFFF75DFF48B1DDED017A9FED047A53
:10581000F8EEE77A67EE877AC4ED007A02B010BD41
:105820000AD7233C07EE900A9FED090AF8EEE77AC3
:1058300008B527EE800A73F017FEDFED067AB4EEA6
:10584000E70AF1EE10FAD8BFB0EE670A08BD00BF54
:1058500050E0EF300AD7233C10B50446806810F0C2
:1058600025FD20B1E068BDE8104010F033BD10BD4B
:105870000D4B83424FF000038B4106DA00F12550B7
:1058800000F5311000F5E0507047084B98424FF09A
:10589000FF3371EB0303BEBF00F1564000F5130068
:1058A00000F52440704700BF00D2496B002EB6942B
:1058B00090EA010F01D4401A7047C317401A63EBF6
:1058C000E1710D4B83424FF000038B4106DA00F18A
:1058D000255000F5311000F5E0507047074B984215
:1058E0004FF0FF3371EB0303BEBF00F1564000F5EC
:1058F000130000F52440704700D2496B002EB69487
:1059000070B52DED028B84B0044668460D46FFF756
:1059100097FEFBF70DFE6946FBF710FC064608B341
:10592000A368029ADFED128A03999B1A07EE903A58
:10593000F8EEE77A67EEA87AC5ED007AE068FFF73F
:10594000B7FF08EE100AA068024402EBD272B8EE6C
:10595000C88A5010FFF766FF28EE288A28EE000A52
:1059600085ED010A304604B0BDEC028B70BD00BF6E
:10597000F67C8E3F37B500230C4601AA022105466E
:105980000193FFF79DFE10B9002003B030BD214602
:105990002846FFF7B5FF0028F6D0DDED017AF8EED6
:1059A000E77AC4ED027AF0E738B52DED028B0C46AC
:1059B0000246C168E068FFF77BFF9568A46808EEBF
:1059C000100A601900EBD0704010641BFFF72AFF2B
:1059D00007EE904AF8EEE77AF8EEC80A87EE807A8A
:1059E000BDEEC70A10EE103A5B4200EE103AB8EE78
:1059F000C00A73F05BFFDFED087A30EE270ABDECDA
:105A0000028BB5EEC00AF1EE10FA44BFDFED037A67
:105A100030EE270A38BD00BFDB0FC93FDB0FC9409E
:105A200030B52DED028B0B4685B08C68D0E9025164
:105A3000D868FFF73DFF08EE100A601900EBD07040
:105A40004010FFF7EFFE641B07EE904AF0EE400AAD
:105A5000B8EEC88A9FED060AF8EEE77A28EE008ACB
:105A600027EE800A68EE200A05B0BDEC028B30BD3F
:105A70008262363C82B002B0FFF7D2BFF0B52DEDA6
:105A8000028B0D4689B08C680646D0E90271E86841
:105A9000FFF70EFF08EE100AE01900EBD07040107F
:105AA000FFF7C0FE73686A689FED0E1A9B1A07EE37
:105AB000903AE41BB8EEE77AF0EE400A07EE904A1F
:105AC0009FED090AB8EEC88AF8EEE77A28EE008A58
:105AD00027EE011A27EE800A68EE200A09B0BDEC15
:105AE000028BF0BD0AD7233C8262363C10B52DED07
:105AF000028B84688A680B46111B08EE901AC168F5
:105B0000D868FFF7D5FE224402EBD27208EE100AE5
:105B10005010FFF787FEB8EEC88AF8EEE88A28EE44
:105B2000000A20EE000AA8EEA80A74F009F8BDECFD
:105B3000028BDFED027A20EE270A10BD8262363C2E
:105B4000094B984206DDC0F1D64000F5930000F500
:105B5000A4407047054B9842BEBFC0F1144000F509
:105B6000360000F53850704700E9A43500175BCACD
:105B7000F8B52DED028BDFED148A076820EE280AB8
:105B80000646FDEEC07A0D4617EE904A04EBD4703F
:105B900007EB6000B0EE608AFFF744FE28EE288A2B
:105BA0003819C8EE007AFFF7CBFF306017EE900A85
:105BB000F7F7D4F92B68C01841EBE371FFF758FEF3
:105BC000BDEC028B2860F8BD02AAB34200F10C01C3
:105BD0000830FFF7CDBF00000148FFF731BD00BF1F
:105BE000DC5A00200121884238BF084671F078BD98
:105BF000FFF7F8BF08B171F077BD7047FFF7FABF44
:105C000000214FF0FF3310B500220363044601600A
:105C10000171C0F80510417280F8251000F13C03B5
:105C200000F50B70D9709A60DA601A615A619A6156
:105C3000DA611A625A629A62DA631A645A649A647E
:105C4000DA641A655A659A65DA65DA661A675A6718
:105C50007C339842E6D1214604F5167007F0AAFA83
:105C6000044B1A6822B904491C6020462CF022FA21
:105C7000204610BDEC5A00200C4C090873B5D0F832
:105C80003C3201919942044613D0D0F840329942F7
:105C900018D0D0F844328B4216D102200AE0D4F852
:105CA000343253B3D4F838324BB34FF0030002B060
:105CB00070BD002094F822308342F8D8431C84F849
:105CC0002230F4E70120F5E7D0F83062002EE6D16B
:105CD00094F841233546B6009AB1A319C3F830129F
:105CE000A319019AC3F83C2294F82230AB429CBF1E
:105CF0006B1C84F822302846D9E70126E8E7022603
:105D0000E6E704F50C7001A930442DF06FF8E7E7E1
:105D100038B504460D462CF0DFFF291D201D2CF060
:105D2000DBFF05F1080104F108002DF0AFF805F1E3
:105D3000140104F114002DF0A9F805F1200104F17B
:105D400020002DF0A3F805F12C0104F12C002CF01B
:105D500057FF05F1300104F130002DF05FF805F137
:105D60003C0104F13C002DF091F8AB6BA3636B6B2D
:105D7000636338BD2DE9F043A1B00023002500F195
:105D80003C0706468DF8075003930493059306934A
:105D90000793089309930A930B931093119312930B
:105DA0001393149315931693179318931C931D93A1
:105DB0001E9300F50F78B94658F8043BF3B1F26E24
:105DC000934223D0D6F8E820934221D0D6F864211C
:105DD000934213D10221EBB299420FD0C1EB411192
:105DE00009EB8104214601A8FFF792FF39462046BE
:105DF000FFF78EFF01A93846FFF78AFF0135032D13
:105E000007F17C07D8D121B0BDE8F0830021E2E79B
:105E10000121E0E72DE9F04706460F46154680468A
:105E200004464FF0000A39463046FFF727FF626FFD
:105E3000BA425FFA8AF90ED1C3B2022B0BD87C2288
:105E400002FB0A66012086F83E0086F83F3085F89E
:105E50000090BDE8F0870AF1010ABAF1030F04F1DE
:105E60007C04E0D1002439463046FFF707FFD8F81C
:105E70006C205FFA84F912B9C3B2022B22D9013423
:105E8000032C08F17C08EED100244FF07C0906F1C8
:105E90003E0A39463046FFF7F1FE034609FB04F09F
:105EA0005FFA84F81AF8002012B9DBB2022B12D97B
:105EB0000134032CEDD196F82300042814D9194895
:105EC00051F0FAF87C2000FB0464012084F83E00C5
:105ED00084F83F30BBE70644012086F83E0086F890
:105EE0003F3085F80080B4E706F54371002251F891
:105EF000043BBB42D4B208D1A04202D8631C86F84E
:105F0000233003342C700020A3E73BB9421C06EB7E
:105F1000800086F82320C0F80C73F2E70132052ACE
:105F2000E5D1F0E7444A0908C9B200EB8101D1F894
:105F30003C3253B1026F93420AD0D0F8EC20934226
:105F400008D0D0F86821934206D04FF00300704784
:105F500000207047012070470220704759B190F827
:105F60002030032B07D05A1C80F8202000EB830040
:105F70004161012070470020704700002DE9F8437F
:105F80000F469146044600F5BA7894F83E5035B96C
:105F90007C344445F9D100252846BDE8F883002328
:105FA0004A46394601200CF0E3FA00210646E06E2D
:105FB0000CF0EEFA8642EBD1EEE700002DE9F0435B
:105FC000DFF87C8085B0044600F50F7600257C273D
:105FD000B14656F80C3CD9F800209342E9B206F1DC
:105FE000040619D1C3B12046FFF79EFFC0B207FBDC
:105FF000004090F83E307BB903A9A9F10C0003934F
:106000002CF0F4FE3AF066F956F8043C0093424650
:106010002B46012133F06EFB0135032DD8D104F15D
:106020006C0504F5F074296821B9AB6813B12846F2
:106030002BF032FB7C35A542F5D105B0BDE8F083ED
:10604000604A090838B504461546FFF76DFFC0B22F
:10605000022808D87C2303FB004029465030BDE8C5
:1060600038402CF003BF38BD38B504461546FFF75D
:106070005BFFC0B2022808D87C2303FB00402946FE
:106080005C30BDE838402CF0F1BE38BD37B50D4668
:1060900004468DED010AFFF747FF022D07D8C0B275
:1060A0007C2303FB004001A968302CF091FD03B074
:1060B00030BD000038B50546FFF736FFC4B2022CEC
:1060C00013D8C4EB4414A4003C3504F10800284460
:1060D00000212BF0E1FA04F1340104F130002944ED
:1060E0002844BDE838402CF081BE38BD70B5054667
:1060F0000E461446FFF718FFC3B2022B0DD87C20C2
:1061000000FB035394E80700443383E8070031465B
:106110002846BDE87040FFF7CDBF70BD37B50446D7
:106120001546FFF701FFC0B2022809D87C2303FB04
:1061300000400DF1070140308DF807502CF0CCFDE8
:1061400003B030BD10B500210446FFF7B3FF204671
:106150000121FFF7AFFF20460221BDE81040FFF705
:10616000A9BF00001FB590F92C30044623B390F965
:1061700021300BB36846FFF767FAFBF7D9F9694698
:10618000FAF7B8FFC0B1DDED037A9FED0C0AF8EE27
:10619000E70ADDED027AF8EEE77A0123C0EE800A25
:1061A00084F83D3387EE800A07F046FADFED047A83
:1061B00020EE270A84ED0A0A04B010BD8096184B21
:1061C00035FA8E3C024690F9210058B192F840030E
:1061D00040B1114491F92C0220B192F92400033806
:1061E00018BF01207047000038B590F822300546EE
:1061F0005BB100242346E1B22846FFF7E3FF08B174
:106200000133DBB20134032CF5D1184638BD000050
:1062100090ED0A0A7047000038B50C46D1ED066AC9
:1062200011460546FFF780FEC3B27C2000FB0353F6
:10623000D4ED087AD3ED260A94ED076AD3ED255AFA
:1062400093ED245A26EE600A67EEA00AA5EEA70A8F
:10625000F0EE607AE5EE867AB7EE007AA6EEE67AA0
:1062600067EEE60AB1EE400AE5EE070A73F01EFBA0
:106270009FED071ADFED070A40F61C000FF084FEC1
:10628000D5ED0A7ABDE8384030EE270A0FF068BE37
:10629000DB0F4940DB0F49C02DE9F04190F8223077
:1062A0008B4204460D4602D20020BDE8F081FFF784
:1062B0003BFEC0B204F13C06C0EB401006EB800090
:1062C000083012F06DFADFED157AB0EEC00AB4EEC8
:1062D000E70AF1EE10FAE7D429462046FFF724FE3C
:1062E000C5B27C2000FB05473B6F002BDCD0032DA3
:1062F000DAD000FB05603030D7F86C802BF0B0FFAF
:10630000D7E91B32934201D1984505D07C2000FB90
:106310000544C4F86C80C7E70120C6E700000034DC
:106320002DE9F74F04460E46174600F50F7A4FF059
:10633000000B5AF8049B5FFA8BF8B9F1000F26D0D6
:1063400041462046FFF73EFF08B341462046FFF78F
:10635000EBFD7C23C0B203FB004090F83E505DB9DA
:1063600008F101031B4ADBB2394630464FF03AFFD1
:10637000284603B0BDE8F08F5AF8102C914506D09E
:10638000154A394630464FF02DFF0025F0E70BF156
:10639000010BBBF1030FCCD14FF0000894F8223071
:1063A0005FFA88F18B420DD920460191FFF774FF07
:1063B000054620B901992046FFF704FF20B908F1EE
:1063C0000108EBE70125D3E7044A394630464FF090
:1063D00009FFCDE7884A09089D4A0908C24A090809
:1063E0002DE9F0412DED048B90F842139FED348A96
:1063F000DFED348A9FED349A82B00646FFF794FDB4
:1064000006F13C07C5B27C2000FB057554354FF002
:10641000000896F822205FFA88F39A424ED919466E
:106420003046FFF7CFFE10B908F10108F1E7194631
:106430003046FFF779FDC4B27C2000FB0474D4ED34
:10644000157AF0EEE77AF4EEC87AF1EE10FA04F17C
:1064500054040ED5D4ED017AF0EEE77AF4EEC87A62
:10646000F1EE10FA05D5002002B0BDEC048BBDE8BA
:10647000F0812946204612F0ABF9B4EEE80AF1EEBD
:1064800010FAF0DC2946204611F0CAFCB4EEC90A25
:10649000F1EE10FAE7DC2146284611F00DFC6846C3
:1064A0008DED000ACDED010A11F0A6FCDFED077AB3
:1064B000B4EEE70AF1EE10FAB6DDD4E70120D3E737
:1064C00000000034DB0FC93F920A863F00004843BA
:1064D000022910B5044608D8FFF726FD7C23C0B278
:1064E00003FB004494F83D0010BD0020FCE70000D1
:1064F00013B590F8421301910446FFF7E9FF30B15C
:106500000199204602B0BDE81040FFF75BBE02B023
:1065100010BD0000F7B590F921500446002D73D04E
:1065200090F84053002D6FD090F84213FFF7D0FF42
:1065300094F83D33064613B92046FFF713FE0025B5
:1065400094F82020EBB29A4207D904EB830301357B
:10655000586903689B689847F2E750F0DFFD002711
:10656000224604F5BA7140F2F315D2F89C30C31AF2
:10657000AB428CBF0023012382F83D307C32914234
:1065800047EA0307F1D194F92430032B07D194F89B
:106590003C33002B3BD0D4F83803002849D167B1F5
:1065A000236B013309D030F01DF9216B2FF040FF30
:1065B00018B130F017F92EF0FFFF94F92C32002BB0
:1065C0003AD194F92D32CBBB94F92E3213B1022378
:1065D00084F8423394F842132046FFF779FF86424D
:1065E000054611D030F0FEF84FF6FF712FF020FF76
:1065F00050B1002D14BF00220422019230F0F2F8B5
:10660000019A03212FF0A6FE284603B0F0BD012316
:1066100084F83C330420FFF7E5FA054610B1214623
:1066200006F05EFE94F92430C4F83853032BB2D040
:10663000B5E706F063FEB2E70023C9E70123C7E729
:1066400038B590F921300446D3B190F84053BDB12C
:10665000FFF76AFCC0B2022812D87C2303FB004477
:10666000D4ED1A7A9FED087AF4EEC77AF1EE10FABB
:1066700006D4B7EE087AF4EEC77AF1EE10FA00DD30
:106680000025284638BD00BFABAA2A3F70B5D0F818
:10669000085315F4003504460E460DD190F84033EA
:1066A0005BB90A78072A07D8012303FA02F290F8A7
:1066B0003F33134380F83F3370BD94F82020EBB292
:1066C0009A42F9D904EB8303314658690368DB68C1
:1066D00098470135F1E7000038B505466C242B5981
:1066E0001BB1002128192AF0D7FF7C34B4F5F07FC4
:1066F000F5D138BD014B1868704700BFEC5A002037
:106700002DE9F04FAA4BD3F800800446D8F80400D6
:1067100003688DB09B689847002507464FF0010934
:1067200009FA05F33B4240F082820135202DF7D172
:10673000D8F804000368DB689847002507464FF047
:10674000010909FA05F33B4240F0B3820135202DDF
:10675000F7D1D8F8040003689B68984700250746DE
:106760004FF0010909FA05F33B4240F0E18201359F
:10677000202DF7D1D8F80400DFF840B203689B68F9
:10678000984700250490049A0123AB40134240F03F
:106790000B830135202DF6D1D8F80400DFF81CB2A8
:1067A0000368DB68984700250490049A0123AB40F6
:1067B000134240F0C9830135202DF6D1D8F80400EA
:1067C0000368DB689847002507464FF0010909FA7E
:1067D00005F33B4240F083840135202DF7D1D8F8F2
:1067E00004000368DB689847002507464FF001095D
:1067F00009FA05F33B4240F0B1840135202DF7D171
:10680000D8F8040003689B689847002507464FF0B6
:10681000010909FA05F33B4240F0DF840135202DE0
:10682000F7D1D8F8040003689B689847002507460D
:106830004FF0010909FA05F33B4240F00E8501359E
:10684000202DF7D1D8F8040003689B6898470025ED
:1068500007464FF0010909FA05F33B4240F03D8538
:106860000135202DF7D1D8F804000368DB6898477C
:10687000002507464FF0010909FA05F33B4240F0B5
:1068800068850135202DF7D14A4B089308AF0425C0
:10689000D8F8040003689B689847002683460123C4
:1068A000B34013EA0B0F40F08F850136202EF6D14E
:1068B000D8F804000368DB68984700268346012364
:1068C000B34013EA0B0F40F0C4850136202EF6D1F9
:1068D000013D15F0FF0507F10107D9D1D8F80400F3
:1068E00003689B6898474FF00109074609FA05F3CA
:1068F0003B4240F0F2850135202DF7D1D8F8040055
:106900000368DB689847002507464FF0010909FA3C
:1069100005F33B4240F01D860135202DF7D1D8F814
:10692000040003689B689847002507464FF001095B
:1069300009FA05F33B4240F048860135202DF7D196
:10694000D8F804000368DB689847002507464FF035
:10695000010909FA05F33B4240F073860135202D09
:10696000F7D1154B0793D8F8040003689B68984744
:10697000002583460123AB4013EA0B0F42D00027CA
:106980005FFA85F9D4F8083313F4803A32D107ABB3
:106990004946DB5D04931A462046FFF7EFFA049B55
:1069A0000646002800F08986CDE908AA08E000BF65
:1069B000EC2500200C0D0E0F20212223801A06004A
:1069C000099B0B93002201210BA8CDE9092204F0B9
:1069D00003FE01462046FFF7C1FA0BA8FDF78AF92E
:1069E0000AA8FDF787F909A8FDF77AF916B108A8F2
:1069F000FDF776F994F82330052B00F04881013734
:106A0000042FBFD10135202DB4D1D8F8040003687C
:106A1000DB689847002583460123AB4013EA0B0F40
:106A200038D000275FFA85F9D4F8083313F4803A98
:106A300028D107AB4946DB5D04931A462046FFF791
:106A40009DFA049B0646002800F04686CDE908AA78
:106A50000022099B0B9311460BA8CDE9092204F0F3
:106A6000BBFD01462046FFF779FA0BA8FDF742F976
:106A70000AA8FDF73FF909A8FDF732F916B108A8F1
:106A8000FDF72EF994F82330052B00F00081013733
:106A9000042FC9D10135202DBED1D8F804000368D8
:106AA0009B689847002682460123B34013EA0A0FE9
:106AB00031D010255FFA86F9D4F8083313F0080BAB
:106AC00020D12A4649462046FFF758FA07460028B3
:106AD00000F01186CDE909BB0A9B002201210BA819
:106AE000CDE90A2301F00AFC01462046FFF736FAF9
:106AF0000BA8FDF7F5F80AA8FDF7F2F817B109A8F9
:106B0000FDF7EEF894F82330052B00F0C080013536
:106B1000EDB2142DD0D10136202EC5D1D8F8040005
:106B200003689B689847002682460123B34013EA16
:106B30000A0F34D014255FFA86F9D4F8083313F419
:106B4000001B24D12A4649462046FFF717FA07467C
:106B5000002800F0E385CDE908BB099B0B930022D8
:106B600001210BA8CDE9092201F0DAFF01462046F8
:106B7000FFF7F4F90BA8FDF7BDF80AA8FDF7BAF87E
:106B800009A8FDF7ADF817B108A8FDF7A9F894F822
:106B90002330052B7BD00135EDB2182DCDD1013638
:106BA000202EC2D1D8F804000368DB68984700267D
:106BB00082460123B34013EA0A0F34D014255FFA4A
:106BC00086F9D4F8083313F4001B24D12A46494629
:106BD0002046FFF7D3F90746002800F0AF85CDE93E
:106BE00008BB0022099B0B9311460BA8CDE9092293
:106BF00001F096FF01462046FFF7B0F90BA8FDF71C
:106C000079F80AA8FDF776F809A8FDF769F817B131
:106C100008A8FDF765F894F82330052B37D0013527
:106C2000EDB2182DCDD10136202EC2D12FE0D4F8EF
:106C3000083313F0010A25D15FFA85FB1E2259465D
:106C40002046FFF79BF9064620B3CDE908AA099A2A
:106C50000B920023082201210BA8CDE9093303F090
:106C600089FA01462046FFF779F90BA8FDF742F8AB
:106C70000AA8FDF73FF809A8FDF732F816B108A8F1
:106C8000FDF72EF894F82330052B7FF44EAD0DB0B0
:106C9000BDE8F08FD8F8041004220B68CDE901029A
:106CA000A84A0092D3F800A05A461E2309A8D0474C
:106CB000CDE7D4F8083313F0010A24D15FFA85FB3D
:106CC0001E2259462046FFF759F9064608B3CDE97A
:106CD00008AA099B0B93062200210BA8CDE90911F4
:106CE00003F048FA01462046FFF738F90BA8FDF7F4
:106CF00001F80AA8FCF7FEFF09A8FCF7F1FF16B19E
:106D000008A8FCF7EDFF94F82330052B7FF41EADA7
:106D1000BDE7D8F8041004220B68CDE90102894AC6
:106D20000092D3F800A05A461E2309A8D047D0E706
:106D3000D4F8083313F4805A21D15FFA85FB0D2271
:106D400059462046FFF71AF90646F0B1CDE909AADF
:106D50000A9B0022CDE90A23012108220BA804F096
:106D600077FA01462046FFF7F9F80BA8FCF7B8FFC1
:106D70000AA8FCF7B5FF16B109A8FCF7B1FF94F813
:106D80002330052B7FF4F3AC81E7D8F804100422FC
:106D90000B68CDE901026B4A0092D3F800A05A4675
:106DA0000D230AA8D047D3E7D4F8083313F480772B
:106DB0003FD15FFA85F90C2249462046FFF7DEF8FD
:106DC0000646002800F08480CDE90677079B0A93E9
:106DD0004FF0000A692249462046CDF81CA0FFF773
:106DE000CDF80746002800F08180CDE908AA099B6C
:106DF0000B9300221A2309920BA901220AA801F081
:106E000005F801462046FFF7A9F80BA8FCF768FF34
:106E100009A8FCF765FF17B108A8FCF761FF0AA8ED
:106E2000FCF75EFF07A8FCF75BFF16B106A8FCF7AE
:106E300057FF94F82330052B3FF429AFD4F80833DB
:106E400013F480777FF4A5AC5FFA85F90C224946EC
:106E50002046FFF793F80646002856D0CDE906777E
:106E6000079B0A934FF0000A682249462046CDF856
:106E70001CA0FFF783F80746002854D0CDE908AAE4
:106E8000099B0B9300221A2309920BA901220AA83D
:106E900000F0BCFF01462046FFF760F80BA8FCF7A6
:106EA0001FFF09A8FCF71CFF17B108A8FCF718FF83
:106EB0000AA8FCF715FF07A8FCF712FF16B106A8F1
:106EC000FCF70EFF94F82330052B7FF462ACDEE66E
:106ED000D8F8041004220B68CDF800B0CDE9010207
:106EE0004A461F6807A80C23B8476FE7D8F8041074
:106EF00004220B68CDF800B0CDE901024A46D3F870
:106F000000A009A86923D04771E7D8F8041004222B
:106F10000B68CDF800B0CDE901024A461F6807A80A
:106F20000C23B8479CE7D8F8041004220B68CDF86E
:106F300000B0CDE901024A46D3F800A009A86823B1
:106F4000D0479DE7801A0600D4F8083313F4807701
:106F50003DD15FFA85F90C2249462046FFF70EF82D
:106F60000646002800F08180CDE90677079B0A934A
:106F70004FF0000A692249462046CDF81CA0FEF7D2
:106F8000FDFF074600287ED0CDE908AA099B0B9398
:106F900000221A230BA90AA8099200F037FF014624
:106FA0002046FEF7DBFF0BA8FCF79AFE09A8FCF7CA
:106FB00097FE17B108A8FCF793FE0AA8FCF790FE0D
:106FC00007A8FCF78DFE16B106A8FCF789FE94F819
:106FD0002330052B3FF45BAED4F8083313F48077ED
:106FE0007FF4E9AB5FFA85F90C2249462046FEF7AB
:106FF000C5FF0646002855D0CDE90677079B0A93C2
:107000004FF0000A682249462046CDF81CA0FEF742
:10701000B5FF0746002853D0CDE908AA099B0B937A
:1070200000221A230BA90AA8099200F0EFFE0146DC
:107030002046FEF793FF0BA8FCF752FE09A8FCF7C9
:107040004FFE17B108A8FCF74BFE0AA8FCF748FE54
:1070500007A8FCF745FE16B106A8FCF741FE94F818
:107060002330052B7FF4A7AB11E6D8F804100422D7
:107070000B68CDF800B0CDE901024A461F6807A8A9
:107080000C23B84772E7D8F8041004220B68CDF837
:1070900000B0CDE901024A46D3F800A009A869234F
:1070A000D04773E7D8F8041004220B68CDF800B07D
:1070B000CDE901024A461F6807A80C23B8479DE79F
:1070C000D8F8041004220B68CDF800B0CDE9010215
:1070D0004A46D3F800A009A86823D0479EE7D4F811
:1070E000083313F0200A24D15FFA85FB1C2259468D
:1070F0002046FEF743FF064608B3CDE908AA002262
:10710000099B0B9311460BA8CDE9092203F030FC33
:1071100001462046FEF722FF0BA8FCF7EBFD0AA86C
:10712000FCF7E8FD09A8FCF7DBFD16B108A8FCF7A1
:10713000D7FD94F82330052B7FF44EABA7E5D8F8A4
:10714000041004220B68CDE90102B84A0092D3F87A
:1071500000A05A461C2309A8D047D0E7D4F808332A
:1071600013F0200A24D15FFA85FB1E2259462046DF
:10717000FEF704FF064608B3CDE908AA0022099BE2
:107180000B9311460BA8CDE9092203F0F1FB014650
:107190002046FEF7E3FE0BA8FCF7ACFD0AA8FCF7BF
:1071A000A9FD09A8FCF79CFD16B108A8FCF798FDFD
:1071B00094F82330052B7FF420AB68E5D8F8041051
:1071C00004220B68CDE90102984A0092D3F800A08E
:1071D0005A461E2309A8D047D0E7D4F8083313F045
:1071E000200A25D15FFA85FB1C2259462046FEF76E
:1071F000C5FE064610B3CDE908AA099A0B920023F2
:10720000022201210BA8CDE9093303F0B1FB0146AD
:107210002046FEF7A3FE0BA8FCF76CFD0AA8FCF7BE
:1072200069FD09A8FCF75CFD16B108A8FCF758FD3C
:1072300094F82330052B7FF4F1AA28E5D8F8041040
:1072400004220B68CDE90102784A0092D3F800A02D
:107250005A461C2309A8D047CFE7D4F8083313F0C7
:10726000200A25D15FFA85FB1E2259462046FEF7EB
:1072700085FE064610B3CDE908AA099A0B920023B1
:10728000022201210BA8CDE9093303F071FB01466D
:107290002046FEF763FE0BA8FCF72CFD0AA8FCF7BE
:1072A00029FD09A8FCF71CFD16B108A8FCF718FD7C
:1072B00094F82330052B7FF4C2AAE8E4D8F8041030
:1072C00004220B68CDE90102584A0092D3F800A0CD
:1072D0005A461E2309A8D047CFE7D4F8083313F045
:1072E000400A21D15FFA85FB0C2259462046FEF761
:1072F00045FE0646F0B1CDE909AA0A9B0022CDE978
:107300000A23012106220BA800F046FD0146204673
:10731000FEF724FE0BA8FCF7E3FC0AA8FCF7E0FC50
:1073200016B109A8FCF7DCFC94F82330052B7FF498
:1073300097AAACE4D8F8041004220B68CDE9010246
:107340003A4A0092D3F800A05A460C230AA8D04724
:10735000D3E7D4F8083313F0400A20D15FFA85FB55
:107360000C2259462046FEF709FE0646E8B1CDE953
:1073700009AA00220A9B11460BA8CDE90A2300F0B6
:107380000BFD01462046FEF7E9FD0BA8FCF7A8FC23
:107390000AA8FCF7A5FC16B109A8FCF7A1FC94F813
:1073A0002330052B7FF46DAA71E4D8F80410042271
:1073B0000B68CDE901021D4A0092D3F800A05A469D
:1073C0000C230AA8D047D4E7D4F8083313F0800A76
:1073D00026D13B78F1B21A462046CDE90413FEF7D8
:1073E000CDFDDDE90413814610B3CDE909AA0A9B5E
:1073F0000022CDE90A2301210C220BA803F086F913
:1074000001462046FEF7AAFD0BA8FCF769FC0AA876
:10741000FCF766FCB9F1000F02D009A8FCF760FC8C
:1074200094F82330052B7FF440AA30E4801A06003C
:10743000D8F80400B84AD0F800E000924FF0040CED
:10744000CDE9019C0A46DEF800A001460AA8D04713
:10745000CDE7D4F8083313F0800A26D13B78F1B297
:107460001A462046CDE90413FEF788FDDDE9041332
:10747000814608B3CDE909AA0A9B0022CDE90A2377
:1074800000210C220BA803F041F901462046FEF72B
:1074900065FD0BA8FCF724FC0AA8FCF721FCB9F158
:1074A000000F02D009A8FCF71BFC94F82330052B31
:1074B0007FF40BAAFFF7EBBBD8F80400964AD0F88C
:1074C00000E000924FF0040CCDE9019C0A46DEF882
:1074D00000A001460AA8D047CEE7D4F8083313F439
:1074E000004A20D15FFA85FB0C2259462046FEF760
:1074F00045FD0646F0B1CDE909AA0A9B002201210B
:107500000BA8CDE90A2302F077FF01462046FEF7DB
:1075100025FD0BA8FCF7E4FB0AA8FCF7E1FB16B17C
:1075200009A8FCF7DDFB94F82330052B7FF4E3A9D1
:10753000FFF7ADBBD8F8041004220B68CDE90102B7
:10754000754A0092D3F800A05A460C230AA8D047E7
:10755000D3E7D4F8083313F4004A20D15FFA85FB4F
:107560000C2259462046FEF709FD0646F0B1CDE94A
:1075700009AA00220A9B11460BA8CDE90A2302F0B2
:107580003BFF01462046FEF7E9FC0BA8FCF7A8FBF1
:107590000AA8FCF7A5FB16B109A8FCF7A1FB94F813
:1075A0002330052B7FF4B8A9FFF771BBD8F804107E
:1075B00004220B68CDE90102574A0092D3F800A0DB
:1075C0005A460C230AA8D047D3E7D4F8083313F45B
:1075D000007A20D15FFA85FB302259462046FEF71B
:1075E000CDFC0646F0B1CDE909AA0A9B0022012193
:1075F0000BA8CDE90A2303F087FC01462046FEF7DD
:10760000ADFC0BA8FCF76CFB0AA8FCF769FB16B1F4
:1076100009A8FCF765FB94F82330052B7FF48DA9AE
:10762000FFF735BBD8F8041004220B68CDE901023E
:10763000394A0092D3F800A05A4630230AA8D0470E
:10764000D3E7D4F8083313F4007A20D15FFA85FB2E
:10765000302259462046FEF791FC0646F0B1CDE9AE
:1076600009AA00220A9B11460BA8CDE90A2303F0C0
:107670004BFC01462046FEF771FC0BA8FCF730FBE3
:107680000AA8FCF72DFB16B109A8FCF729FB94F812
:107690002330052B7FF462A9FFF7F9BAD8F804105C
:1076A00004220B68CDE901021B4A0092D3F800A026
:1076B0005A4630230AA8D047D3E7D8F8041004204C
:1076C0000A68CDE9016014480090D2F800A009A82A
:1076D0004A46D047FFF774B9D8F8041004200A6866
:1076E000CDE901600C480090D2F800A009A84A46F4
:1076F000D047FFF7ADB9D8F8041004220B68CDE9E4
:107700000102054A0092D3F800B04A462B460AA867
:10771000D847FFF7E1B900BF801A0600D8F8041077
:1077200004220B68CDE901020C4A0092D3F800B0A4
:107730004A462B4609A8D847FFF70FBAD8F80410D5
:1077400004220B68CDE90102044A0092D3F800B08C
:107750004A462B4609A8D847FFF743BA801A0600C5
:1077600073B50446FEF7CCFF94F82330052B32D0D6
:10777000002594F83F33EB40DA07E9B216D401351F
:10778000082DF6D194F82330052B24D094F820301E
:1077900013B194F82230F3B9104B11491B68986962
:1077A00003681B6802B0BDE870401847D4F808337E
:1077B0009B030CD42C200191FEF714FA064610B15D
:1077C000019903F019FC31462046FEF7C7FB94F8F7
:1077D0002330052BD3D102B070BD00BFEC250020B3
:1077E000DC4A09082DE9F04F90F9213089B00446B0
:1077F000002B00F00481012300F50C7580F8413363
:10780000024600F50F712B462E46D06E002859D047
:10781000002384F8413394F94030642B5BD094F911
:10782000BC30642B00F08D8094F93831642B00F06B
:107830008A80D4F830722FBB01A9204629F010FFAE
:1078400000B30C230593012306978DF81830714B74
:1078500007936946BDF80430049704A8ADF81030CA
:107860008DF800702AF0CEF89DF9001051B1022970
:1078700008DC38B1C9B27C2303FB01416C312846D6
:107880002BF0CCFA94F841B3BBF1000F5DD0E36E5E
:107890006367D4F8E830C4F8F030D4F86431C4F841
:1078A0006C3194F8233003F1C30204EB820200210F
:1078B000042B7CD852F8040B1061013342F8041CED
:1078C000DBB2F5E753F8040B0028A1D18B4202F19B
:1078D0007C029AD19FE7002066238DF810307C232C
:1078E00003FB004004A940302BF0DCF904A920463A
:1078F00029F0B6FE00289CD004238DF81830002310
:10790000CDE90133039331230593694604A82AF096
:1079100079F8059B28B108AA02EB8302009942F886
:10792000E01C0133332B0593EFD94CF0D7FF9DEDCD
:10793000031ADDED020A9DED010A66214CF08CFF71
:1079400077E70120C8E70220C6E70127A94655F8D6
:10795000043B23B1AB600137042FF7D197E7AA4668
:10796000B8465FFA88F3022BF5D8DAF8002055F80C
:10797000043C9A4205D104A95046CDF810B02BF032
:107980004DFA5AF8043B08F101020BB99046E8E7BA
:1079900004A906EB88000193CDF810B02BF03EFA55
:1079A000019BAB6001A948462BF038FAD3E794F865
:1079B000413313B92046FEF7DDF994F822300BB3BA
:1079C000154B1B68986A036864215B6898472046DA
:1079D000FEF7A0FD94F83E3003B9E36694F8BA30A0
:1079E0000BB9C4F8E83094F836310BB9C4F86431F7
:1079F000F9F79EFDF9F726FE0123A4F8403309B0FC
:107A0000BDE8F08F2046FFF7ABFE94F82230002B44
:107A1000E0D0D5E774E30908EC25002070470000AA
:107A20000120704701207047436898687047000044
:107A300010B5054B03600446806A10B103685B68AB
:107A40009847204610BD00BFA04F09084068036852
:107A50005B6A184733B46C46406884E80C000368DE
:107A60009D6A94E80C00AC4602B030BC6047000050
:107A700010B50446FFF7DCFF2046FEF7BBF82046B2
:107A800010BD000040680AF0A5BC0000406801235A
:107A90000AF0A0BC40680AF079BC000040680A22E5
:107AA0000AF01EBC40680AF033BC000040680AF0CF
:107AB000B5BC000090F82E2022B190F82D100022C5
:107AC00001F06EB97047000073B504460525002625
:107AD000A06A8DF8076003680DF10702DB680121D9
:107AE000984778B19DF807300C2B09D0102B05D0A2
:107AF000092B07D184F8303002B070BD1523F9E7A7
:107B00001423F7E7013DE3D12846F5E710B4806A76
:107B100003681C690822A44601235DF8044B312147
:107B20006047000010B4806A03681C690122A44603
:107B300000235DF8044B322160470000F0B5044695
:107B4000806A036885B05B6998470546002800F0A5
:107B50008480A06A03685B69984703689B689847BC
:107B6000A06A03689B69984760B93D4B3D491B6813
:107B7000986903681B6898472B682846DB68984714
:107B8000002667E02046FFF7CDFF0028F4D020460E
:107B9000FFF79AFF0028EFD0A06A03680121DB6A93
:107BA00098472046FFF7B2FF30B92D4B2E491B688E
:107BB000986903681B68DEE7A06A0368DB69984779
:107BC00030B9274B29491B68986903681B68D2E7BD
:107BD000A06A94F83010012784F82E7003685B6A5D
:107BE0009847A06A03689B6A984704F12D020146F2
:107BF000204601F023F906460028BDD0A06A94F87B
:107C00002D10036801919B6A98470199024620460E
:107C100001F018F994F82C302BB194F82D103A4655
:107C2000204601F023F994F82F2094F82D102046D7
:107C300001F03EF92B682846DB689847A06A029459
:107C400003681D6A0A4B039304AB13E90C0042F26C
:107C50001071A847304605B0F0BD0646FAE700BFF0
:107C6000EC2500200C4F0908324F0908514F090834
:107C7000697D010870B5002586B0CDE90055002367
:107C80000446806A8DF808500593039304930368B3
:107C90006A469E6810210923B047A0B19DF80030C4
:107CA00013F0010615D194F831300133DBB2052B06
:107CB00084F8313007D12046FFF734FF2046FFF724
:107CC00025FF84F83160A06A03681B6B984706B0F3
:107CD00070BD9DF8083084F831501B07F3D4BDF90E
:107CE00001309FED1F6A06EE903ABDF9033007EEB2
:107CF000103ABDF90530F8EEE66A07EE903ACDEDA0
:107D0000036AF0EEE66AB8EEC77AF8EEE77AF4EEC8
:107D1000C66AF1EE10FA8DED047ACDED057A0DD537
:107D2000B0EEC77AB4EEC67AF1EE10FA06D5F0EEF0
:107D3000E77AF4EEC67AF1EE10FAC4D49FED090AA0
:107D400003A810F083F9B2EE040A03A810F07EF93C
:107D500094F82D200A2303A9204601F00FF9B2E779
:107D6000000000349A99193EFFF784BF10B5044B08
:107D7000044640F8043BFBF7B3FF204610BD00BFAC
:107D8000B84F090810B50446FFF7F0FF2046FDF78D
:107D900031FF204610BD0000F7B503680F461646B8
:107DA0001BB90024204603B0F0BD00240460082065
:107DB0000193FDF717FF054620B1124B0360019BAD
:107DC0004360019401A8FBF78BFF002DE9D034201C
:107DD000FDF708FF04460028E3D000F0E1FE0A4B5F
:107DE000A562236084F82C7084F82F602046FFF78A
:107DF000A5FE05460028D5D1236820465B68984734
:107E00002C46CFE7B84F0908A04F09082DE9F74FD6
:107E1000046806460D4690469946002C6CD00B68C7
:107E2000002B49D0236820465B6A984703689B680B
:107E30009847012328680DEB030200210AF0CAFAD3
:107E400098B39DF80130EA2B2FD1DFF8F0B04FF056
:107E5000060A28680023802206210AF097FA20B338
:107E6000DBF80070B86A03680A215B689847002352
:107E700028681A4606210AF089FAB0B1B86A036880
:107E80000A215B689847012328680DEB030206214D
:107E90000AF0A0FA48B19DF8014014F040042FD038
:107EA0000AF1FF3A1AF0FF0AD3D1306803685B6A1F
:107EB00098470368DB68984700241DE002222346A8
:107EC0000F2128680AF062FAB86A036801215B682A
:107ED0009847306803685B6A98470368DB6898478F
:107EE000336834604A46414601A80193FFF754FFC6
:107EF000044601A8FBF7F4FE204603B0BDE8F08F6E
:107F0000224623460F2128680AF040FAB86A03681F
:107F100001215B6898470223214630680DEB03027C
:107F20000AF058FA04460028C8D0B8690249036824
:107F30001B689847B9E700BF784F0908EC25002077
:107F400090F82C10002200F02BBF000070B5044602
:107F50008CB00426013E76B2731C4AD0A06A152369
:107F60006A465D210AF036FA0028F3D0A06A15238C
:107F700006AA5D210AF02EFA05460028EAD015224D
:107F800006A9684673F01EFE0028E3D19DF8003074
:107F900084F82E309DF8073084F830309DF8143086
:107FA00084F83A309DF813309DF8102084F83B3067
:107FB0009DF80F3043EA0223A3879DF8013084F82F
:107FC0002F309DF8083084F83130039B9DF80C2049
:107FD000C3F30F2363869DF80B3043EA0223A38685
:107FE000049BC3F30F23E386019BC3F30F23238773
:107FF00007E0054B05491B68986903681B689847AB
:10800000002528460CB070BDEC250020EC4F090877
:108010002DE9FF4104460023806A8DF8073003688C
:10802000DFF868815B6A984703689B689847A06A95
:1080300003680A219B6C9847A06A0A2204210AF06F
:108040004FF90425013D6DB26B1C32D000234B214A
:10805000A06A82220AF09AF9D8F800600746B06A4E
:10806000036802215B689847002FEBD001231A4672
:108070004B21A06A0AF08AF90746B06A0368022118
:108080005B689847002FDDD0A06A01230DF107023D
:1080900040210AF09FF90028D4D09DF80720322A09
:1080A00010D0002DCED1B069364903681D68322347
:1080B000A847A06A03685B6A98470368DB6898472B
:1080C00000255BE02046FFF741FF0028F1D0A06AC1
:1080D0000123172251210AF059F90028E9D0522230
:1080E000A06A012311460AF051F90028E1D0A06AE4
:1080F000012338224C210AF049F90028D9D0A06A7E
:1081000003685B6A98470368DB689847A06A0521A3
:108110000AF0FEF8A36A04F12C029968204600F0E8
:108120008DFE054650B3A36A94F82C109A68204639
:1081300000F088FE94F8442094F82C10204600F0BB
:10814000B7FE94F845302BB194F82C10012220464C
:1081500000F08CFEA06A036802219B6C9847A06A1D
:10816000029403689E6A084B039304AB13E90C0066
:1081700044F21B11B0474EF0D1FF2064284604B0F2
:10818000BDE8F08114500908F9820108EC250020AF
:1081900070B5858F90F93B60AD03B5FBF2F2A2F5A7
:1081A000804404FB04F2D51190F83A200498D201DF
:1081B000624306FB05225212A03002F580124243B0
:1081C00012134A43DB0003EB623000B270BD0000C3
:1081D00010B5448E53005C43B0F93830C91A838F10
:1081E000D31AB0F93620B0F93400534304F50044F3
:1081F0009B10C3EBC13300EB2440044993FBF0F028
:108200004FF400420DF0EEFE00B210BD0080FFFF03
:1082100010B52DED028B8AB004460823806A05AAAA
:1082200042210AF0D7F818B1BDF81A20D30719D4A3
:10823000A06A0AF0F3F84EF071FF236CC31AFA2B10
:108240000CD92064002382224B21A06A0AF09EF8F8
:108250000123A06A1A464B210AF098F80AB0BDEC37
:10826000028B10BDBDF9141094F9303000939208C0
:1082700094F92E300392C9102046FFF789FFBDF90B
:10828000161094F93130039A009308EE900A94F98D
:108290002F30C9102046FFF77BFFBDF91810039A55
:1082A000491008EE100A2046FFF792FF07EE900AE9
:1082B000F8EEE88AF8EEE77AB8EEC88AB3EE000A7C
:1082C00007A8CDED097ACDED078A8DED088A0FF06C
:1082D000D1FEB2EE040A07A80FF0B8FE4EF01EFF62
:1082E00094F82C2020640A23204607A900F046FEBB
:1082F000A06A0AF093F8B1E7FFF78ABFF7B5036801
:108300000D4616461BB90024204603B0F0BD0027D9
:1083100007604820CDE90073FDF764FC044650B1C6
:1083200000F03EFC0E4B2360019BA362019784F892
:10833000446084F8455001A8FBF7DCFC6846FBF775
:10834000D9FC002CDFD02046FFF762FE054600284E
:10835000DAD1236820465B6898472C46D4E700BFF3
:108360004C50090810B5044B044640F8283BFBF775
:10837000C1FC204610BD00BF4C50090810B5044692
:10838000FFF7F0FF2046FDF735FC204610BD00004A
:1083900090F82C10002200F003BD0000F8B5044650
:1083A0000D4617461E4600F0FBFB094B23602B6869
:1083B000A362002200232A6084F82D7084F82E60C6
:1083C00023656365A365E365236663662046F8BDA0
:1083D00064500908F8B51C4609331646DB086A469E
:1083E000A2EBC30300AF9D46806AA31C6A4609F056
:1083F000F1FF054628B122460DF10201304673F027
:10840000F1FB2846BD46F8BD2DE9F34106460F466F
:1084100014464EF083FE114BD3F800800546D8F881
:108420002800036801215B68984701230DF10702CA
:1084300007213046FFF7CEFF60B19DF80730DA071D
:1084400002D4B7EB531F05D04EF068FE431BA34286
:10845000E5D3002002B0BDE8F08100BFEC2500208C
:108460002DE9F041DFF8608292B0044602AF0026A9
:1084700046F02002A06A0023D2B2502109F086FF04
:10848000002800F00C810325013D6DB26A1C00F04C
:108490000681D8F80030986A03684FF496719B689B
:1084A000984701230DF1060255212046FFF792FF60
:1084B000002800F0F4809DF8063013F0E00F40F043
:1084C000EE80DB07E0D502230DF1060252212046A3
:1084D000FFF780FF002800F0E280BDF8063001368B
:1084E0005BBA202E27F8023BC2D1BDF824309DF89C
:1084F00026109FED6D7ADFED6D6A9FED6D6A43F397
:108500000B0207EE902A1B0903F47063BDF82620C6
:10851000F8EEE77A0B4343F30B03C4ED0C7A07EE56
:10852000903A02F470639DF82820F8EEE77A13433E
:1085300043F30B03C4ED0D7A07EE903A9DF9223018
:10854000F8EEE77AC4ED0E7A07EE903A9DF92930FD
:10855000F8EEE77A67EE877A07EE103AB8EEC77A58
:108560009DF92A30C4ED0F7A27EE267ADFED517A95
:1085700084ED107A07EE103AB8EEC77A9DF92B30E9
:10858000E7EE267AC4ED117A07EE903AF8EEE77A34
:108590009DF9233067EEA67ADFED476AC4ED127AC3
:1085A00007EE903A9DF92C3007EE103AB8EEC77AF4
:1085B0009DF92E3027EE267AF8EEE77A84ED147ACC
:1085C00067EE867A07EE103A9DF93030C4ED137AE3
:1085D00007EE903AF8EEE77A9DF92D3067EEA67A2D
:1085E000B8EEC77AC4ED167A27EE267A07EE903AEF
:1085F00084ED157AF8EEE77A9FED307A9DF92F3009
:1086000067EE877AC4ED177A07EE903A9DF931301C
:10861000F8EEE77A06EE903A67EE877AF8EEE66AC9
:10862000C4ED187ADFED267ABDF93830E6EE877AA8
:1086300007EE103A9DF93230C4ED197AB8EEC77AD8
:10864000F3EE077AE7EE067A07EE103ADFED1D6AE1
:10865000C4ED1A7AB8EEC77A27EE267A84ED1B7A33
:108660009DF9333007EE103AB8EEC77A9DF93430F1
:1086700027EE267A84ED1C7A07EE103A9DF9353004
:1086800007EE903AB8EEC77AF8EEE77A27EE267A48
:1086900067EEA67A84ED1D7AC4ED1E7A00E0002014
:1086A00012B0BDE8F08100BFCDCC4C3E0000803B55
:1086B0000000003B0AD7233C0000003D000080384A
:1086C00017B7D1B80AD7A33AEC25002073B5012318
:1086D0000E460DF1070206210446FFF77BFE18B98E
:1086E0000025284602B070BD9DF80730013B012BE4
:1086F0000CD80023A06A1A46062109F047FE00287C
:10870000EED0062200212046FFF77EFEA06A00235D
:108710003246062109F03AFE05460028E0D026221E
:1087200031462046FFF770FEDBE7000013B501235A
:108730000DF1070207210446FFF74CFE10B9002097
:1087400002B010BD9DF807301B070CD50023A06AAE
:108750001A46062109F01AFE0028F0D00622002150
:108760002046FFF751FEA06A00230722062109F0E8
:108770000DFE0028E3D0132207212046FFF744FE18
:108780000028DCD0A06A00230522062109F0FEFDA6
:108790000028D4D0172205212046FFF735FE0028F7
:1087A000CDD001212046FFF791FFC9E7F7B5044678
:1087B000806A5B4F03685B6A984703689B689847C9
:1087C000A06A03680A219B6C9847A06A0A220421C8
:1087D00009F086FD0525013D6DB26B1C00F0968009
:1087E000A06A0023B6227E2109F0D0FD0028F2D035
:1087F0003B68986A036818215B686E4698470123B6
:10880000324600212046FFF7E5FD0028E3D09DF821
:108810000030332BDFD12046FFF722FE002875D031
:10882000A06A00238022502109F0B0FD00286DD0FD
:108830002046FFF77BFF002868D0A06A002386222D
:108840002E2109F0A3FD002860D0A06A0023242275
:10885000042109F09BFD002858D0A06A00230222C1
:10886000062109F093FD002850D014220221204651
:10887000FFF7CAFDA06A00230722052109F086FD43
:10888000002843D001212046FFF720FF00283DD0DB
:10889000A06A036803219B6C9847A06A03685B6A1F
:1088A00098470368DB689847A06A172109F030FDF4
:1088B000A36A04F12C029968204600F0BFFA05462D
:1088C00008B3A36A94F82C109A68204600F0BAFA0C
:1088D00094F82E2094F82C10204600F0E9FA94F831
:1088E0002D302BB194F82C100122204600F0BEFA56
:1088F000A06A03689F6A0B4B0094019396E80C00F2
:1089000042F21071B847284603B0F0BDA06A036870
:108910005B6A98470368DB6898470025F3E700BF68
:10892000EC2500201D8B010810B586B00C236A468B
:1089300031210446FFF74EFD002800F0DF809DF84E
:1089400001309DF80020DFED717ADFED715A1B04D4
:1089500003EB02239DF8022003EB02631B1206EED9
:10896000903A9DF804309DF803201B0403EB02238A
:108970009DF8052003EB02631B1207EE103A9DF8E9
:1089800007309DF806201B0403EB02239DF8082006
:1089900003EB02631B1206EE103A9DF80A309DF8B5
:1089A00009201B0403EB0223F8EEE66AB8EEC77A4F
:1089B0009DF80B2066EEA76A27EE277AB8EEC66A06
:1089C000DFED547A03EB02631B1226EE276A07EEF3
:1089D000903AF8EEE77A67EEA57AF5EEC07AF1EE16
:1089E00010FA40F38D80DFED4C5A77EEE57AD4ED46
:1089F000134A94ED0F5A94ED1C4AD4ED1D3A94F8A5
:108A00002C20F7EE005A74EEA54AF0EE632AA4EE8D
:108A1000A75A0A2303A9D4ED107AD4ED0C4A77EEB5
:108A2000A57A2046E7EEA64AD4ED1A7A75EE677A63
:108A300094ED145AF0EE646AD4ED174AE5EE276A15
:108A4000B0EE655AA7EEA45AC6EE854A94ED115AC7
:108A5000D4ED0D6A35EE255AE5EE076A94ED157AE8
:108A6000E7EE876A94ED187AB0EE655AA7EE875A5A
:108A700086EE857A94ED125AD4ED0E6A35EE255ABB
:108A8000E5EE066A94ED166A94ED195AE7EE866AE9
:108A9000B0EE656AA7EE856AF0EE657A86EE863AF4
:108AA00094ED1B6AF0EE646AE6EE447AE6EE476AFD
:108AB00086EEA75AF0EE476AE4EE646AC6EEA75A5D
:108AC000D4ED1E6AD4EE262AE6EE636AB2EE046A9C
:108AD00027EE667A65EE066AA2EEA47ACDED036A09
:108AE00065EE866ACDED046AC7EE276A76EE837A74
:108AF00067EE867ACDED057A00F040FA06B010BD3B
:108B000044BFDFED055A77EEA57A70E747ABE73B48
:108B10005B9E803AF61BEB3B85EBCB41FFF704BF36
:108B200030B51346026885B00D461AB900242046B8
:108B300005B030BD002101607C2001930392FDF758
:108B400051F8044620B1019B2A4603A9FFF726FCF1
:108B500003A8FBF7CFF8002CE8D02046FFF726FE4D
:108B600005460028E3D1236820465B6898472C46D9
:108B7000DDE7000010B5044B044640F8283BFBF746
:108B8000B9F8204610BD00BF6450090810B504466E
:108B9000FFF7F0FF2046FDF72DF8204610BD00003E
:108BA000064B10B503600446FDF7A4FD606004F1B8
:108BB00008004DF07DF9204610BD00BF7C5009082B
:108BC00073B50646144675687C2303FB0253C4EB59
:108BD000441405EB8404084693F8A41001900FF0A8
:108BE000CBFA94F93C3001983BB9736893F825109F
:108BF00002B0BDE870400FF0BFBA94F84010F7E73C
:108C000037B5446801917C2505FB024595F83F3056
:108C100004EB8304D4F84C325BB14EF07FFAC5F814
:108C20009C000199D4F84C0203B0BDE8304003F039
:108C300079BE03B030BD00002DE9F04FC2EB421405
:108C400047684FEA840881460E4607F13C0B08F15D
:108C500008018BB01546594430460FF0C3F9D9F8D6
:108C6000040029460BEB8404FDF7EAFC38B17C23B1
:108C700003FB057393ED1A0A30460FF0E7F97C23E6
:108C800003FB057393ED146ADFED3A7AD3ED156AB1
:108C9000B0EEC67AB4EEE77AF1EE10FA0FD5B0EE88
:108CA000E67AB4EEE77AF1EE10FA08D594ED077A99
:108CB000B0EEC77AB4EEE77AF1EE10FA1BD47C235B
:108CC00003FB0573D86D196E5A6E9B6D029003916C
:108CD0000490079101A831468DED016ACDED056A3A
:108CE0000692089209930DF02FFB86ED000AC6ED5F
:108CF000010A86ED021A7C2303FB05770023C7F8DF
:108D00008C30C7F88830C7F88430D9F8040090F95F
:108D10005C3208F13C0A08F14808DA44D84463B1EF
:108D20005DB9414600F5167004F0B4FA414630468C
:108D30000BB0BDE8F04F0FF055B990F93430012B6E
:108D40000BD190ED0E0A50460FF02CF984ED120A6B
:108D5000C4ED130A84ED141AE8E7022BE6D1FBF701
:108D600009FD002201A9FBF705FA0028DED09DEDE0
:108D7000010AE8E70000003410B543687C2404FBD6
:108D8000023407C904F1900383E807004EF0C6F9E6
:108D9000C4F89C004EF0B6F9C4F8A00010BD000065
:108DA000F0B5074685B00D46164600F10801A92228
:108DB00003A809F069FD7C687C2303FB0543D3F815
:108DC000B42022B903A809F081FD05B0F0BDBEB101
:108DD00096ED007AD3ED2A7A67EE877AC3ED2A7A88
:108DE00096ED017AD3ED2B7A67EE877AC3ED2B7A75
:108DF00096ED027AD3ED2C7A67EE877AC3ED2C7A62
:108E00007C2607EE902A06FB0541A831B8EE670ADA
:108E1000084601910FF02EF901992A463846FFF7CE
:108E2000ABFF06FB05410023C1F8B030C1F8AC3000
:108E3000C1F8A8300023C1F8B430C3E74068FCF79C
:108E4000E9BF0000F7B50646406801927C2707FBA2
:108E500001000D466C3001A9144629F0BFFF71686E
:108E600007FB05152C6703B0F0BD000007B540688F
:108E70007C2303FB010393F93C30022B0BD000F160
:108E80003C03C1EB411003EB80000DF107018DF8AD
:108E9000072029F0FDFE03B05DF804FB43687C2247
:108EA00002FB013191F93C00003818BF01207047E6
:108EB00043687C2000FB013181F8A420704700004A
:108EC000F8B5054608460F460FF032F910B10024F8
:108ED0002046F8BD38460FF011F904460028F6D1B7
:108EE0006B6893F934637EB138460FF059FC95ED09
:108EF000087ADFED1F7AF0EEC76AF4EEE76AF1EE6A
:108F000010FA03D585ED080A0124E1E777EE407AEF
:108F100030EE076AF0EEE77AC7EE866AF6B207EE41
:108F2000906A9FED146AF8EE677A26EE866AF4EE90
:108F3000C67AF1EE10FA48BFB2EE046ADFED0E7A9F
:108F400045BF6B6A66EE866AB0EE676A87EEA66A10
:108F500046BF01336B620124F7EE007A77EEC67AE2
:108F600020EE060AA7EE270A85ED080AB0E700BF43
:108F70000000003400004843CDCCCC3D2DE9F74340
:108F800004460E4615461F46FFF71AFE2A4631468E
:108F90002046FFF735FE314620462A46FFF74CFEB5
:108FA00031462046FFF78CFF28B39B2204F10801CD
:108FB00001A809F069FC64684FF07C0909FB0548C9
:108FC00008F1A808314640460FF00CF809FB0542AD
:108FD000D2F8B4100131C2F8B4104FB1B94207D37E
:108FE0004908C2F8B410B0EE000A40460FF042F84B
:108FF00001A809F06BFC03B0BDE8F08310B504468E
:10900000FCF792FFC0B23C34C0EB401004EB800090
:1090100010BD0000F8B50A4E044600F5167704F5B9
:10902000137555F8040B08B103F0B0FFBD42F8D139
:109030003368986A036801215B689847EFE700BFCF
:10904000EC25002008B5FFF7E5FF0000F0B5144E51
:1090500000EB810773780446D7F84C026FF34103A5
:1090600087B00D467370C8B102F07EFB68B17378AB
:1090700043F0100373702C440023A372D7F84C0202
:1090800007B0BDE8F04002F0F3BAD7F84C126846DA
:1090900002F09AFB009B012BEDD1E8E707B0F0BD91
:1090A0004C5B002070B506460D46002445FA04F3DB
:1090B000DB07E1B202D53046FFF7C8FF0134032CCD
:1090C000F4D170BDFF21FFF7EDBF000030B500F512
:1090D000137587B000F5167455F8041B21B9A54225
:1090E000FAD1002007B030BD684602F06DFB009B4E
:1090F000013B022BF3D80120F4E700002DE9F047F3
:109100002DED028B88B004460D469046B0EE408AA5
:10911000FDF7DEF930B90026304608B0BDEC028B11
:10912000BDE8F08729462046FDF74CF806460028A2
:10913000F1D004EB8507D7F83C22D7F830329A42B9
:1091400006D037F0C7F85C4A032130F0D3FAE2E7E3
:10915000D7F84C3283B94FF49870FCF743FD814641
:1091600008B103F017F8C7F84C92B9F1000F03D11A
:1091700037F0B0F8514AE7E7B4F84A32D90711D5C9
:1091800005F078FE90F8082390F8C43232B9B02286
:1091900002FB030090F8A130012B03D837F09AF8B6
:1091A000474AD1E72046FFF791FF20B9454A537857
:1091B00043F00203537094F9353053B329462046E7
:1091C000FFF71CFF90F90030002B53D029462046B2
:1091D000FFF714FF90F80490B9F12B0F19D8294626
:1091E0002046D7F84CA2FFF709FF94F9353090F9E3
:1091F0000020022BD4BF00210121012BD4BF00236A
:109200000123003A009118BF01224946504602F05E
:1092100043FA631900229A7275B3D4EDC10AB4F807
:109220004822D7F84C0270EEA00A2B46B0EE480A4E
:10923000414602F051FA94F83E33002B31D1224AD4
:10924000069412680127E773906A0268156D1F4A39
:109250000792029309224FF40063CDE9003208AA75
:1092600012E906001A4BA847C8B937F033F8194A73
:1092700002216AE79946B2E729462046FFF7BEFE7B
:1092800090F90030002BC8D0D4EDC10AB4F84822C0
:10929000D4F84C022B46B0EE480A4146C9E784F8A0
:1092A0003E7300230DF1170104F124008DF81730EF
:1092B00029F0F8FC30E700BF8C500908BE500908BF
:1092C000E15009084C5B0020EC2500204590010886
:1092D000FF5009080A5109082DE9F0412DED028BD4
:1092E000002443739DF82030837305460F46904653
:1092F000B0EE408A264647FA04F3DB07E1B210D508
:10930000B0EE480A42462846FFF7F8FE064640B946
:1093100039462846FFF7C6FEBDEC028B3046BDE855
:10932000F0810134032CE6D1F6E70000F8B5002403
:109330002DED028B05460F46B0EE408A42738373D3
:109340002646E1B2B0EE480A3A462846FFF7D6FE76
:109350000134002818BF0646032CF2D1BDEC028B65
:109360003046F8BDF0B500EB81030D46D3F84C1242
:109370009BB0044611B900201BB0F0BD0BA802F051
:1093800007FA6319987A0028F6D10B9A002A48D078
:10939000042AF0D101229A720DAA07CA02AB83E80F
:1093A000070010AA07CA05AF87E8070013AA07CA73
:1093B0009DED180A08AE86E807001A4629462046A1
:1093C0008DED010AFCF792FE3A4629462046FCF74D
:1093D00039FE324629462046FCF746FE9DED010A3D
:1093E00029462046FCF752FE9DF8643083B1294699
:1093F0002046FFF703FE90F900304BB194F9353069
:10940000012B05DD9DF85D2029462046FCF786FEF0
:109410002046FFF75BFE20B9034A537843F004036C
:1094200053700120A8E700BF4C5B00202DE9F041FC
:109430000546884600F513770024012657F8043BBB
:10944000E1B26BB148FA04F3DB0709D52846FFF710
:1094500089FF002857F8040C08BF002602F008F91D
:109460000134032CEAD13046BDE8F0812E4B2DE9C2
:10947000F04F1F68FB6A93F89C8087B00446B8F1F0
:10948000000F38D1DFF8A8A000F5137600F1030B28
:10949000054656F8040BA5EB04095FFA89F9E8B113
:1094A00002F04EF928B19AF8013043F008038AF827
:1094B000013056F8040C02F057F9F8B9637B6BB130
:1094C000AB7A5BB956F8041C684602F07DF9009B44
:1094D000042B03D149462046FFF744FF01355D4583
:1094E000D7D1124B204683F81280FFF7EFFD0546D7
:1094F00030B10123237407B0BDE8F08F8046EDE75B
:10950000237C002BF7D0A37B002BF4D0B86A036830
:109510004FF47A715B689847B86A03689B6B294679
:1095200007B0BDE8F04F1847EC2500202D5B002068
:109530004C5B0020F0B5002587B000F513762C4673
:10954000012756F8041B41B1684602F03DF9009B23
:109550001BB107FA05F31C43E4B20135032DF0D12A
:10956000204607B0F0BD00002DE9F04F2DED028B35
:1095700003270E7C9FED348A91B005468846B94694
:10958000AC5D0134E4B2B4FBF9F303EB4303E41A3A
:10959000E4B205EB8403D3F84C1209B9AC554CE0A6
:1095A00003A802F011F9DDF80CB00BF1FF33022B28
:1095B000F4D8304631F02CF88246304631F02CFF9A
:1095C00000F11B039A4508D2304630F09DFA002086
:1095D00011B0BDEC028BBDE8F08FAC55284698F871
:1095E00010A0FFF7A7FFDDED057A8DF83100FCEE46
:1095F000E77A9DF810208DF8332017EE903A8DF819
:10960000343006AB03CB1B88ADF83D305C221B2306
:10961000CDE90032CDF83500CDF8391009AABF21C7
:1096200050468DED098A8DED0A8A8DED0B8A8DF8F5
:1096300030408DF832B031F055F8013F17F0FF0798
:109640009ED10120C4E700BF000000002DE9F04FCB
:109650000F7CA1B006468846032500EB070999F860
:1096600005400134E4B20323B4FBF3F303EB4303FB
:10967000E41AE4B206EB8403D3F84C1211B989F86A
:1096800005400AE011A802F083F8DDF844A0BAF121
:10969000030F08DCBAF1000FF1DA013D15F0FF0508
:1096A000DDD1012012E0AAF10402032AF5D83846E0
:1096B00030F0AEFF8346384631F0AEFE00F13602A0
:1096C000934506D2384630F01FFA002021B0BDE89D
:1096D000F08F89F80540304698F810B0FFF72AFF60
:1096E000DDF848E0CDF80CE0DDF84CE0CDF810E016
:1096F000DDF850E0CDF814E0DDF854E0CDF818E0E6
:10970000DDF858E0CDF81CE0DDF85CE0CDF820E0B5
:10971000DDF860E0CDF824E03219DDF864E01C9B50
:10972000CDF828E0DDF868E092F80AC09DF87410E2
:109730009DF87520CDF82CE00E93DDF86CE01E9BB3
:109740008DF835008DF83C108DF83D20CDF830E0D7
:109750008DF834408DF836A08DF837C02422CDF82E
:109760003E303623CDE90032C0212C2303AA5846CF
:1097700030F0B8FF91E700007FB58A8B0B464AF2C4
:10978000B9518A4205465FD04AF2BA518A4274D032
:109790004AF2B8518A420BD1474A1268D26A92F80B
:1097A0009C203AB136F096FD444A05212FF0A2FFE5
:1097B000042479E0D3ED007AF5EEC07AF1EE10FAE8
:1097C000F6D49FED3F7AF4EEC77AF1EE10FAEFDCB3
:1097D00093ED017ADFED3B6A1C6993ED030AB0EE6D
:1097E000C77AB4EEE67A93ED027AFCEEE77AB0EE51
:1097F000C77AF1EE10FAB4EEE67A17EE903A54BF5B
:1098000001260026F1EE10FA54BF01220022003C8E
:1098100018BF012413F0FF0110D18DED030A02924D
:10982000FCF7CCFB9DED030A029A234631462846FD
:10983000FFF77CFD0028BBD0002435E013460094E0
:109840003246FFF749FDF5E7D3ED007AF5EEC07A31
:10985000F1EE10FAACD49FED1A7AF4EEC77AF1EE7D
:1098600010FAA5DCFCEEE77A17EE903A13F0FF0150
:1098700008BFFF21FFF7DAFDDCE7D3ED007AF5EE54
:10988000C07AF1EE10FA93D49FED0D7AF4EEC77A18
:10989000F1EE10FA8CDCFCEEE77A17EE904A14F049
:1098A000FF0404D1FFF70EFC204604B070BD214632
:1098B000FFF7F8FBC0E700BFEC2500203C5109088A
:1098C00000007F4300000034F0B58BB00E46144614
:1098D0000746FFF793FB543007C884E8070031467A
:1098E0003846FFF78BFB90ED057ADFED267AB0EE78
:1098F000C77AB4EEE77AF1EE10FA054611D590ED8D
:10990000067AB0EEC77AB4EEE77AF1EE10FA08D52F
:1099100090ED077AB0EEC77AB4EEE77AF1EE10FA7E
:1099200024D431463846FFF769FB016A426A836AEC
:10993000E869D5F814E0D5F818C0099001A8CDF869
:1099400004E0029103920491CDF814C006930792AB
:1099500008930CF0A5FE98B1214601A80CF0F4FC88
:1099600084ED000AC4ED010A84ED021A314638463E
:10997000FFF744FB00F1080120460EF04DFB0120EB
:109980000BB0F0BD000000342DE9F0472DED048B45
:10999000ACB0B0EE608A0546B0EE409A0F46F0EEED
:1099A000418A9046FCF70AFBDFED8B7AB0EEC87A6D
:1099B000B4EEE77AF1EE10FA4BD5B0EEE87AB4EEF9
:1099C000E77AF1EE10FA44D523AC2046FBF73CFED3
:1099D000F7F7AEFD2146F7F78DFB064658BB05F0BD
:1099E00049FA90F8083390F8C42233B1B02303FB4E
:1099F000020393F8A130012B07D84FF0B00909FBFF
:109A0000020090F8A130022B0BD836F063FC734AA9
:109A100003212FF06FFE30462CB0BDEC048BBDE867
:109A2000F08705F027FA90F8C43209FB0300AC3048
:109A30000FC884E80F00DDED257A9FED691AB8EEB6
:109A4000E78ADDED267AF8EEE78A28EE018A68EEED
:109A5000818A04AA03A902A8F0EE680AB0EE480AB7
:109A600003F0D4FC064618B936F034FC5D4ACFE763
:109A70009FED5D7ADDED027A9FED5C8ADFED5C8A19
:109A80008DED068A67EE877A2422002111A8CDED9C
:109A9000057A8DED078A72F0EFF89DED031ADDED82
:109AA000040ADFF858A121EE281A68EEE00AB0EEA9
:109AB000480A11A80CF014FE05A911A80CF044FCEA
:109AC000242200211AA8CDED060A8DED071A8DED8E
:109AD000050A72F0D1F8F7F72BFD90ED810A8DEDB4
:109AE000010AF7F725FD29EE281AD0ED820A9DED2F
:109AF000010A1AA80CF0F4FD1AA923A80CF012FD13
:109B000005A923A80CF020FC4FF000098DED050AF3
:109B1000CDED060A8DED071A95F822305FFA89F42B
:109B2000A3427FF678AF1FB127FA04F3DB071AD5FB
:109B30002B1993F92C32B3B1B8F1000F0DD0214697
:109B40002846FCF7C5FC88B936F0C4FB294A2346F1
:109B500003212FF0CFFD00265DE721462846FCF7C4
:109B600031FB0028EBD109F10109D5E708AA21460C
:109B700028468DED088A8DED098A8DED0A8AFFF75A
:109B8000A3FE20B936F0A6FB1B4A2346E0E708A94E
:109B900005A80EF0F1F90BAA214628468DED0B0A17
:109BA000CDED0C0A8DED0D1AFCF7A0FA9AE807002E
:109BB0000EAB83E807001A4621462846FCF742FA16
:109BC00023AA214628468DED238A8DED248A8DED2A
:109BD000258AFCF749FAC6E70000003460510908FD
:109BE00095BFD6337B51090800007A44000000007D
:109BF00035FA8E3C90510908A4510908F0FD080877
:109C00000120704701207047436898687047000042
:109C1000406803689B6C184710B5054B0360044609
:109C2000806A10B103685B689847204610BD00BF8A
:109C30008C520908406803685B6A184733B46C4665
:109C4000406884E80C0003689D6A94E80C00AC4608
:109C500002B030BC6047000010B50446FFF7DCFFDF
:109C60002046FBF7C7FF204610BD0000406808F003
:109C70004FBB0000406808F0ADBB00004068012306
:109C800008F0A8BB4068002308F080BB90F844208F
:109C9000D20705D590F8421000F12C02FFF780B8EA
:109CA00070470000F8B504461E460F461546FEF7FD
:109CB00077FF084B23600023E3622363636394F818
:109CC0004430A76265F3410384F8436084F844306C
:109CD0002046F8BD8C52090810B50D4B836304462D
:109CE000806A036898221B690021984770B1A06AB6
:109CF000036820221B690121984738B1A06A0368D4
:109D0000BDE810401B69012202211847002010BD48
:109D1000C5DC6A3F37B50446806A03686A469D68B9
:109D200003210623A847D0B1BDF80020BDF80410D8
:109D300052BA95B249BAB5F5704F0BB211D013F5BE
:109D4000805F0ED0BDF802305BBA9DB2B5F5704FA2
:109D500007D052425B42A287E187A4F8403003B0AB
:109D600030BD0020FBE70000806A036801221B6908
:109D70000221184730B585B00446FFF7CBFF0546F2
:109D80002046FFF7F1FF6DB3B4F93C3094ED0E0AB5
:109D900006EE903AB4F93E3007EE103AB4F940308E
:109DA00007EE903AF8EEE66AB8EEC77AF8EEE77A90
:109DB00001A8CDED016A8DED027ACDED037A0EF0AA
:109DC00045F994F842102046FFF768F818B10221CF
:109DD00001A80EF0D1F994F842200E2301A92046E3
:109DE000FFF7CCF805B030BDFFF7C4BF13B5806AEC
:109DF000036801AA9C680A210323A04738B10549DA
:109E0000032201A871F0DEFEB0FA80F0400902B032
:109E100010BD00BFC45109082DE9F84300252DED00
:109E2000028BDFF888819FED5D8A04462E462F461F
:109E3000A06A036811221B69002101379847002896
:109E40007BD0D8F80090D9F82800036832215B68ED
:109E50009847A06A036860221B690121984700287F
:109E60006BD0A06A036801221B6902219847002871
:109E700063D0D9F82800036832215B6898472046F0
:109E8000FFF748FF002858D00135022FEDB256DD0C
:109E9000B4F93C309FED425A9FED426A07EE903A8A
:109EA000F8EEE77AC5EE276AF0EEE66AF4EEC66AE7
:109EB000F1EE10FA41DDF4EEC86AF1EE10FA3CD58D
:109EC000B4F93E30DFED385A07EE903AF8EEE77A13
:109ED00085EEA77AB0EEC77AB4EEC67AF1EE10FA44
:109EE0002BDDB4EEC87AF1EE10FA26D5B4F9403085
:109EF00005EE903AF8EEE55AC5EE257AF0EEE77AEF
:109F0000F4EEC67AF1EE10FA17DDF4EEC87AF1EE4F
:109F100010FA12D594ED0B6A76EE266A0136C4ED7E
:109F20000B6AD4ED0C6A36EE877A84ED0C7A94EDE8
:109F30000D7A77EE277AC4ED0D7A192F02D0052E0F
:109F40007FF476AFA06A036810221B69002198474E
:109F5000052E18D1D4ED0B6AF1EE047A86EEA77ABD
:109F60000120D4ED0C6A84ED0B7A86EEA77AD4ED4D
:109F70000D6A84ED0C7A86EEA77A84ED0D7ABDEC3D
:109F8000028BBDE8F8834FF07E53052DE362236317
:109F9000636394BF00200120F1E700BFCDCCAC3F4C
:109FA00000002E443333333F00002244EC250020D0
:109FB000F0B50446806A036885B05B69984705463A
:109FC00048B9504B50491B68986903681B6898470B
:109FD000284605B0F0BD03689B689847A06A0368EF
:109FE0000A21DB6A9847A06A03689B69984760B9B1
:109FF000444B46491B68986903681B6898472B685F
:10A000002846DB6898470025E2E72046FFF7EEFE8A
:10A010000028F4D02046FFF7FFFE30B9394B3C4909
:10A020001B68986903681B68E8E72046FFF754FE41
:10A030000028E4D0A06A0368DB69984730B9314B47
:10A0400034491B68986903681B68D7E794F8443063
:10A05000A06A43F0010384F8443003680321DB6AFB
:10A0600098472B682846DB689847236820469B68FA
:10A070009847A06A036807215B6A9847A06A03684B
:10A080009B6A984704F1420201462046FEF7D6FE3D
:10A09000054600289CD0A06A94F8421003680191FC
:10A0A0009B6A9847019902462046FEF7CBFE94F83A
:10A0B000432094F842102046FEF7FAFE94F844300C
:10A0C0009B0705D594F8421001222046FEF7CEFEEC
:10A0D000A06A029403681E6A0F4B039304AB13E952
:10A0E0000C0043F21541B047064BA06A1B689E69FD
:10A0F00033681F6803689B6A9847084902463046E0
:10A10000B84765E7EC250020C8510908EE51090859
:10A110001452090839520908E99D010867520908D3
:10A1200010B5084B036004460023086860600B60AC
:10A13000037A03F00703022B02D1C02108F016FABC
:10A14000204610BDA452090810B5044B044640F83F
:10A15000043BF9F7CFFD204610BD00BFA45209080B
:10A1600010B50446FFF7F0FF2046FBF743FD2046FD
:10A1700010BD0000F7B503680E4617461BB9002452
:10A18000204603B0F0BD0022026008200193FBF7D7
:10A1900029FD054610B101A9FFF7C2FF01A8F9F793
:10A1A000A9FD002DEBD04820FBF71CFD044600283C
:10A1B000E5D029463B463246FFF774FD2046FFF7BF
:10A1C000F7FE05460028DBD1236820465B689847E8
:10A1D0002C46D5E790F82D100022FEF7E1BD0000D7
:10A1E000F0B50446806A036889B05B6A98470368E3
:10A1F0009B689847A06A03680A219B6C9847A06AED
:10A2000001230DF11702002108F0E4F8002838D0EE
:10A210009DF81730082B34D14E4F0525002301221D
:10A22000A06A322108F0B2F83B689B6A1A6852684B
:10A2300040B90A2118469047013D15F0FF05EDD1C0
:10A2400045481CE018461421904706AEFF238DF8C0
:10A250001830A06A01233246322108F0BBF80028EA
:10A26000EAD09DF8183013F00103E5D1A06A0393FA
:10A270000822322108F08AF8039B58B937484CF07D
:10A2800019F8A06A03685B6A98470368DB68984717
:10A2900000255CE0A06A03931A46342108F076F8A2
:10A2A0000028EBD0039BA06A2422412108F06EF81D
:10A2B0000028E3D0039BA06A0822312108F066F849
:10A2C0000028DBD0A06A036803219B6C9847A06A32
:10A2D00003685B6A98470368DB689847A06A1021A7
:10A2E00008F016F8A36A04F12D0299682046FEF7DB
:10A2F000A5FD054658B3A36A94F82D109A68204628
:10A30000FEF7A0FDA36A16481A7A597A00919B6855
:10A310001449D2084BF0CEFF94F82C2094F82D105D
:10A320002046FEF7C5FD94F82E302BB194F82D1081
:10A3300001222046FEF79AFDA06A03689F6A0A4B35
:10A340000694079396E80C0042F21071B84728462D
:10A3500009B0F0BDEC25002034530908D452090897
:10A360000B53090803530908F5A3010810B586B07B
:10A3700004460123806A0DF10302102108F02AF837
:10A3800098B39DF80330DB072FD5A06A062301AAF6
:10A39000112108F01FF840B3BDF904309FED146A95
:10A3A00094F82D2006EE903ABDF9063007EE103AEB
:10A3B000BDF808305B421BB207EE903AF8EEE66A51
:10A3C000B8EEC77AF8EEE77A66EE866A27EE067A86
:10A3D00067EE867A0A2303A92046CDED036A8DED48
:10A3E000047ACDED057AFEF7C9FD06B010BD00BFB9
:10A3F00085EBC13FFFF7BABFF7B503680D461646B8
:10A400001BB90024204603B0F0BD002707603020B0
